:020000040800F2
:1000000000000110810F04087BE5030821BF0008F0
:1000100085100408851004088510040800000000FD
:10002000000000000000000000000000BDEB03081D
:10003000BBEB030800000000B9EB030831D5000852
:10004000851004088510040885100408851004082C
:100050008510040885100408554A0108814B0108E1
:10006000454B0108094B0108CD4A0108119E0008C3
:10007000019E0008F19D0008E19D0008D19D000847
:10008000BD9D0008A99D000885100408851004087E
:10009000851004088510040885100408914A010899
:1000A00085100408851004088510040885100408CC
:1000B0002DCC00081DCC0008851004088DB7000861
:1000C00093B7000881B7000887B7000885100408B7
:1000D000851004089DD7000885100408FDD6000887
:1000E0001B4A010885100408CDEC0308DDCB00088D
:1000F000EDCB000885100408FDCB0008959D000895
:1001000085100408851004080DCC0008851004082B
:100110005DD6000885100408890402086D040208F1
:10012000819D00086D9D0008599D0008459D0008AF
:10013000319D000885100408851004088510040806
:100140008510040885100408851004087DE503085F
:100150001D9D0008099D0008F59C0008BDD50008FC
:1001600075B700087BB700088510040885100408DF
:1001700085100408851004088510040885100408FB
:08018000851004088510040835
:08018800180B04000100000047
:1001900002020300941F0020901F002000000000B6
:1001A000000000000E020200D4240020D824002009
:1001B000000000004006000816000800EC240020A3
:1001C0000425002000000000420600081D00010078
:1001D000C826002054270020000000004A0600081E
:1001E00027000400E8260020582700200000000017
:1001F0004C0600080A020A008827002098270020E1
:10020000000000005006000801010400E42700205F
:10021000843B0020000000000000000008020900EC
:10022000A83A0020883B002000000000BD390108EA
:1002300006020C00203B0020943B00200000000040
:10024000C93F010807020200543B0020A03B0020E8
:10025000000000005A06000802000C002C3B0020A1
:10026000A43B00200000000000000000F701060091
:100270009C3A0020B03B0020000000005C06000813
:100280002C00100008400020F83F00200000000073
:10029000112B02082B0024003C40002018400020B5
:1002A00000000000E12A020829005000303F002031
:1002B000604000200000000000000000030001007A
:1002C000644200206C42002000000000000000009A
:1002D000031233008F4600205C460020000000001F
:1002E0006406000825005A00A845002002460020A8
:1002F0000000000000000000F6110C009C450020EA
:1003000090450020000000009806000815007000CD
:10031000B044002020450020000000000000000044
:100320002A006000F043002050440020000000003C
:10033000A91503081E0004004C470020844A002031
:1003400000000000A406000822000C00EC49002078
:10035000884A002000000000A80600081B00F400E6
:10036000085000208460002000000000E1A0020886
:1003700026000E0088610020786100200000000047
:100380006DD302080B201000B851002098610020A6
:1003900000000000B406000803010A000862002003
:1003A0001462002000000000C406000805100600CA
:1003B00058630020A464002000000000D00600085C
:1003C0000E20EA0038620020AC640020000000002B
:1003D00015160308130004006C63002098650020C4
:1003E00000000000D806000802010300236200207C
:1003F0009C6500200000000005050208012008009F
:10040000A06B0020C06B002000000000DC0600088C
:100410001A000800846B0020C86B00200000000058
:10042000E4060008140002006C6E0020706E0020CC
:1004300000000000EC060008100003005C6E0020C5
:10044000746E002000000000EE0600082800100076
:100450004C6E0020786E002000000000FDB80208FD
:10046000230010003C6E0020886E00200000000079
:1004700015B9020819000500346E0020986E00209E
:1004800000000000F2060008F8110100306E0020A4
:10049000A06E002000000000F80600080001040023
:1004A0002C6E0020A46E002000000000FA06000858
:1004B0002F001100186E0020A86E00200000000020
:1004C000FE06000809020100196F0020486F002095
:1004D00000000000100700083400100020820020F7
:1004E000F482002000000000D115030811000C0068
:1004F000B8760020048300200000000045050208B3
:1005000018102C00507600201083002000000000FE
:10051000DD3402080D003C007C7600203C83002086
:1005200000000000C9AF0308FA0102005C6F002060
:100530007883002000000000A5B80008FE01090033
:10054000A0850020B48500200000000091B80008BC
:10055000FD012400489300206C930020000000005F
:100560003D39010806001600C08F0020909300203E
:100570000000000035160308FB010100FC8E00207E
:10058000A89300200000000089B80008FC010900C1
:10059000C88D0020AC9300200000000055B8000872
:1005A0000A1012009C8D0020B8930020000000006B
:1005B000120700081F000E00209A0020F49B002064
:1005C000000000002407000805020100089A00202E
:1005D000049C0020000000003207000812200C00DC
:1005E000289C0020E09C0020000000003407000848
:1005F0000C002400349C0020EC9C00200000000033
:10060000DD04020800020500089C0020109D002067
:10061000000000000000000004008000ACB00020DA
:10062000E8B900200000000000000000F90104000B
:1006300090A5002068BA002000000000AD39010834
:100640000000C40900001901282800002003000050
:1006500000004A01B400D6010000013C0000010086
:10066000000000000000000000000000000000008A
:10067000000000000000000000000000000000007A
:10068000000000000000000000000000000000006A
:100690000000000000000100000000000000000059
:1006A0000000000000000100C800141E01006400EA
:1006B0002C0128002B21231E6400020000000100F1
:1006C0000A012900040101006C160000000000006E
:1006D000200003010000000008000000E80364009F
:1006E000040A00017E05EA05B4053200030000019A
:1006F0000500000028010000040090010000000037
:1007000000000000000000000000000000000000E9
:100710002E0000300100005A0000000090012C0162
:10072000C800640000000000000001000000000597
:10073000000000000000000100055245564F000077
:10074000500100000700000002000000000000004F
:10075000000000000102030406070809010100006F
:10076000985B0408F0870408000000000000000007
:10077000A85B0408B05B0408000000000120000032
:10078000B45B0408BC5B04080000000001400000EA
:10079000C05B04084473040800000000012000004E
:1007A000CC5B0408D85B04080000000004000000D3
:1007B000DC5B0408E85B04080000000004000000A3
:1007C000EC5B04089C8604080000000001000000A7
:1007D00002010000685E0C00FF0000000000803F86
:1007E0000000803F0000000000000000000000004A
:1007F0000000803F6C2E0408050804000000000083
:10080000A04F0408204B04088C4F0408000000008F
:10081000982E040805080A0000000000A04F0408F4
:10082000204B0408444B0408000000000101D601DD
:10083000B92402080000000000000000FFFFFFFFD5
:10084000000001FFFF0000000001010101000000A5
:1008500001000000447D04080000000000000000CA
:1008600019050208A0860100040000000000000035
:100870000000000000000000000000000000000078
:100880000000000000000000B88F0408847904080C
:1008900000000000A18001087D00000006000000AB
:1008A0000000000000000000000000000000000048
:1008B000000000000000000000000000F4870408B1
:1008C0000000000000000000C1110108E803000062
:1008D0000300000000000000000000000000000015
:1008E0000000000000000000000000000000000008
:1008F000FC870408000000000000000071170308D6
:1009000010270000030000000000000000000000AD
:1009100000000000000000000000000000000000D7
:10092000000000000888040800000000692902088F
:100930002D160108204E00000500000000000000F8
:1009400000000000000000000000000000000000A7
:100950000000000000000000D07E0408000000003D
:10096000000000009DD800081027000001000000D2
:100970000000000000000000000000000000000077
:100980000000000000000000000000000C880408C7
:10099000000000000000000021B80008E80300008B
:1009A0000500000000000000000000000000000042
:1009B0000000000000000000000000000000000037
:1009C00018880408000000000000000079070208F1
:1009D000204E0000030000000000000000000000A6
:1009E0000000000000000000000000000000000007
:1009F000000000002888040800000000000000003B
:100A000081050208204E00000300000000000000E5
:100A100000000000000000000000000000000000D6
:100A200000000000000000003888040800000000FA
:100A30000000000001BC0008400D0300030000009E
:100A400000000000000000000000000000000000A6
:100A5000000000000000000000000000087E040804
:100A60000000000000000000DDBA030810270000AD
:100A70000100000000000000000000000000000075
:100A80000000000000000000000000000000000066
:100A9000A079040800000000000000002DB3020847
:100AA000102700000300000000000000000000000C
:100AB0000000000000000000000000000000000036
:100AC000000000004888040800000000000000004A
:100AD0004D100108A0860100010000000000000088
:100AE0000000000000000000000000000000000006
:100AF00000000000000000009079040800000000E1
:100B0000000000006D0F010850C30000010000004C
:100B100000000000000000000000000000000000D5
:100B200000000000000000000000000050880408E1
:100B30000000000000000000D50A0108A8610000C4
:100B400001000000000000000000000000000000A4
:100B50000000000000000000000000000000000095
:100B60005C880408000000000000000001DD0308AC
:100B7000A08601000100000000000000000000004D
:100B80000000000000000000000000000000000065
:100B900000000000D87E04080000000000000000F3
:100BA000EDDD0008A00F00000100000000000000C3
:100BB0000000000000000000000000000000000035
:100BC0000000000000000000688804080000000029
:100BD00000000000F1D5020810270000010000000D
:100BE0000000000000000000000000000000000005
:100BF000000000000000000000000000307E04083B
:100C0000000000000000000081090208A00F0000A1
:100C100001000000000000000000000000000000D3
:100C200000000000000000000000000000000000C4
:100C30003C7F0408000000000000000079C00308A9
:100C4000102700000100000000000000000000006C
:100C50000000000000000000000000000000000094
:100C6000000000006C790408000000000000000093
:100C7000B50803081A410000010000000000000050
:100C80000000000000000000000000000000000064
:100C9000000000000000000074880408000000004C
:100CA0000000000029FF0308400D030000000000C1
:100CB0000000000000000000000000000000000034
:100CC0000000000000000000000000007C88040814
:100CD0000000000000000000D1D00108400D03001A
:100CE0000000000000000000000000000000000004
:100CF00000000000000000000000000000000000F4
:100D000084880408000000000000000031DA0308B5
:100D1000A0860100030000000000000000000000A9
:100D200000000000000000000000000000000000C3
:100D3000000000002D202D2D202D2D2D2D202D2DBE
:100D40002D2D000000000000000000000000000049
:100D5000000000000000000001020304010203047F
:100D60000607080920700020702D720000000000A6
:100D700000000000CC130020FFFFFFFFFA0000007E
:100D80000100000001000000F888040800000000D5
:100D9000000000000000000000000000E3880408DC
:100DA00004000000FB5F03080000000000000000DA
:100DB000008904080100000000000000000000009D
:100DC00000000000000000000D0000000000000016
:100DD00000000000000000005EB100200100C40916
:100DE000000000005CB100200100C4090000000008
:100DF0005AB100200100C4090000000058B10020D1
:100E00000100C4090000000054B100200100C40921
:100E10000000000056B100200100C40900000000DD
:100E200052B100200100C4090000000050B10020B0
:100E30000100C409000000000000000000000000E4
:100E400048060020E26100209CFF2C010000000009
:100E5000C81400200A000000444B0408BC6E0020A7
:100E6000E0150C1700000000CA1400200800000064
:100E7000204B0408C914002005000000A04F0408FE
:100E8000BE6E0020020000005C4B04085E63002080
:100E90000100FF7F010000005763002002000000F6
:100EA000684B04082C62002003000000784B040803
:100EB0002B62002003000000784B04082A63002006
:100EC0000000F40101000000286300200000F4018C
:100ED00001000000266300200000F4010100000072
:100EE000246300200000F4010100000022630020C0
:100EF00000FF010042630020E803D0070A00000061
:100F000040630020006401000A0000003C630020F0
:100F1000006401003B630020006401004163002085
:100F2000006401000A0000003A6300200064010030
:100F30000A0000003F630020006401000A00000076
:100F40003E630020006401000A0000003D630020B1
:100F5000006401000A0000003963002000FF010066
:100F60000A0000003863002000FF01000A000000B2
:100F7000346200200000F401010000003262002011
:100F80000000F40101000000306200200000F401C4
:100F9000010000002E6200200000F40101000000AA
:100FA000346300201400E8030100000032630020D5
:100FB000E8033075010000003163002000C8010023
:100FC0003063002000C801002F63002000C801002A
:100FD0002E630020006401000A0000002D63002041
:100FE00000FF01000A0000004D63002000C801005E
:100FF0004C63002000C801004B63002000C80100C2
:101000004A63002000C801004963002000C80100B5
:101010004863002000C801004763002000C80100A9
:101020004663002000C801004563002000C801009D
:1010300028890408000000000000000000000000F3
:1010400000000000388904080900000000000000CA
:10105000EC0600200400000040890408090000009C
:1010600000000000E0060020040000001C8D0408C1
:101070000900000000000000D40600200400000069
:10108000488904080900000000000000C80600208C
:10109000040000004C890408090000000000000062
:1010A000BC06002004000000548904080900000068
:1010B00000000000B0060020040000005C89040865
:1010C0000900000000000000A40600200400000049
:1010D0006489040809000000000000009806002050
:1010E0000400000000890408010000000000000066
:1010F0000000000000000000000000000D000000E3
:101100000000000000000000000000006C8A0408DD
:1011100000000000000000000000000000000000CF
:101120007C8A040805000000000000002A620020FC
:101130000000000000890408010000000000000019
:101140000000000000000000000000000D00000092
:10115000000000000000000000000000848A040875
:10116000000000000000000000000000000000007F
:10117000F08704080000000000000000F4050020D3
:1011800004000000908A04080C0000005D60030861
:101190004007002000000000249204080C0000001A
:1011A000655A03083407002000000000948A0408F0
:1011B0000C000000495A0308280700200000000026
:1011C0009C8A040808000000000000001C070020A2
:1011D00004000000A48A04080C00000095590308CC
:1011E0001007002000000000AC8A0408090000007D
:1011F000000000000407002004000000B48A040876
:10120000030000003D050308F80600200000000070
:101210000089040801000000000000000000000038
:1012200000000000000000000D00000000000000B1
:101230000000000000000000B88A04080000000060
:10124000000000000000000000000000C88A040840
:101250000C00000000000000580700200000000003
:10126000D08A04080A00000000000000C8630020C3
:1012700000000000DC8A04080A00000000000000F2
:10128000D063002000000000E48A04080A00000087
:1012900000000000D863002000000000EC8A040871
:1012A00008000000000000004C07002000000000C3
:1012B000F48A04080400000071060308000000001E
:1012C0000000000000890408010000000000000088
:1012D0000000000000000000000000000D00000001
:1012E000000000000000000000000000008B040867
:1012F00000000000000000000000000000000000EE
:10130000148B04080C00000000000000700700208F
:1013100000000000248B040804000000850303087B
:1013200000000000000000002C8B04080C000000EE
:10133000000000006407002000000000408B04084B
:101340000400000065030308000000000000000026
:1013500000890408010000000000000000000000F7
:1013600000000000000000000D0000000000000070
:101370000000000000000000488B0408000000008E
:101380000000000000000000000000005C8B04086A
:101390000700000000000000AC0700200000000073
:1013A000688B04080800000000000000A00700206F
:1013B00000000000748B040808000000000000001A
:1013C0009407002000000000808B04080800000043
:1013D0000000000088070020000000008C8B04083B
:1013E00008000000000000007C0700200000000052
:1013F0000089040801000000000000000000000057
:1014000000000000000000000D00000000000000CF
:101410000000000000000000988B0408000000009D
:10142000000000002706002000000000A48B040834
:101430000B00000000000000240800200000000055
:10144000AC8B04080B00000000000000180800200E
:1014500000000000B88B04080B0000000000000032
:101460000C08002000000000C48B04080B000000E2
:10147000000000000008002000000000D08B0408DD
:101480000B00000000000000F40700200000000036
:10149000DC8B04080B00000000000000E8070020BF
:1014A00000000000E48B04080B00000000000000B6
:1014B000DC07002000000000F08B0408070000009B
:1014C00000000000D407002000000000F88B040892
:1014D0000700000000000000CC0700200000000012
:1014E000048C04080B00000000000000C00700206E
:1014F00000000000108C040808000000000000003C
:10150000B40700200000000000890408010000006A
:1015100000000000000000000000000000000000CB
:101520000D000000000000000000000000000000AE
:101530001C8C0408000000000000000000000000F7
:1015400000000000308C04080800000000000000CB
:1015500054080020000000003C8C04080800000033
:10156000000000004808002000000000488C04082B
:1015700008000000000000003C08002000000000FF
:10158000548C04080800000000000000300800200F
:1015900000000000008904080100000000000000B5
:1015A0000000000000000000000000000D0000002E
:1015B0000000000000000000000000005C8C040837
:1015C00000000000000000002406002000000000D1
:1015D0006C8C04080B000000000000009C08002038
:1015E00000000000788C04080B00000000000000E0
:1015F0009008002000000000848C04080700000010
:10160000000000008808002000000000908C040802
:10161000070000000000000080080020000000001B
:101620009C8C0408070000000000000078080020DF
:1016300000000000A88C0408080000000000000062
:101640006C08002000000000B08C040808000000B6
:10165000000000006008002000000000008904086D
:101660000100000000000000000000000000000079
:10167000000000000D00000000000000000000005D
:1016800000000000B88C040800000000000000000A
:101690002406002000000000C48C0408070000009D
:1016A00000000000E808002000000000CC8C0408C6
:1016B0000700000000000000E0080020000000001B
:1016C000D48C04080700000000000000D8080020A7
:1016D00000000000DC8C040807000000000000008F
:1016E000D008002000000000E48C0408070000007F
:1016F00000000000C808002000000000EC8C040876
:101700000700000000000000C008002000000000EA
:10171000F48C04080700000000000000B808002056
:1017200000000000FC8C040807000000000000001E
:10173000B008002000000000048D0408070000002D
:1017400000000000A8080020000000000089040834
:101750000100000000000000000000000000000088
:10176000000000000D00000000000000000000006C
:1017700000000000000000005DFF0208F0080020EB
:10178000286200201B000000884B0408276200200C
:101790000A3201002662002001FA010022620020C4
:1017A00000C8010020620020E803D007010000000B
:1017B0005245564F0000000073FF0208390303082A
:1017C000CC090020D1590308000000001C0A0020A9
:1017D00051060308B9010308F80A002095FF020822
:1017E00000000000AC0B00201D000308EDFF020804
:1017F000380C0020A5000308E9000308D80C0020DD
:101800003663002001030100C9FF0208A5FF02089A
:10181000F00D00204D000308A50303087C0E0020F6
:1018200019010308FD030308440F00202C63002066
:10183000010301000C8D04080000000000000000FE
:101840000000000000000000188D040808000000DF
:10185000000000006410002000000000208D04083B
:1018600007000000000000005C10002000000000E5
:10187000308D040807000000000000005410002014
:10188000000000003C8D040807000000000000007C
:101890004C10002000000000488D04080C000000DF
:1018A000000000004010002000000000548D0408DB
:1018B000030000003D050308341000200000000074
:1018C0000089040801000000000000000000000082
:1018D00000000000000000000D00000000000000FB
:1018E00000000000000000005C8D04080000000003
:1018F0000000000000000000000000006C8D0408E3
:101900000A00000000000000505C04080000000015
:10191000748D04080A00000000000000785B0408D1
:10192000000000007C8D04080A0000000000000098
:101930004E63002000000000848D04080A000000AF
:101940000000000070100020000000000089040862
:101950000100000000000000000000000000000086
:10196000000000000D00000000000000000000006A
:10197000000000008C8D0408000000000000000042
:101980000000000000000000A08D0408030000001B
:101990003D0503089010002000000000AC8D0408F5
:1019A000030000003D050308CC14002000000000E7
:1019B000B48D0408030000003D05030884100020D6
:1019C00000000000BC8D0408030000003D05030872
:1019D00078100020000000000089040801000000C9
:1019E00000000000000000000000000000000000F7
:1019F0000D000000000000000000000000000000DA
:101A0000C88D040800000000000000000000000075
:101A100000000000D48D04080700000049040308FA
:101A2000EC10002000000000B88F04080300000044
:101A30003D050308E010002000000000E08D0408D0
:101A4000030000003D050308D41000200000000042
:101A5000E88D0408030000003D050308C8100020BD
:101A600000000000F08D0408070000002D040308AA
:101A7000C010002000000000409204080300000095
:101A80003D050308B410002000000000FC8D040890
:101A9000030000003D050308A8100020000000001E
:101AA000088E0408030000003D0503089C10002078
:101AB0000000000000890408010000000000000090
:101AC0000000000000000000000000000D00000009
:101AD00000000000000000000000000025FF0208D8
:101AE000EDFE0208F410002085010308000000004C
:101AF000A8110020000000000000000034120020A7
:101B00005D01030865040308C0120020148E040858
:101B100000000000000000000000000000000000C5
:101B2000208E0408030000003D050308C0130020B8
:101B300000000000288E0408030000003D05030893
:101B4000B413002000000000348E040803000000DD
:101B50003D050308A813002000000000408E040883
:101B6000030000003D0503089C1300200000000056
:101B7000488E04080200000021070308000000004E
:101B800000000000508E0408020000002107030836
:101B900001000000000000005C8E0408020000004C
:101BA0002107030802000000000000000000000000
:101BB0000D00000000000000000000000000000018
:101BC0000000803F00000000000000000000000056
:101BD0000000803F00000000000000000000000046
:101BE00000000000000000000000000000000000F5
:101BF00000000000000000000000803F0000000026
:101C0000000000000000000001010100815A0308EB
:101C10000000000040160020789204080000000038
:101C2000000000000000000000000000F087040831
:101C30000000000000000000801A002004000000E6
:101C4000249204080C00000011030308681A002005
:101C500000000000948A04080C000000E902030858
:101C60005C1A0020000000009C8A040808000000A4
:101C700000000000501A002004000000A48A04089C
:101C80000C000000C9FE0208441A002000000000F9
:101C9000B48A0408030000003D050308381A002038
:101CA0000000000088920408030000003D050308BE
:101CB0002C1A002000000000008904080100000028
:101CC0000000000000000000000000000000000014
:101CD0000D000000000000000000000000000000F7
:101CE00078920408000000000000000000000000DE
:101CF00000000000F0870408000000000000000061
:101D0000801A002004000000CC91040803000000A9
:101D100081600308201A002008000000A48A04083B
:101D20000C000000C9FE0208441A00200000000058
:101D3000B48A0408030000003D050308381A002097
:101D40000000000088920408030000003D0503081D
:101D50002C1A002000000000008904080100000087
:101D60000000000000000000000000000000000073
:101D70000D00000000000000000000000000000056
:101D80009092040800000000000000000000000025
:101D900000000000F08704080000000000000000C0
:101DA000801A002004000000D49104080300000001
:101DB0003D050308741A0020000000000089040893
:101DC0000100000000000000000000000000000012
:101DD000000000000D0000000000000000000000F6
:101DE00000000000C26E002088136F170100000081
:101DF000C46E002088136F170000000028910408AB
:101E000000000000000000000000000000000000D2
:101E1000389104080800000000000000B0160020FF
:101E200004000000449104080800000000000000C5
:101E3000A416002000000000B48A0408040000007A
:101E4000C1600308000000000000000000890408D1
:101E50000100000000000000000000000000000081
:101E6000000000000D000000000000000000000065
:101E700000000000C06E002088136F1701000000F2
:101E8000009A002088136F1700000000E15A030831
:101E900000000000BC160020186F002001000000A8
:101EA000604F0408029A0020010000006C4F0408F3
:101EB000F899002002000000744F0408A6B1002029
:101EC0000000000000000000A4B10020000000009D
:101ED00000000000A2B1002000000000000000008F
:101EE000A0B1002000000000000000009EB1002012
:101EF00000000000000000009CB100200000000075
:101F000000000000001D0020000000000000000094
:101F1000BF6E002002000000804F04088491040876
:101F200000000000000000000000000000000000B1
:101F3000389104080800000000000000401700204D
:101F400004000000449104080800000000000000A4
:101F50003417002000000000B48A040804000000C8
:101F6000B55A0308000000000000000000890408C2
:101F70000100000000000000000000000000000060
:101F8000000000000D000000000000000000000044
:101F90000000000094910408000000000000000010
:101FA0000000000000000000A49104080C000000E4
:101FB000910203087017002004000000B09104088B
:101FC0000C00000039020308641700200400000020
:101FD000BC9104080C0000005D02030858170020A3
:101FE00000000000C891040803000000A16003087D
:101FF0004C17002008000000D491040803000000E2
:102000003D050308741A0020000000000089040840
:1020100001000000000000000000000000000000BF
:10202000000000000D0000000000000000000000A3
:1020300000000000F8880408000000000000000014
:102040000000000000000000DC9104080400000013
:10205000DD600308000000000000000000890408A3
:10206000010000000000000000000000000000006F
:10207000000000000D000000000000000000000053
:10208000000000002C920408000000000000000086
:102090000000000000000000D07F04080C000000D9
:1020A00000000000D0170020040000003C9204084B
:1020B0000800000000000000C41700200400000019
:1020C000489204080800000000000000B817002033
:1020D0000400000050920408080000000000000006
:1020E000AC1700200400000058920408080000000B
:1020F00000000000A0170020040000006092040807
:1021000008000000000000009417002004000000F8
:1021100068920408080000000000000088170020F2
:102120000400000070920408080000000000000095
:102130007C17002004000000008904080100000052
:10214000000000000000000000000000000000008F
:102150000D00000000000000000000000000000072
:10216000CD5A030800000000DC170020000000002A
:1021700000000000541800200000000000000000D3
:10218000F4180020FE990020040000008C4F040881
:10219000FC990020E0150C1700000000FB990020BE
:1021A00008000000204B0408FA99002005000000F8
:1021B000A04F0408000000000000000044190020A7
:1021C0002D202D2D202D2D2D2D202D2D2D000000ED
:1021D00000000000000000000000000000000000FF
:1021E00000000001000000000000000000000000EE
:1021F00093E403084DE40308FBEB03080000000030
:10220000B5E00308C1E203083DE3030829E203083F
:102210000000000000000000A9E003088DE00308B2
:102220008BE0030889E0030883E0030881E00308EA
:1022300087E0030885E003089DE003088FE00308BA
:1022400001E2030815E20308EDE10308D9E1030800
:10225000C5E1030800600240106002400000000079
:10226000000B000000002000000000000000000043
:10227000006002402860024000000000060C0000E0
:10228000000020000000000000000000006002408C
:102290004060024000000000100D0000000020001F
:1022A0000000000000000000006002405860024092
:1022B00000000000160E00000000200000000000DA
:1022C000000000000060024070600240000000005A
:1022D000200F0000000020000000000000000000AF
:1022E00000600240886002400000000026100000EC
:1022F000000020000000000000000000006002401C
:10230000A06002400000000030110000000020002A
:10231000000000000000000000600240B8600240C1
:1023200000000000362F0000000020000000000028
:102330000000000000640240106402400000000041
:102340000038000000004000000000000000000015
:1023500000640240286402400000000006390000CA
:102360000000400000000000000000000064024087
:102370004064024000000000103A000000004000ED
:1023800000000000000000000064024058640240A9
:1023900000000000163B00000000400000000000AC
:1023A0000000000000640240706402400000000071
:1023B000203C000000004000000000000000000081
:1023C00000640240886402400000000026440000CF
:1023D0000000400000000000000000000064024017
:1023E000A0640240000000003045000000004000F2
:1023F000000000000000000000640240B8640240D9
:102400000000000036460000000040000000000010
:10241000000000000100000000FFFF0000000000BD
:10242000AA550501000001AA550B010000AA550795
:10243000010000AA55090200000000000100000090
:10244000C012AA5503009F000403090412010002F0
:102450000202004083044057000201020301000011
:1024600009024300020100C0320904000001020217
:1024700001000524001001052401000104240202CA
:102480000524060001070582030800FF0904010076
:10249000020A000000070501024000000705810252
:1024A00040000000FF00000051F7020869E3030844
:1024B00005F20208F5E0030829E5030805E1030831
:1024C00021E10308E7E00308D9E003080000000069
:1024D000000000000000803F01000000A01D00205F
:1024E00000000000000000000000000000000000EC
:1024F00000000000000000000000000000000000DC
:1025000000000000000000000000000000000000CB
:1025100000000000000000000000000000000000BB
:1025200000000000000000000000000000000000AB
:10253000000000000000000000000000000000009B
:102540004300000000000000000000000000000048
:10255000000000000000000000000000000000007B
:102560004300000000000000000000000000000028
:10257000000000000000000000000000000000005B
:102580004300000000000000000000000000000008
:10259000000000000000000000000000000000003B
:1025A00043000000000000000000000000000000E8
:1025B000000000000000000000000000000000001B
:1025C00043000000000000000000000000000000C8
:1025D00000000000000000000000000000000000FB
:1025E00043000000000000000000000000000000A8
:1025F00000000000000000000000000000000000DB
:102600004300000000000000000000000000000087
:1026100000000000000000000000000000000000BA
:10262000C7120408A312040800000000059604085D
:10263000DF880408A5630408A5630408A5630408EB
:10264000A5630408A5630408A5630408A56304083A
:10265000A5630408A5630408FFFFFFFFFFFFFFFF5A
:10266000FFFFFFFFFFFF0000010041534349490006
:10267000000000000000000000000000000000005A
:1026800000000000000000000000415343494900E1
:10269000000000000000000000000000000000003A
:1026A0000000000000000000000000000100000029
:108000000378407840EA032010FB01F04FF48071C0
:1080100090FBF1F000F30F0000B270472DE9F74F2D
:108020006A4CDFF8ACE123880091DEF80010B4F967
:108030000480C3EB21125B00C3EBE103B4F902102F
:1080400052435943131308FB03F84FEAA83808EBCF
:10805000E12101EB8102B1F5FA3802F180024FEA29
:10806000E1794FEA222349F1FF39B4F9082001935D
:10807000A8FB08AB08FB09F30BEB430BA161D3177B
:1080800002FB09F108FB0311A2FB08230B441F03A9
:10809000160347EA1257B4F90A2002FB0BF1D31773
:1080A0000AFB03130546A2FB0A011944020A42EA2D
:1080B000016292194FEA2123E6887B41003243F5A1
:1080C0000043A2FB060106FB03114A10CB1752EA3C
:1080D00003016FD0B4F91060B4F90E00F71706FB76
:1080E0000BF10AFB0711A6FB0AAB8B4400FB09F658
:1080F000C11708FB0161A0FB08898944DEF8041060
:108100004FEA4846C1F5801E4FEA494747EAD8374B
:108110001AEB060AB4F90C8076464BEB070BF717FF
:1081200000264FEACE70F90716EB0A064FEAC80799
:1081300041EA5E0147EB0B0740F6354E861B61EBCB
:108140000707A6FB0E010EFB071138F045FDB4F939
:1081500016204E13470B47EAC14702FB06FED31712
:1081600007FB03EEA2FB07237344564307FB03669A
:10817000A2FB07233344560E46EAC3163218B4F95D
:1081800014604FEA636747EB01037143F71700FB85
:108190000717A6FB00013944C60C46EA413692197E
:1081A0004FEAE147B4F912607B41100A40EA0360EC
:1081B000320112180DB1120A2A60009B13B11A463F
:1081C000019B136003B0BDE8F08F00BF204F00207B
:1081D000701F0020704770472DE9F041324E334F39
:1081E00074893B89B6F91420B6F902E0B6F90E801D
:1081F000B6F920C01B1B34895C43E313B6F9124067
:108200001A44E4020A2594FBF2F41C44B6F9043043
:10821000F4616543A4F57A6404FB04F204FB0EFEEA
:108220005C43B6F90C30121302FB08F85A431214DF
:108230004FEAEE2E02EB64340EEBE828B6F900E0CC
:10824000F388FE680234A41008EB8E0804F500449D
:1082500008FA0CF863434CF2503208F10208DC0BC8
:10826000A6EBA80642FA0CF3734353BF5B00B3FBC3
:10827000F4F35B00B3FBF4F31A1202FB02F440F6D2
:10828000DE3262430A4C12145C4302EB244208358E
:1082900002F6CF622D1103EB221300B1036001B18E
:1082A0000D60BDE8F08100BFE84E0020701F002087
:1082B00043E3FFFF2DE9F04F654B664EB3F80AC06C
:1082C0003469B3F8048087B04FEA0C2A0590188906
:1082D000B4EB0A0A4FF000024FF0000565EB020B09
:1082E000A0FB0A4500FB0B55E00940EA45604FEA58
:1082F000084407198E46D8884FEAE51141EB020879
:10830000A0FB0A45CDE90278B3F8028000FB0B55CB
:10831000200A40EA05604FEAC83410EB04084FEA2F
:10832000252141EB02099A89A2FB0A0102FB0B11EC
:10833000C20D42EA412212F5FA604FEAE15343F1DD
:108340000001B0F5FA6FCDE9000171F10001B4460A
:108350005EDA0524A2FB040104FB031100FB03F415
:1083600002FB0144DDE90267A0FB020121444D103C
:108370004FEA3004361B4FEA900444EA817467EBFD
:1083800005078D10B8EB040869EB0509DDE9004528
:1083900031484FF0FF31844275EB0101CDE90267AE
:1083A00023DA40F6AC5012184FF000014B4102FBAB
:1083B00003F1A2FB022303EB4103D900D000101A02
:1083C00041EA527163EB0101341847EB0105CDE935
:1083D00002450B24A2FB040104FB031149104FEAE0
:1083E0003000B8EB000869EB01090AFB0BF3DDE98B
:1083F0000001AAFB0AAB0BEB430B4FEADA7242EA2D
:108400004B02801A4FEAEB7361EB0301CDE90001E7
:10841000DCF81410A1FB082301FB0933540D5D1592
:1084200044EAC324DDE90223A21A65EB03031D46D7
:10843000D30B059A43EA454302B11360BEF1000F26
:1084400002D0009BCEF8003007B0BDE8F08F00BF2F
:108450000C4F0020701F002024FAFFFF4FF4006330
:10846000838270474FF40063838270473122F42186
:108470000CF022BD044B93F820209201343202F01C
:10848000FC02F4210CF018BDE84E00202E22F4214D
:108490000CF012BD012248210CF00EBD0122582122
:1084A0000CF00ABD012380F8453070474FF480532B
:1084B00083827047BFF34F8F0549064BCA6802F4A9
:1084C000E0621343CB60BFF34F8F00BFFDE700BFF7
:1084D00000ED00E00400FA0570B4037B04681F2B74
:1084E00008D9203B2021626801FA03F31A421CD10B
:1084F00070BC70472021226801FA03F31A42F7D0BA
:10850000426914495C2000FB021251685689CD680B
:108510000868296821F001012960828992B222EA63
:1085200006028281A36070BC7047426909495C20E1
:1085300000FB021251685689CD680868296821F04D
:1085400001012960828992B222EA06028281E360F7
:1085500070BC7047E88F00202B4B1978002951D050
:108560002A4B30B41C68988800226262A5899A80E0
:10857000284380B20129A08143D09C689889626217
:10858000A589284380B20229A0819A8139D01C692B
:10859000988A6262A589284380B20329A0819A82C1
:1085A0002FD09C69988B6262A589284380B20429E8
:1085B000A0819A8325D01C6A988C6262A589284381
:1085C00080B20529A0819A841BD09C6A988D626232
:1085D000A589284380B20629A0819A8511D01C6BF9
:1085E000988E6262A589284380B20729A0819A8665
:1085F00007D0986B998F42628489214389B2818127
:108600009A8730BC704700BFC8920020CC920020EF
:1086100010B4037B01681F2B09D9203B20224C6832
:1086200002FA03F31C4214D15DF8044B7047202278
:108630000C6802FA03F31C42F6D00C4A406800248E
:10864000147002685DF8044B22F0010202608B6036
:108650007047064A40680024147002685DF8044BB5
:1086600022F001020260CB60704700BF055000207D
:10867000F0B5C40022189200AE498B585B689D8A01
:10868000ADB2EEB2F7070A445CD4B70732D5BFF3F8
:108690005F8F167EF6B2012E00F0C780A64D1A8BB2
:1086A000BFF35F8F221801EB8202167E022E00F0CC
:1086B000D580221801EB8202167E032E00F08880FE
:1086C0009A8895F9186092B242F480629A802218D2
:1086D00001EB8202127E013296425BD1AA7E002615
:1086E0006E76002A40F09580204401EB8000002344
:1086F0004375F0BD77074ED416F0400600F0C980F0
:108700008D4D1E8A95F918E0176AF6B207F80E60CB
:108710005FFA8EFE0EF1010C4FFA8CFC177E85F885
:1087200018C00CF103029742664600F01C81221823
:1087300001EB8202127E9445C9D10EF1020676B297
:108740002E76C4E71E887C4D26F400663604360C6F
:108750001E801E88B6B246F480661E80967E002774
:108760002F76002E48D06E7E002E42D0221801EBCC
:1087700082020126127E6E76022A00F0B98022184B
:1087800001EB8202927D42F001021A82204401EB49
:108790008000037EF0BD684D967E0127AF76002EE7
:1087A00073D06E7E002E7BD1221801EB8202527EA6
:1087B000002A00F0A3801A882E7E92B2013642F47D
:1087C000007276B21A802E761A88D205FCD47EE723
:1087D000927E002A3FF474AF6A7E002A3FF470AFA5
:1087E0009A8895F9186022F480621204120C9A801B
:1087F0006DE7D27DFF2AB9D0221801EB8202967D67
:1088000006F0FE061E82D37DFF2BBFD0FF232B7602
:10881000BCE79A8822F4407212042044120C01EB47
:1088200080009A8000234375F0BD927E424D002A5D
:108830003FF435AF6A7E002A3FF431AF1A8822F444
:1088400080621204120C1A80BFF35F8F1A8B1A8891
:10885000AE7692B242F400721A8031E7927E002A1C
:108860003FF427AF6A7E002A3FF423AF1A8895F9B8
:10887000186022F480621204120C1A809A8822F482
:1088800080621204120C9A8021E76A7E002A8BD043
:1088900091E715F0800F284D3AD195F9186016E749
:1088A000167ED2F820E01F88022E95F9186045D96F
:1088B00027F480673F043F0C1F801F8AFFB20EF829
:1088C00006701F88D2F820E0BFB247F400771F80FF
:1088D000F2B21F8A561C76B2FFB20EF806709F885D
:1088E000961CBAB276B242F480622E769A806BE71A
:1088F0001A8892B242F400621A8040E71A8895F909
:10890000186092B242F4807201271A806F765BE79A
:1089100095F91870B7F1FF3F2CD0D669F65D1E822D
:1089200092F818E001377AB2964516462A767FF417
:10893000CEAEA3E7B43A0020701F0020BFB247F4C8
:1089400000771F801F8AFFB20EF80670F6B21F8AEA
:10895000D2F820E0721C52B20336FFB276B20EF8A3
:1089600002702E7630E79A8822F480621204120C8C
:108970009A80DCE6D77D1F822E76957E1DB9127E09
:10898000002A7FF403AF9A8822F480621204120C4A
:108990009A80FBE637B506236A4604460D460C303E
:1089A00003210CF0C1F9024690B1B4F91A106846DF
:1089B000FFF726FB2880B4F91E100DF10200FFF727
:1089C0001FFBA880B4F91C1001A8FFF719FB6880F1
:1089D000104603B030BD2DE9F04F4FF4807385B0E1
:1089E00043838383C38300F10C050446322004F0E3
:1089F00001FD1122002128460CF05EFA60220121BF
:108A000028460CF059FA642004F0F4FC02A9204630
:108A10000027FFF7BFFF0123B946B8463E46019342
:108A2000012E14BF11221222002128460CF044FA14
:108A3000002E0CBF4FF0010B4FF0FF3B4FF00A0A26
:108A40000122022128460CF037FA142004F0D2FC4F
:108A500002A92046FFF79EFFBDF90A20BDF90C00D0
:108A6000BDF90810224B82420BFB0299A8BF0246B7
:108A70008A42A8BF0A469A4201FB0B880BFB00778B
:108A800033DB01200BF0B9FBBAF1010AD8D1013672
:108A9000022EC5D1174B93FBF8F893FBF9F970221E
:108AA000A3F58423002193FBF7F7A4F81A80A4F818
:108AB0001C90E78328460CF0FFF92022012128466C
:108AC0000CF0FAF90022314628460CF0F5F9642042
:108AD00004F090FC019B23B94FF480736383A3835C
:108AE000E383012005B0BDE8F08F00230193CEE7BA
:108AF00001F0FFFF00D03B0007B506236A46F721CF
:108B00000CF012F99DF801309DF800100B4A1B0182
:108B100043EA01339DF8021043EA111353609DF8B4
:108B200004309DF803101B0143EA01339DF8051042
:108B300043EA1113136003B05DF804FB701F0020BB
:108B400007B5032301AAF6210CF0EEF89DF80530D5
:108B50009DF804201B0243EA02439DF806201343BC
:108B6000054AB2F92020C2F10802D340034AD3607B
:108B700003B05DF804FB00BFE84E0020701F00202A
:108B800007B5022301AAF6210CF0CEF89DF80420C7
:108B90009DF8053043EA0223024A138103B05DF8D1
:108BA00004FB00BF701F002007B5032301AA0021AA
:108BB0000CF0BAF89DF805309DF804001B0243EA5A
:108BC00000439DF80600184303B05DF804FB08B5A8
:108BD000FFF7EAFF014B586108BD00BF701F00207E
:108BE00008B5FFF7E1FF014B186108BD701F0020B9
:108BF00070B582B00446062310306A4643210CF05B
:108C000093F8A8B19DF804009DF800609DF801104C
:108C10009DF802509DF803209DF8053041EA062199
:108C200043EA002342EA052221876287A3870120C5
:108C300002B070BD70B582B00446062308306A46A3
:108C40003B210CF071F8A8B19DF804009DF800607C
:108C50009DF801109DF802509DF803209DF8053005
:108C600041EA062143EA002342EA0522E182228307
:108C70006383012002B070BDF0B5876983B00646FA
:108C800017B13B68BA885A837069DFF8A4E083891A
:108C9000C3244FF47A734FF0060C6D464FF6FF7104
:108CA0000EF1010E03E0013B9BB28B4220D0028902
:108CB0009207F8D5A3B283814FF47A7302E0A3B28E
:108CC0008B4215D00289D20703F1FF34F7D5828990
:108CD00092B20DB12A700135BCF1000F0BD00CF12E
:108CE000FF3CFF24BEF1000FE1D09EF80040D7E723
:108CF0000BF0B9FFB76917B13B68BA881A839DF8C2
:108D000005009DF801509DF802109DF803409DF864
:108D100004209DF8063041EA052143EA002342EA97
:108D20000422012031877287B38703B0F0BD00BFF2
:108D3000D8230408F8B5057B466903681F2D29D997
:108D4000A5F120045F682021A1400F422A4613D0DC
:108D50001022A240D960DA605A68E240D10703D5F8
:108D6000012202FA04F4DC600446304604F066FD99
:108D7000227B23681F2A20D9A2F1200008215A68EB
:108D80008140114200D0D9600422596882400A42D1
:108D900021D1F8BD20211C68A9400C422A460CD0E4
:108DA0001022AA4099609A601A68EA40D207DBD57F
:108DB000012202FA05F59D60D6E708211868914066
:108DC000014200D099600421186801FA02F20242BF
:108DD00003D09A60F8BDDA60F8BDF8BD064A074BCB
:108DE00010781B7883428ABFC3F18003C01AC01871
:108DF000C0F17F00704700BFA06400201D64002008
:108E0000F0B55FEA930E33D000F1100601F11005C2
:108E100002F11004774616ED046A55ED044A56ED4A
:108E2000026A15ED025A16ED037A55ED035A56ED16
:108E3000017A26EE246A66EE856A04ED046A15ED71
:108E4000016A44ED026A27EE257A67EE867A013FD1
:108E500004ED037A44ED017A06F1100605F11005E0
:108E600004F11004D7D14FEA0E14204421442244C7
:108E700013F003030BD000EB8303F0EC017AB1ECA9
:108E8000017A67EE877A8342E2EC017AF5D1F0BD90
:108E9000144B984224D003F58063984220D0038875
:108EA00023F040031B041B0C0380038823F03803CA
:108EB0001B041B0C59B141F48071002991FAA1F2F5
:108EC000B2FA82F108BF4FF0FF310139C9001943EE
:108ED00089B2018003889BB243F04003038070474E
:108EE0004908DCE70038004008B540F2E93300E00B
:108EF000A3B10289013B12F0020F9BB2F8D089B2F4
:108F0000818140F2E93300E043B10289013B12F074
:108F1000010F9BB2F8D08089C0B208BD0BF0A3FE50
:108F2000C0B208BD38B504460D4600BF80680BF0DE
:108F30003FFD29466068FFF7D7FFA0680BF03DFDB5
:108F400000BF38BD0C4B984213D0A3F58063984204
:108F50000FD003F5804398420BD003F5806398420D
:108F600007D003F58063984203D0044B186840088B
:108F70007047024B1868704700040140F0820020DF
:108F8000F0B5774B774A87B01968914200AF00F08F
:108F9000DB800023744A3B607B60136843F48033BA
:108FA000136003E03B68B3F5A04F09D0136803F4E6
:108FB00000337B603B6801333B607B68002BF1D062
:108FC000694B1B6813F4003318BF01237B607B6877
:108FD000012B7BD0654D644B654AEA606549586F4B
:108FE000654A0860AA605E6B644C654A654826F075
:108FF00080065E635E6F46F080765E67196B0C4399
:109000001C63596B5963996B9963196C41F05B51FF
:1090100041F47B1141F41F6141F00F011964596C57
:1090200007F118040A4348F2FF715A6444F8101D0E
:10903000002621460123FB733E737E73BE7326F028
:10904000DDFE21464FF6FF734F48BB6026F0D6FE8B
:109050004FF6FF7321464D48BB6026F0CFFE2146F8
:109060004B4826F0CBFE21464A4826F0C7FE214653
:10907000494826F0C3FE2146484826F0BFFE214657
:10908000474826F0BBFE2146464826F0B7FE20465C
:1090900026F06CFC444B454C1B68BA684448454973
:1090A000A4FB03439B09A0FB0202013B920CB3F11A
:1090B000807F0A6007D2404AF0200721536085F87C
:1090C0002300966011601C37BD46F0BD264B3B4D1A
:1090D0001A6C3B4842F080521A642C6842688168DE
:1090E00044F440442C609C689C609C6844F40044B8
:1090F0009C609C6844F4A0549C600068120642EA9C
:10910000801242F48002490842F00802013942EA22
:1091100001425A601A6842F080721A601A6892011D
:10912000FCD52849104A40F205700860996821F082
:1091300003019960996841F002019960936803F016
:109140000C03082BFAD145E700221A6062B61E4BC9
:109150001B6883F308881D4B1B689847FEE700BF18
:10916000FCFF0120EFBEADDE0038024000ED00E064
:109170000005FA058CA5002000000008FF9167009B
:10918000335F070000000240000402400008024074
:10919000000C02400010024000140240001802407F
:1091A000001C024000200240F0820020D34D6210DB
:1091B00083DE1B434085002010E000E0007000408B
:1091C00000000020003C02400000FF1F0400FF1FC1
:1091D00008B5054B1B6803B19847044B044A1A6055
:1091E00072B6FFF767F900BF084B0020FCFF0120B3
:1091F000EFBEADDE2DE9F04F87B090F8553001900D
:10920000002B40F0B38004AB0393554BDB7E002B67
:1092100000F00781019B10330293019B5869514B69
:10922000984200F02A82504A90420CBF30223822E5
:10923000038823F040031B041B0C038003889BB2AC
:1092400023F038031A4302800388019A9BB243F04B
:1092500040030380936992F84E4013B11A689B88CB
:10926000538340F2E93304E0013B9BB2002B00F052
:10927000C78202899607F7D51A23838140F2E93322
:1092800004E0013B9BB2002B00F0BA820289D507B3
:10929000F7D5838940F2E93304E0013B9BB2002B10
:1092A00000F0AB8202899107F7D5A4B2848140F225
:1092B000E93304E0013B9BB2002B00F09E8202895F
:1092C000D207F7D58389019B9B6913B11A689B88E4
:1092D0001383012004F034F8019B224A5B69934216
:1092E00000F09B8220498B4214BF082100211A887C
:1092F000029822F040021204120C1A801A8892B2CC
:1093000022F03802114319801988039A89B241F07A
:1093100040011980062343210BF006FD002800F0D0
:10932000F6819DF810409DF812509DF813309DF87D
:1093300011109DF814009DF8152041EA042143EA1C
:109340000523019C1BB242EA002263872187A28782
:109350005BB2013300F0B08107B0BDE8F08F00BF11
:10936000701F002000380040003C00401D09013DF6
:10937000032D03F00F0300F24882C14A32F81500B2
:1093800040FA03F2D40740F14082012404FA03F3C7
:10939000013B184037F070FCBA4BBB4A5B5D184488
:1093A00012EBC00500F0318200232021EB71A9717E
:1093B00052F83000B54A00F13F4303F57E039B0AA3
:1093C000D25C02F01F035209032A04FA03F300F0EF
:1093D0003082042A00F02882022A00F02082AB8822
:1093E000049304A900230391059326F007FD019936
:1093F000A74B41F80C3F28462FF086FEAB88B3FA06
:1094000083F3C3F11F03012212FA03F33FF4FDAE0D
:10941000A0490A6813430B609F4BDB7E002B7FF44F
:10942000F9AE019B9D4A5B69934200F009829C4919
:109430008B420CBF302138211A889A4C9A4FDFF8A2
:1094400070A222F040021204120C1A801A8892B202
:1094500022F03802114319801A88019992B2103112
:1094600042F040021A800291084680226B210BF0E4
:1094700015FC96238D48DFF83CC24FF010084FF4DE
:109480007A759E46DAF80430C3F30803002B40F0E7
:109490009881EFF31183002B40F09381216882685B
:1094A00000BF23689942F9D13E6805FB06F39B1A79
:1094B000B3FBF6F305FB013101260091DAF8043025
:1094C000C3F30803002B40F04381EFF31183002B1B
:1094D00040F03E812368816800BF22689342F9D141
:1094E000D7F800B005FB0BF2521AB2FBFBF205FBFA
:1094F0000323009A9B1AB3F57A7FDFD3BEF1010EE6
:10950000C0D1032268210298DFF8A4A10BF0C6FBAA
:1095100096236648DFF89CC14FF010084FF47A7527
:109520009E46DAF80430C3F30803002B40F02D8187
:10953000EFF31183002B40F028812168826800BF7F
:1095400023689942F9D13E6805FB06F39B1AB3FBE9
:10955000F6F305FB013101260091DAF80430C3F37C
:109560000803002B40F0D780EFF31183002B40F06D
:10957000D2802368816800BF22689342F9D1D7F86E
:1095800000B005FB0BF2521AB2FBFBF205FB032302
:10959000009A9B1AB3F57A7FDFD3BEF1010EC0D1DA
:1095A000029D03226B212846744676460BF076FB1B
:1095B0000F2003F0C5FE10226A2128460BF06EFB37
:1095C0000F2003F0BDFE22466C2128460BF066FBFF
:1095D0000F2003F0B5FE019C192194F85020284675
:1095E0000BF05CFB0F2003F0ABFE18221B2128467A
:1095F0000BF054FB0F2003F0A3FE10221C21284681
:109600000BF04CFB0F2003F09BFE10223721284665
:109610000BF044FB0F2003F093FE01223821284673
:109620000BF03CFB0F2003F08BFE62691B4B9A4250
:1096300000F0048103F580639A4214BF08230023DD
:10964000118821F040010904090C1180118889B2A8
:1096500021F038010B43138013889BB243F0400381
:109660001380012003F06CFE0B4A0123D376019B8B
:1096700058690A4B98427FF4D6AD3022D8E500BF36
:109680002C510408285104087C830020B84F04089A
:10969000A5840008003C0140701F002000380040F5
:1096A000003C00403C8500204085002010E000E0A8
:1096B00000ED00E038850020019B93F9383001333C
:1096C0007FF44AAE0A2632202FF060FA4FF4FA7582
:1096D00003F0EAFD044603F0E7FD001BB0F57A7FD6
:1096E000F9D3013DF4D107202FF0B2F84FF47A7589
:1096F00003F0DAFD044603F0D7FD001BB0F57A7FD6
:10970000F9D3013DF4D1013EDDD1FFF761FD019BAD
:10971000B3F93A301CE6EFF3118988F312888168B7
:109720000368DB0344BFCCF8006081682368DCF881
:1097300000205FFA89F989F31188D7F800901A445C
:1097400005FB09F35B1AB3FBF9F305FB02331FE7D3
:10975000EFF3118988F3128881680368DB0344BF43
:10976000CCF8006081682368DCF800205FFA89F992
:1097700089F31188D7F800901A4405FB09F35B1AA6
:10978000B3FBF9F305FB0233B3E6EFF3118288F381
:10979000128886680368D90303D50123CCF800300A
:1097A00086682368DCF80010D2B282F311883A6828
:1097B000194405FB02F39B1BB3FBF2F305FB0131DC
:1097C000C9E6EFF3118288F3128886680368D9032B
:1097D00003D50123CCF8003086682368DCF800103C
:1097E000D2B282F311883A68194405FB02F39B1B3D
:1097F000B3FBF2F305FB01315EE60BF034FA62E5F0
:109800000BF031FA019B586944E501990D4B41F881
:109810000C3F00202FF078FCF5E4002167E50A4AB0
:10982000516C0B435364DAE5074A116B0B43136326
:10983000D5E5054A116C0B431364D0E53346FFE6CA
:109840003021F9E5A58400080038024008B5034B33
:109850001B6803B1984772B6FEF72CFE084B002038
:10986000084B10B507281B68C8BF143818440C46AD
:10987000007E0AF053FE20B12146BDE810400BF0F7
:10988000A1B810BDA43A002038B50C4B07281B68BE
:10989000CCBFA0F11404044623440546187E0AF008
:1098A0003DFE50B128220134C47182712EF06CFF4C
:1098B00028460021BDE83840D2E738BDA43A002050
:1098C00070B50F4C0F4DC0EBC00004EB8004286B4B
:1098D00026693043286382B09209667BA160002527
:1098E000012101A863618DF804608DF805208DF8D1
:1098F00006508DF8071025F0F1FF02B070BD00BFD3
:10990000141B002000380240074BC0EBC00030B4ED
:1099100003EB8000054C0569236B2B432363017621
:10992000427630BC704700BF141B00200038024054
:109930002DE9F04F5B4C54F8204083B0002C00F030
:10994000AC80266E002E00F0AA809046564A3569FB
:109950002260994604F2662204F166036361A26103
:109960004FF400737268A1600746E3602361A2654B
:10997000A246B5B14D4B00205A68954203F11C0335
:1099800076D001301028F7D100207A1CD2B20C21F9
:10999000FFF7BAFFA36DB168326962630433E16314
:1099A0006365F068E8B1414B00215A68904203F1C9
:1099B0001C035BD001311029F7D100257A1CD2B2EB
:1099C0000B212846FFF7A0FF2346F27F384928469F
:1099D000FFF776FFA36DB168F268A26304332164D8
:1099E000236594F865000AF099FD054694F8640033
:1099F0000AF094FD8346307F00284BD119F0080F00
:109A000038D118F0020F09D045B10B227B1CAA7186
:109A1000EB712846727F22210AF046FE18F0010FF2
:109A200015D1E36B7BB996F82020B17F8DF8063015
:109A300001A8930901228DF805308DF804108DF8E6
:109A4000072025F04BFF504603B0BDE8F08FBBF177
:109A5000000FE6D001370C238BF807708BF8063027
:109A60005846727F22210AF01FFEDAE7CDB2A5E741
:109A7000C0B28AE70137FFB215B10B23EF71AB71AA
:109A800019F0100F284614BF02211221727F0AF02C
:109A90000BFEC6E72EF05AFEB0E7A246D3E7B24669
:109AA000D1E700BF843A0020E0230408141B002003
:109AB000358D000800B97047F0B599B006462FF013
:109AC00075FD804DC36802682A600446002B00F0D3
:109AD000DE8030460AF022FD7B4BD86118B1292286
:109AE00000238271C371227A2A210AF0DDFD2868E1
:109AF00003F054FA2EF02AFE2E68338823F0010377
:109B00001B041B0C33803046FFF71CFA6F4A90424F
:109B1000034600F2BE80002218A9DFF8D4E16C4FA2
:109B200021F85C2D304601326A4EB3FBF2F303227A
:109B3000B3FBF6F3002602939BB2B3FBF2F3AEF84D
:109B400000305B003B80ADF80C60ADF806608DF82E
:109B50000E602FF0E3FCE379ADF812606022990704
:109B6000ADF814600696ADF81C60ADF81E60ADF857
:109B70002060ADF82260ADF8102040F1948013F021
:109B8000010F0CBF324608220423ADF81E20ADF8A9
:109B90001430002304AA61792868069302F0E8FDD6
:109BA000617928684C4E2FF089FC2B68B3F844206B
:109BB0006FEA42426FEA524292B2A3F844201A88F6
:109BC00092B242F080021A80E2796079198C920791
:109BD0004CBF04220122824092B289B221EA0201E2
:109BE0001984198C89B20A431A841A8892B242F0F5
:109BF00001021A80207D00222921FFF785FE6022C4
:109C00003649207D0023FFF75BFEE068306025F0D9
:109C10009BFF3068036823F00103036025F094FF85
:109C200009A825F053FF2B686279216930680991F2
:109C300034331A4440F22A330A920D934FF480626F
:109C4000274B0F920B9340224FF48053002709A912
:109C50000C9210934FF480424FF4403311920E97C0
:109C60001297139325F044FF637929681D480C2B44
:109C70009CBF1D4A32F813708B8932689BB23B43FC
:109C80008B811368012143F010031360017019B038
:109C9000F0BD00F1B77202F558521449B2FBF1F26F
:109CA000013A92B238E713F0010F0CBF00210221F4
:109CB00001224FF48073ADF81C10ADF81220ADF8FE
:109CC000203066E7446F0020701F0020FF6BDC022D
:109CD0003A6F002000350C00406F0020118600080C
:109CE000DC5300203C6F002044510408006CDC026F
:109CF000386F00200348D0F8AC3113B100F5D270B2
:109D000018477047141B00200348D0F8903113B156
:109D100000F5C47018477047141B00200348D0F8A2
:109D2000743113B100F5B67018477047141B00204A
:109D30000348D0F8583113B100F5A87018477047A0
:109D4000141B00200348D0F83C3113B100F59A7081
:109D500018477047141B00200348D0F8203113B176
:109D600000F58C7018477047141B00200348D0F88A
:109D700004310BB1FC301847704700BF141B0020A2
:109D80000348D0F8E8300BB1E0301847704700BF07
:109D9000141B00200348D0F8CC300BB1C430184756
:109DA000704700BF141B00200348D0F8B0300BB13F
:109DB000A8301847704700BF141B00200348D0F894
:109DC00094300BB18C301847704700BF141B002033
:109DD0000248836F0BB1703018477047141B002086
:109DE0000248C36D0BB1543018477047141B002054
:109DF0000248036C0BB1383018477047141B002021
:109E00000248436A0BB11C3018477047141B0020EE
:109E10000248836803B11847704700BF141B002035
:109E2000F8B584894FF6FF764FF47A7433B319B3DB
:109E30000F78013101E0B44218D00589013CAD072B
:109E4000A4B2F8D5BCB284814FF47A7402E0BCB2FB
:109E5000B4420BD00589ED0704F1FF37F7D58589AA
:109E6000ADB20AB115700132013BDFE70AF0FBFE2B
:109E7000003018BF0120F8BDFF27DEE70120F8BD44
:109E800030B5134C237883B01BB90120237003B085
:109E900030BD1049052200230D688DF804208DF88F
:109EA000053000BFA8680AF083FD6A4601A90223B5
:109EB0006868FFF7B5FFA8680AF07FFD00BF9DF84E
:109EC000013003F0010383F00100237003B030BDC3
:109ED000916F00204C6F002070B5064C0646256837
:109EE00003E023685B1BB34203D8FFF7C9FF0028D8
:109EF000F7D070BD3C8500202DE9F04F89B0B2F15C
:109F0000000A02900491039340F3C5800B4600229F
:109F100001EB8A0153F8040B8B420244FAD1039BF4
:109F20000592002B00F0AF80059B002B7CD05E4B90
:109F3000059A1B68DFF8889100920099DAB25118EF
:109F4000B1F5807F8CBFC2F58072009A0192574AAA
:109F500092689A4240F28280554A11780022069215
:109F60008DF81C2002228DF81820002960D01A0ECE
:109F70008DF819200DF11A021C0C190A9370147037
:109F800051700620FFF7A8FF0621D9F80000FEF760
:109F9000C9FF484A0123137000BFD9F80030986800
:109FA0000AF006FD424BD9F800201B785068002BC0
:109FB00006A90CBF042305230022FFF731FF00246C
:109FC000049D029E019FA34629684FEA840800224F
:109FD0000B46013471B1B9422DD2D9F80000316875
:109FE0004068FFF71DFF2A68336813443360BF1AC7
:109FF000C5F800B0A24505F1040506F10406E3D159
:10A00000D9F8003098680AF0D8FC00BF264B0199B7
:10A0100000981B68421A0092234A0B441360039A6B
:10A020004AB3009A002A88D1059809B0BDE8F08F9C
:10A030000DF11902A0E7029CD9F8003054F808107D
:10A04000586800223B46FFF7EBFE54F808202B68C7
:10A050003A44DF1B44F808202F60D1E70598009CA4
:10A060001549164A001B0590059800230B701370C4
:10A0700009B0BDE8F08F059B009A9B1A05930598DF
:10A0800009B0BDE8F08FFFF7FBFE00287FF44CAF6E
:10A09000039B0593C8E7039C1CB9FFF7F1FE0594E9
:10A0A000C2E700230593BFE7686E0020A01A0020D6
:10A0B000906F0020916F0020A06400201D6400209C
:10A0C0004C6F002010B50C4C45F20820FFF704FF40
:10A0D00020680621FEF726FF084B20680122C721D1
:10A0E0001A70FEF71FFF06480649074A002303704F
:10A0F0000B70136010BD00BF4C6F0020916F0020EB
:10A10000A06400201D640020686E0020F0B51F4C84
:10A1100083B0277800234FF0030E00930E461546B8
:10A120008DF804308DF800E06FB3030E8DF8013028
:10A130000DF10203010C020A9870197006205A7082
:10A14000FFF7CAFEE8B100BF114F3B6898680AF0FC
:10A150002FFC23783A68002B14BF0523042369469B
:10A1600050680022FFF75CFE3B68324600215868C9
:10A170002B46FFF755FE3B6898680AF01EFC00BFAF
:10A18000284603B0F0BD0DF10103D3E7906F002026
:10A190004C6F0020F8B5654C0601A7190546387AC2
:10A1A0002EF0D4FA3B7A03F01F015B090122032B46
:10A1B00002FA01F26DD0042B66D0022B5CD0A319F9
:10A1C000013518790AF0AAF9EDB2074610B1122349
:10A1D000C5718371A31958790AF0A0F910B113233E
:10A1E000C5718371A31998790AF098F910B11423F5
:10A1F000C5718371A5190A21EA7938460AF054FA23
:10A2000068790AF08BF9EA790A210AF04DFAA879FF
:10A210000AF084F9EA790A210AF046FAA359444A75
:10A22000934247D0434A934250D0434A934259D035
:10A23000424A934262D0424A93426BD0414A93428F
:10A240002CD03444227BE2B901200222198801F487
:10A25000415141F445710A4302431A809A8B22F41A
:10A2600000621204120C07219A8319821A8892B292
:10A2700042F040021A80F8BD334B596A0A435A62D1
:10A280009DE700200246E1E72F4B19690A431A6156
:10A2900095E72D4B196A0A431A6290E702F564426A
:10A2A0004FF40010536A43F40013536225F04EFB41
:10A2B000A359C6E702F584324FF48050536A43F441
:10A2C0008053536225F042FBA359BAE702F50032EE
:10A2D0004FF48040136A43F48043136225F03EFB41
:10A2E000A359AEE702F5FE324FF40040136A43F47F
:10A2F0000043136225F032FBA359A2E702F5823234
:10A300004FF40050536A43F40053536225F01EFB90
:10A31000A35996E702F568424FF48010536A43F45C
:10A320008013536225F012FBA3598AE7606F002067
:10A330000030014000380040003C00400034014043
:10A34000005001400054014000380240431C00F01E
:10A3500014812DE9F04F4FEAC00808EB00039B0081
:10A36000DFF8F4A25AF803B087B00AEB0304BBF19C
:10A37000000F00F0FF8014330AEB03010022DBF82A
:10A3800004704AF803204A608A60CA600346A568E0
:10A3900001900133D4F80C90DBB2002D00F0EE8078
:10A3A0001522EB71AA71B9F1000F00F0008116229D
:10A3B00089F8062089F807309BF80E002EF0C6F9C0
:10A3C000BB8823F440731B041B0CBB8028460AF097
:10A3D000F4FA48460AF0F1FA1121284609F0E8FF9C
:10A3E0001121484609F0E4FF0826642404E00A200D
:10A3F0003CB102F0A5FF013C28460AF005FB00280D
:10A40000F5D028460AF0D4FA0A2002F099FF28462F
:10A410000AF0D3FA0A2002F093FF013EECD148463D
:10A420000AF0C6FA0A2002F08BFF28460AF0C0FAAA
:10A430000A2002F085FF28460AF0BFFA0A2002F03F
:10A440007FFF48460AF0B9FA019B08EB03040AEBC8
:10A4500084042846637C002B0CBF12213221042285
:10A460000AF022F9637C002B0CBF122132214846EE
:10A4700004220AF019F9704B9F4200F0B7806F4B2D
:10A480009F4200F0BD806E4B9F4200F0A580BB88CC
:10A4900001996C4A6C4C23F440731B041B0CBB8069
:10A4A0003B8888440AEB880A9BB243F001039AF880
:10A4B00010103B80BD8802A8002918BF144625F063
:10A4C00055FA049A6148B2FBF4F325F03F05A0FB6E
:10A4D00002122D04900C2D0C0543BD805C4C398874
:10A4E0004FF4967202FB00F284FB02409BB2D2173B
:10A4F000002BC2EBA01221F0010108BF01230904C7
:10A50000013243F40043090C92B239803A84BB8390
:10A510003B889BB243F001033B803B8823F481637B
:10A5200023F002031B041B0C43F480634FF48042AE
:10A530003B803A813B8823F080031B041B0C3B804B
:10A540009BF810308DF808300024012302A88DF804
:10A550000B308DF809408DF80A4025F0BFF99BF8C3
:10A560000F308DF8083002A88DF809408DF80A40A8
:10A5700025F0DAF907B0BDE8F08F7047B9F1000FA8
:10A5800048D0162289F8073089F806209BF80E007B
:10A590002EF0DCF8BB8823F440731B041B0C284608
:10A5A000BB800AF00AFA48460AF007FA18E79BF857
:10A5B0000E002EF0CBF8BB8823F440731B041B0C59
:10A5C000BB8028460AF0F9F948460AF0F6F911214D
:10A5D000284609F0EDFE07E71E4A136A43F400031C
:10A5E00013624FF4000025F0B9F950E7194A136AD5
:10A5F00043F4001313624FF4001025F0AFF946E75F
:10A60000144A136A43F4800313624FF4800025F068
:10A61000A5F93CE79BF80E002EF098F8BB8823F4D0
:10A6200040731B041B0C4846BB800AF0C6F9484621
:10A630000AF0C3F9D8E600BF0054004000580040BB
:10A64000005C0040009F2400804F120083DE1B430B
:10A65000D34D621000380240B43A0020F0B5C60075
:10A6600033189B00254DEA585468A28A83B092B2F1
:10A670000192019A2B4412F4706F1CBF01221A75CB
:10A68000019B13F4E06F07460CD1A38A3E4423F4E8
:10A69000706305EB86051B041B0C0022A3826A7500
:10A6A00003B0F0BD238BA38823F480631B041B0C31
:10A6B000A380019B9B05E8D423889805E5D42388D3
:10A6C000D9050ED52388DA05FCD423889BB243F440
:10A6D0000073238023889B05FCD43846FFF736FEA1
:10A6E000D3E723889BB243F400732380A38823F429
:10A6F00040731B041B0CA380C7E700BFB43A0020C3
:10A70000F0B583B0441C8DF8073001D0032802DD7A
:10A71000002003B0F0BDC700244E3B1806EB8303B6
:10A720005D68002DF4D04900C9B29975012400215B
:10A73000DA755C7699761C765C751975A9880DF1C9
:10A7400007028905DA611A6214D42B88DA050CD461
:10A750004FF4805401E0013C1ED02B889B05FAD4B5
:10A760002B889BB243F480732B80AB889BB243F45D
:10A770004073AB80074406EB87024FF4805401E03E
:10A78000013C09D0537D002BFAD106EB87073C7DB5
:10A7900084F0010003B0F0BD054A138801339BB279
:10A7A0001380FFF7D3FD2046B3E700BFB43A002083
:10A7B0007C4200202DE9F04F87B090F85530029090
:10A7C000002B40F0D985029A137C1032012B1046E1
:10A7D000039200F03186022B00F0C885B44CB54DD1
:10A7E000DFF8D892B448DFF8D8E24FF0640A4FF0AF
:10A7F000100C4FF47A76D9F80430C3F30803002B19
:10A8000040F0EA84EFF31183002B40F0E5842168E7
:10A81000826800BF23689942F9D12F6806FB07F3CD
:10A820009B1AB3FBF7F306FB013101270191D9F81D
:10A830000430C3F30803002B40F02283EFF31183AD
:10A84000002B40F01D832368816800BF226893427B
:10A85000F9D1D5F800B006FB0BF2521AB2FBFBF2AD
:10A8600006FB0323019A9B1AB3F57A7FDFD3BAF173
:10A87000010AC0D1029B1B7C012B00F0D385022B67
:10A8800000F06D856423DFF834A28B4FDFF830824F
:10A8900001934FF010094FF47A7EDAF80430C3F3D5
:10A8A0000803002B40F0B584EFF31183002B40F038
:10A8B000B0842168BA6800BF23689942F9D128683A
:10A8C0000EFB00F39B1AB3FBF0F30EFB01310120EA
:10A8D0008B46DAF80430C3F30803002B40F0ED8216
:10A8E000EFF31183002B40F0E8822368BE6800BFBD
:10A8F00022689342F9D1D5F800C00EFB0CF2921BEE
:10A90000B2FBFCF20EFB0323A3EB0B03B3F57A7F40
:10A91000DFD3019B013B0193BFD1029B1B7C012B29
:10A9200000F0BF85022B00F01385DFF8909162489C
:10A93000DFF88CE14FF0640A4FF0100C4FF47A7698
:10A94000D9F80430C3F30803002B40F00C84EFF374
:10A950001183002B40F007842168826800BF2368C0
:10A960009942F9D12F6806FB07F39B1AB3FBF7F363
:10A9700006FB013101270191D9F80430C3F3080324
:10A98000002B40F0B582EFF31183002B40F0B08232
:10A990002368816800BF22689342F9D1D5F800B0DE
:10A9A00006FB0BF2521AB2FBFBF206FB0323019AE1
:10A9B0009B1AB3F57A7FDFD3BAF1010AC0D1029BAB
:10A9C0001B7C012B00F06485022B00F0BA84DFF8B9
:10A9D000EC903948DFF8E8E04FF00F0A4FF0100C28
:10A9E0004FF47A76D9F80430C3F30803002B40F013
:10A9F000D783EFF31183002B40F0D2832168826864
:10AA000000BF23689942F9D12F6806FB07F39B1A10
:10AA1000B3FBF7F306FB013101270191D9F80430AC
:10AA2000C3F30803002B40F08082EFF31183002B67
:10AA300040F07B822368816800BF22689342F9D18D
:10AA4000D5F800B006FB0BF2521AB2FBFBF206FB84
:10AA50000323019A9B1AB3F57A7FDFD3BAF1010A77
:10AA6000C0D1029A92F84F30127C032B8CBF1A236C
:10AA70001823012A00F02985022A00F05B84DFF800
:10AA80003C900D48DFF838E04FF00F0A4FF0100C03
:10AA90004FF47A76D9F80430C3F30803002B40F062
:10AAA0002A83EFF31183002B40F025830AE000BFD7
:10AAB0003C8500204085002010E000E000ED00E033
:10AAC000388500202168826800BF23689942F9D147
:10AAD0002F6806FB07F39B1AB3FBF7F306FB013164
:10AAE00001270191D9F80430C3F30803002B40F08B
:10AAF0003982EFF31183002B40F0348223688168A0
:10AB000000BF22689342F9D1D5F800B006FB0BF2E2
:10AB1000521AB2FBFBF206FB0323019A9B1AB3F510
:10AB20007A7FDFD3BAF1010AB4D1029B1B7C012BDF
:10AB300000F0C184022B00F0F783DFF80893BF48D0
:10AB4000DFF8FCE24FF00F0A4FF0100C4FF47A766A
:10AB5000D9F80430C3F30803002B40F0E882EFF388
:10AB60001183002B40F0E3822168826800BF2368D4
:10AB70009942F9D12F6806FB07F39B1AB3FBF7F351
:10AB800006FB013101270191D9F80430C3F3080312
:10AB9000002B40F00482EFF31183002B40F0FF8183
:10ABA0002368816800BF22689342F9D1D5F800B0CC
:10ABB00006FB0BF2521AB2FBFBF206FB0323019ACF
:10ABC0009B1AB3F57A7FDFD3BAF1010AC0D102999B
:10ABD0000A7C91F84E30012A00F04084022A00F0ED
:10ABE0009D83DFF860929548DFF854E24FF00F0A3A
:10ABF0004FF0100C4FF47A76D9F80430C3F3080301
:10AC0000002B40F05C82EFF31183002B40F0578261
:10AC10002168826800BF23689942F9D12F6806FB3A
:10AC200007F39B1AB3FBF7F306FB013101270191F0
:10AC3000D9F80430C3F30803002B40F0CD81EFF3C3
:10AC40001183002B40F0C8812368816800BF22680F
:10AC50009342F9D1D5F800B006FB0BF2521AB2FBC1
:10AC6000FBF206FB0323019A9B1AB3F57A7FDFD32D
:10AC7000BAF1010AC0D102990A7C91F85030012A38
:10AC800000F0E483022A00F04383DFF8B8916B48B8
:10AC9000DFF8ACE14FF0640A4FF0100C4FF47A7615
:10ACA000D9F80430C3F30803002B40F0CF82EFF350
:10ACB0001183002B40F0CA822168826800BF23689C
:10ACC0009942F9D12F6806FB07F39B1AB3FBF7F300
:10ACD00006FB013101270191D9F80430C3F30803C1
:10ACE000002B40F09681EFF31183002B40F091810F
:10ACF0002368816800BF22689342F9D1D5F800B07B
:10AD000006FB0BF2521AB2FBFBF206FB0323019A7D
:10AD10009B1AB3F57A7FDFD3BAF1010AC0D1029B47
:10AD20001B7C012B00F0AB83022B00F0EB82DFF8E1
:10AD300014914248DFF808E14FF00F0A4FF0100C71
:10AD40004FF47A76D9F80430C3F30803002B40F0AF
:10AD50009982EFF31183002B40F09482216882687E
:10AD600000BF23689942F9D12F6806FB07F39B1AAD
:10AD7000B3FBF7F306FB013101270191D9F8043049
:10AD8000C3F30803002B40F06181EFF31183002B24
:10AD900040F05C812368816800BF22689342F9D14A
:10ADA000D5F800B006FB0BF2521AB2FBFBF206FB21
:10ADB0000323019A9B1AB3F57A7FDFD3BAF1010A14
:10ADC000C0D1029B1B7C012B00F05183022B00F0B1
:10ADD0009382DFF870801949194F4FF00F094FF037
:10ADE000100E4FF47A70D8F80430C3F30803002B28
:10ADF00040F06482EFF31183002B40F05F82226801
:10AE00008E6800BF23689A42F9D1D5F800C000FBD4
:10AE10000CF39B1BB3FBFCF300FB023301930126F5
:10AE2000D8F80430C3F30803002B40F02C81EFF373
:10AE30001183002B40F0278106E000BF10E000E006
:10AE40003885002000ED00E02368D1F808A000BF9D
:10AE500022689342F8D1D5F800B000FB0BFCACEBB4
:10AE60000A0CBCFBFBFC00FB03C3019A9B1AB3F565
:10AE70007A7FD5D3B9F10109B5D107B0BDE8F08F1C
:10AE8000EFF311888CF3128881680368DB0344BFF9
:10AE9000CEF8007081682368DEF800205FFA88F839
:10AEA00088F31188D5F800801A4406FB08F35B1A72
:10AEB000B3FBF8F306FB0233D4E4EFF3118689F316
:10AEC0001288B9683B68DB0344BFC8F80000B96862
:10AED0002368D8F80020F6B286F311882E681A4449
:10AEE0000EFB06F35B1AB3FBF6F30EFB02330BE526
:10AEF000EFF311888CF3128881680368DB0344BF89
:10AF0000CEF8007081682368DEF800205FFA88F8C8
:10AF100088F31188D5F800801A4406FB08F35B1A01
:10AF2000B3FBF8F306FB023341E5EFF311888CF332
:10AF3000128881680368DB0344BFCEF80070816823
:10AF40002368DEF800205FFA88F888F31188D5F8C6
:10AF500000801A4406FB08F35B1AB3FBF8F306FB08
:10AF6000023376E5EFF311888CF312888168036869
:10AF7000DB0344BFCEF8007081682368DEF8002050
:10AF80005FFA88F888F31188D5F800801A4406FB28
:10AF900008F35B1AB3FBF8F306FB0233BDE5EFF3EE
:10AFA00011888CF3128881680368DB0344BFCEF8F4
:10AFB000007081682368DEF800205FFA88F888F363
:10AFC0001188D5F800801A4406FB08F35B1AB3FB1E
:10AFD000F8F306FB0233F2E5EFF311888CF31288E5
:10AFE00081680368DB0344BFCEF800708168236882
:10AFF000DEF800205FFA88F888F31188D5F8008021
:10B000001A4406FB08F35B1AB3FBF8F306FB0233A2
:10B0100029E6EFF311888CF3128881680368DB035B
:10B0200044BFCEF8007081682368DEF800205FFA24
:10B0300088F888F31188D5F800801A4406FB08F3D5
:10B040005B1AB3FBF8F306FB023360E6EFF31188FB
:10B050008CF3128881680368DB0344BFCEF800706C
:10B0600081682368DEF800205FFA88F888F3118889
:10B07000D5F800801A4406FB08F35B1AB3FBF8F31B
:10B0800006FB023395E6EFF3118A8EF312888A6885
:10B090000B68DB0344BF3E608A682368D7F800C0B2
:10B0A0005FFA8AFA8AF31188D5F800A09C4400FB65
:10B0B0000AF39B1AB3FBFAF300FB0C33D5E6EFF36C
:10B0C00011828CF3128887680368D90303D50123A2
:10B0D000CEF8003087682368DEF80010D2B282F321
:10B0E00011882A68194406FB02F3DB1BB3FBF2F359
:10B0F00006FB01319AE5EFF311828CF31288876821
:10B100000368D90303D50123CEF80030876823688C
:10B11000DEF80010D2B282F311882A68194406FBC7
:10B1200002F3DB1BB3FBF2F306FB0131D8E4EFF3D0
:10B1300011828CF3128887680368D90303D5012331
:10B14000CEF8003087682368DEF80010D2B282F3B0
:10B1500011882A68194406FB02F3DB1BB3FBF2F3E8
:10B1600006FB01310EE5EFF311828CF3128887683C
:10B170000368D90303D50123CEF80030876823681C
:10B18000DEF80010D2B282F311882A68194406FB57
:10B1900002F3DB1BB3FBF2F306FB0131FFF7EABB63
:10B1A000EFF311828CF3128887680368D90303D503
:10B1B0000123CEF8003087682368DEF80010D2B291
:10B1C00082F311882A68194406FB02F3DB1BB3FBE8
:10B1D000F2F306FB01311FE4EFF311828CF31288C6
:10B1E00087680368D90303D50123CEF80030876848
:10B1F0002368DEF80010D2B282F311882A6819445D
:10B2000006FB02F3DB1BB3FBF2F306FB0131FFF796
:10B210000CBBEFF3118289F31288B8683B68D9033D
:10B2200003D50123C8F80030B8682368D8F80010A7
:10B23000D2B282F311882A6819440EFB02F31B1A5A
:10B24000B3FBF2F30EFB0131FFF741BBEFF31182C9
:10B250008CF3128887680368D90303D50123CEF8DD
:10B26000003087682368DEF80010D2B282F31188BC
:10B270002A68194406FB02F3DB1BB3FBF2F306FB5F
:10B28000013127E5EFF311828CF312888768036898
:10B29000D90303D50123CEF8003087682368DEF890
:10B2A0000010D2B282F311882A68194406FB02F317
:10B2B000DB1BB3FBF2F306FB01315DE5EFF3118617
:10B2C0008EF31288D1F808C00B68DA0303D5012386
:10B2D0003B60D1F808C023683A68F6B286F311885B
:10B2E0002E681A4400FB06F3A3EB0C03B3FBF6F342
:10B2F00000FB0233019392E503980122382109F003
:10B30000CDFC66E510223721039809F0C7FC0EE555
:10B310001A461921039809F0C1FCB6E41A461A210D
:10B32000039809F0BBFC5CE418221C21039809F087
:10B33000B5FC02E41A461B21039809F0AFFCFFF7A5
:10B340009EBB01226B21039809F0A8FCFFF73FBBCD
:10B35000019A03986B2109F0A1FCFFF7E6BA0722D6
:10B360006821039809F09AFCFFF78CBA80226B21C0
:10B3700009F094FCFFF732BA1D09013D032D03F0DB
:10B380000F0300F2B080614A32F8150040FA03F270
:10B39000D40740F1A880012404FA03F3013B1840CC
:10B3A00035F06AFC5A4B5B4A5B5D184412EBC005F2
:10B3B00000F0998000232021EB71A97152F8300030
:10B3C000554A00F13F4303F57E039B0AD25C02F02D
:10B3D0001F035209032A04FA03F300F09280042A9F
:10B3E00000F08A80022A79D0AB88049304A9002354
:10B3F000059324F003FD0299484B41F80C3F284681
:10B400002DF082FEAB88B3FA83F3C3F11F03012250
:10B4100012FA03F33FF4D7A941490A6813430B60BA
:10B42000FFF7D1B902980723417D90F914006822F3
:10B43000FFF766F9FFF726BA02988023417D90F95D
:10B4400014006B22FFF75CF9FFF7C8B90846192210
:10B45000497D90F91400FFF753F916E408461A22C3
:10B46000497D90F91400FFF74BF9FFF7BABB02983A
:10B470003822417D90F91400FFF742F9A9E40298BF
:10B480001023417D90F914003722FFF739F94EE47B
:10B4900002986B22417D90F91400FFF731F9FFF714
:10B4A00096BA0298019B417D90F914006B22FFF738
:10B4B00027F9FFF73ABA02981823417D90F9140052
:10B4C0001C22FFF71DF9FFF738BB02981B22417DB4
:10B4D00090F91400FFF714F9FFF7D1BA114A516C33
:10B4E0000B43536480E702990C4B41F80C3F00205A
:10B4F0002DF00AFEFFF767B90A4A116B0B4313637D
:10B5000072E7084A116C0B4313646DE72C51040871
:10B51000285104087C830020B84F0408A584000843
:10B52000003C0140003802402DE9F04F8A4A43694F
:10B5300083B09342019000F00D8188498B420CBF8B
:10B54000282130211A8822F040021204120C1A809D
:10B550001A8892B222F03802114319801A8892B2E6
:10B5600042F040021A80012001F0EAFE019C2046D0
:10B57000FFF720F9A36913B11A689B885383019BD5
:10B58000586940F2E93302E0002B00F0DB800289C9
:10B59000013B12F0020F9BB2F6D06A23838140F286
:10B5A000E93302E0002B00F0CD800289013B12F06C
:10B5B000010F9BB2F6D0838940F2E93302E0002B01
:10B5C00000F0C5800289013B12F0020F9BB2F6D059
:10B5D0001023838140F2E93302E0002B00F0B780B2
:10B5E0000289013B12F0010F9BB2F6D08389019BC7
:10B5F0009B6913B11A689B881383594CDFF86CE17F
:10B60000DFF86C915748584F4FF0640A4FF0100C18
:10B610004FF47A75D9F80430C3F30803002B76D1C0
:10B62000EFF31183002B72D12168826800BF236879
:10B630009942F9D1DEF8006005FB06F39B1AB3FBD3
:10B64000F6F305FB013101260091D9F80430C3F36C
:10B650000803002B40D1EFF31183002B3CD123686A
:10B66000816800BF22689342F9D1DEF800B005FB83
:10B670000BF2521AB2FBFBF205FB0323009A9B1A52
:10B68000B3F57A7FE1D3BAF1010AC3D1019B324A03
:10B690005B69934207D0DFF8C4A0534514BF4FF055
:10B6A000080A4FF0000A1A8822F040021204120C15
:10B6B0001A801A8892B222F038024AEA020AA3F8E3
:10B6C00000A01A8892B242F0400201201A8003B012
:10B6D000BDE8F04F01F034BEEFF311888CF312880F
:10B6E00081680368DB0344BF3E60816823683A6871
:10B6F0005FFA88F888F31188DEF800801A4405FBA9
:10B7000008F35B1AB3FBF8F305FB0233B6E7EFF37C
:10B7100011828CF3128886680368D90302D501234D
:10B720003B60866823683968D2B282F31188DEF8FC
:10B730000020194405FB02F39B1BB3FBF2F305FB4E
:10B74000013180E709F08FFA019B586934E709F06D
:10B750008AFA4CE72821F5E600380040003C00401A
:10B760003C85002010E000E0388500204085002066
:10B7700000ED00E00220FCF77BBF0220FEF76EBF69
:10B780000120FCF775BF0120FEF768BF0020FCF721
:10B790006FBF0020FEF762BF1549164B16480A68B6
:10B7A00010B48C681549B2FBF4F203FB02F303609A
:10B7B000D1F88820124B134C42F47002C1F8882053
:10B7C0001A68002042F001021A6098601A6822F09C
:10B7D000847222F480321A605C601A684FF0006450
:10B7E00022F480221A60D8608C605DF8044B7047A8
:10B7F0000000002040420F00F082002000ED00E039
:10B800000038024010300024044B4FF4F0700A213D
:10B81000022283E80700FFF7BFBF00BF000000203F
:10B8200038B50B4C23688BB15A68821A002A05463A
:10B8300004DA0CE05A68AA1A002A07DB9A68226028
:10B8400018461A6890472368002BF3D138BD38BDDD
:10B85000CC3E00200B4B002210B4027203F584741E
:10B86000032102E0072A09DC9979890702D51979B1
:10B87000815401329C4203F11803F3D15DF8044B6B
:10B88000704700BF085004082E230370704700BFA4
:10B89000012332213122417042710372037003711E
:10B8A000704700BF2322032302704370704700BF1C
:10B8B0002DE9F0410B78047BDB43DEB200F110028E
:10B8C00000F1380342F8044F9342FBD1DFF89CC0EB
:10B8D00000F16001002243F8042F8B42FBD14FF0AE
:10B8E000140E0521002546FA01F303F00103002B95
:10B8F0001D4414BF4FF019084FF00A0811F0010F52
:10B90000EDB214BF2746002700220EEB02039BB2C4
:10B9100000EB8303013242455F61F6D1013A92B2F6
:10B92000013201390EEB02034A1C9BB201D09E4644
:10B93000D9E715F0010F14BF19250A2500215A185F
:10B9400092B200EB82020131A9425461F7D10B445B
:10B950009BB21A1D00EB8202013300219BB25160A1
:10B96000ACF800300361BDE8F08100BF981F0020F3
:10B97000254B5B880B332DE9F04F8A4601F1060B0E
:10B980001FFA83F94FF00108002100271AF801EB94
:10B990003E464C460122A4F10B039BB207E0013363
:10B9A0009BB2B0F80CC0C5F814C09C420AD000EBA2
:10B9B0008305002AF3D100EB830501339BB29C423F
:10B9C0006A61F4D1231D00EB83030136092FF6B21F
:10B9D00059600CD0092E14D008FA07F313EA0E0FA1
:10B9E00014BF012200220C34A4B20137D3E709F1BD
:10B9F0007809DA451FFA89F9C7D1034B5980BDE8A8
:10BA0000F08F0022EFE700BF981F00202DE9F047DC
:10BA1000DFF85C80B8F8043004338A461FFA83FCF0
:10BA200001F109094FF0010E1AF8017B6446002666
:10BA3000231F0EFA06F29BB23A40BAB1818900EB9D
:10BA4000830501339BB29C426961F6D1013604340F
:10BA5000082EA4B2ECD10CF1200CCA451FFA8CFCC4
:10BA6000E2D10023A8F80430BDE8F0871146E6E7EC
:10BA7000981F002010B5027B01681F2A4FF0200399
:10BA80000ED94C68203A93401C4216D00B4A4068AD
:10BA900000241470026822F001020260CB6010BD25
:10BAA0000C6893401C4208D0044A4068002414707B
:10BAB000026822F0010202608B6010BD5528002050
:10BAC000436A8269D154436A0169826B01338B42B4
:10BAD00028BF00234362002A2FD0EFF311825023A6
:10BAE00083F31288836B1968C9072CD470B45E681D
:10BAF0006EB9456A816A8D4217D084690C44DC6056
:10BB00000ED9691A59608562002180F85C101968A5
:10BB100041F00101D2B2196082F3118870BC704704
:10BB20000469611A59608662EEE7012380F85C308F
:10BB3000D2B282F3118870BC7047826DD36843F033
:10BB40008003D3607047D2B282F31188704700BF80
:10BB5000426B10B462B1C36CC2684469D11A013B34
:10BB6000615C5DF8044B08BF1346C364C8B27047FC
:10BB7000016A4369C4685B5C0131A14228BF114678
:10BB800001625DF8044BD8B2704700BF836B13B1FC
:10BB900090F85C007047836A406A181AB0FA80F027
:10BBA00040097047416A836A99420AD3CB1A816B74
:10BBB000026961B14968501E0B4483420AD2C01A1F
:10BBC000704702691144CB1A816B0029F2D1501ED3
:10BBD000C01A704700207047436B43B1C26C5B686A
:10BBE00093422FBF981AC0689B1AC0187047C26949
:10BBF000036A9A422FBFD01AC0688018C01A7047D3
:10BC00002DE9F0478C4B1B78DB07074644D58B4B5F
:10BC10008B4D1C788B4E012C59D01CD3022C07D194
:10BC200089498A4A09881288914201D901241C70E5
:10BC3000EB7AE3B12B89D3B1854B1B78BBB114F000
:10BC400017FF002800F09B802B7B83422CBF012133
:10BC5000002131700CE07C497E4A098810886A7B9B
:10BC6000801A8842E2DAEB7A0024002BE2D13178A4
:10BC70002A79632A06D8022C774E00F0BA803378EE
:10BC8000002B5DD1754AAB7A8C4238BF0C461470DC
:10BC9000002B4CD1BDE8F0876B4B694D19885B8850
:10BCA000E878CB1A83EAE3728142A2EBE3721DD3F8
:10BCB0002B788B421AD3614B1C78E01E012861D986
:10BCC0006749097802294FD0012C5E4EA5D15F4A01
:10BCD0005D491288687B0988121A914239DD5D4AF4
:10BCE00012888A42A4D200241C70A1E7B1EB400F55
:10BCF000E1DC524B1C78E11E012940F29480022ABB
:10BD0000DEDC57494F4E0878DFF84481DFF844C144
:10BD1000DFF838E100210324022834701C7088F811
:10BD20000010ACF80010AEF8001081D11FE0012C1B
:10BD300071D0022C0BD10720BDE8F0472FF088BE50
:10BD40007068381A474B984258DD72709AE7BDE820
:10BD5000F08702241C706BE7022AD2DD4049097883
:10BD600002294FF0040464D13949364E09783E481F
:10BD7000022ACCBF00220122C28081804BE702212F
:10BD8000317075E7022A9BDC95F800C091FBFCFC42
:10BD90000CF1010CBCF1080FDFF8B4A0304EA8780C
:10BDA00095F801E096F800802A4CDFF8A090254E27
:10BDB000A8BF4FF0080C8AF800C01FFA8CFA10FBDD
:10BDC0000AF01EFB0AFE80B2DFF88CA02080A9F8E2
:10BDD00000E000244FF0640EB8F1020F34701C70C4
:10BDE000CAF804408AF801E07FF439AF0FFA8CF109
:10BDF000BDE73078A0B9012377603370C2F16402E7
:10BE00001A4B00FB02F083FB0023C017A0EBA350EA
:10BE10006430707036E70820BDE8F0472FF018BE98
:10BE20007368F81A8EE7032C96D10D490978022918
:10BE30009AD0044EFCE600BF006200204C2800208F
:10BE4000B851002052280020189A002050280020C5
:10BE50002E9A00204E280020B42600201D470020E6
:10BE60003C9900207F969800409900206BCA5F6B38
:10BE7000038A2DE9F0478589ADB21D4029D00F46D0
:10BE800006464FF000484FF00009B5FA85F328FA4E
:10BE900003F2D24391B21B3B15403182042B16D8DA
:10BEA000DFE803F03129211903007B6A002B32D02F
:10BEB00003F1FF3A1FFA8AFAC7F824903C6A34B1BA
:10BEC00023682046514698476468002CF8D1002D1D
:10BED000DBD1BDE8F0873868716B036889B2984799
:10BEE000002DD2D1F5E77868B16B036889B2984725
:10BEF000002DCAD1EDE7B868F16B036889B29847A5
:10BF0000002DC2D1E5E7F868316C036889B2984723
:10BF1000002DBAD1DDE7F36A1FFA83FACEE700BF3E
:10BF20001C4C08B50121022008F054FD237803F0D1
:10BF30000502052A29D003F00903092B08D00021A6
:10BF4000012008F047FD0021084608F043FDFEE708
:10BF5000114A124B11681A680B68114C23F0010347
:10BF60000B601388206823F001031B041B0C138053
:10BF700018B12A2200238271C37109224A2108F0D4
:10BF800093FB206808F014FDD9E727F0BFF8237869
:10BF9000D1E700BF803A00206028002064280020FC
:10BFA000783B0020022828BF022010B4084C094B1F
:10BFB000207000EB8002C0EBC20207495DF8044B21
:10BFC000013003EB4203C0B20B602FF067BE00BF2D
:10BFD000289C0020386200202852002008B517F065
:10BFE000B9FC09F08FF8BDE8084017F09BBC00BF12
:10BFF0002DE98048013085B0C3B203938B4D8C4F3F
:10C000008C4C8D4E0A2302933220DFF830922CF0B4
:10C01000BDFD4FF4FA7A4FF0100C4FF47A70D9F856
:10C020000430C3F30803002B40F0C180EFF3118309
:10C03000002B40F0BC802968A26800BF2B689942A1
:10C04000F9D1D7F800E000FB0EF39B1AB3FBFEF327
:10C0500000FB01314FF0010E0191D9F80430C3F318
:10C060000803002B40F08780EFF31183002B40F092
:10C0700082802B68A16800BF2A689342F9D1D7F863
:10C0800000B000FB0BF2521AB2FBFBF200FB0323E1
:10C09000019A9B1AB3F57A7FDFD3BAF1010ABED1B8
:10C0A000039B002B40F0BD804FF47A7ADFF88C912F
:10C0B00050464FF0100CD9F80430C3F30803002B9E
:10C0C00040F09280EFF31183002B40F08D802968BF
:10C0D000A26800BF2B689942F9D1D7F800E000FBB5
:10C0E0000EF39B1AB3FBFEF300FB01314FF0010E80
:10C0F0000191D9F80430C3F3080303BBEFF31183B4
:10C10000EBB92B68A16800BF2A689342F9D1D7F830
:10C1100000B000FB0BF2521AB2FBFBF200FB032350
:10C12000019A9B1AB3F57A7FE3D3BAF1010AC2D11F
:10C13000029B013B02937FF467AFFDF749F8EFF3F1
:10C1400011888CF31288A1682368DB0344BFC6F80A
:10C1500000E0A1682B6832685FFA88F888F31188DC
:10C16000D7F800801A4400FB08F35B1AB3FBF8F31E
:10C1700000FB0233D4E7EFF311888CF31288A16837
:10C180002368DB0344BFC6F800E0A1682B6832686F
:10C190005FFA88F888F31188D7F800801A4400FB0A
:10C1A00008F35B1AB3FBF8F300FB023370E7EFF31D
:10C1B00011828CF31288D4F808E02368D90303D5E0
:10C1C00001233360D4F808E02B683168D2B282F3DF
:10C1D00011883A68194400FB02F3A3EB0E03B3FB8A
:10C1E000F2F300FB013135E7EFF311828CF3128893
:10C1F000D4F808E02368D90303D501233360D4F8C9
:10C2000008E02B683168D2B282F311883A68194489
:10C2100000FB02F3A3EB0E03B3FBF2F300FB0131CF
:10C2200064E718462CF014FB3EE700BF3C85002075
:10C230004085002010E000E03885002000ED00E09F
:10C2400038B5484B5A899989914224BF00225A81B6
:10C25000198ADA89914224BF0022DA81DA78CAB1D8
:10C26000072A41496AD091F85300404D012400212A
:10C270000A282C709C70D9715DD00C2807D0002A38
:10C280006CD0DFED3B7A072A0ED00A2862D0DFEDB2
:10C29000397A09E0344A92F853000A2856D00C281B
:10C2A0005BD1D979DFED347A344C9FED350AA27831
:10C2B000002918BFF0EE407A062A04D8314901EB74
:10C2C000820191ED000A217979B1013A032A0BD854
:10C2D000F7EE007A87EE800A35F052F8238898420C
:10C2E00028BF1846208038BD38BD9B781F4A07EE0E
:10C2F000103A1178B8EEC77A67EE277A07EE101A6F
:10C30000B8EEC77A27EE277AB4EEC70AF1EE10FA34
:10C31000EADD80EE277AFDEEC77A17EE903A102B11
:10C32000A8BF1023012BB8BF0123DBB28B4238BF5B
:10C330000B46137038BDDFED147AA4E791F8530073
:10C340000A2803D00C28ACD0D9799AE7D979DFED47
:10C350000E7AA9E7DFED0D7AA6E7D979DFED047A49
:10C36000A2E700BF9C8D0020C0850020306E002019
:10C370006F1203396F12833A0AD7A339C08F002096
:10C380006F120338082404085304E9380F506E3A3A
:10C390002DE9F047AA4FAB4E17F0DCFABE421ED291
:10C3A000DFF82483DFF824934446258862197DB1A1
:10C3B0004A450DD2052D0BD933886188C3F30B0391
:10C3C000994200F0E080144625886219002DEFD1D3
:10C3D00071683046143608F021FEBE42E4D39A4A12
:10C3E0001378A3F1170102290FD9984911F83300E6
:10C3F000002840F0F780D8000144497829B19449D9
:10C4000011F833300BB918231370924B5A78022A63
:10C4100000F2D9809049914802EB420201EB82017F
:10C420001A780160022A00F2D78002EB82018C4B5D
:10C43000C2EBC10203EB4203998C5A8C894C9142A6
:10C44000236001D300225A84874B9A78042A00F093
:10C45000EA8032B91A88B2F5F07F84BF4FF4F072E7
:10C460001A80824DFFF7ECFE2B68814A1A40002AA1
:10C4700000F0E280D80700F1D180590400F1C980B2
:10C480001A0700F1B8809B0400F1BC802BF0D2FBAE
:10C4900010B978482EF098FD4FF4007008F0F4FDC4
:10C4A0004FF4802008F0F0FD4FF0007008F0ECFD34
:10C4B0004FF0806008F0E8FD27F00EFB00213022ED
:10C4C0006D4835F01AFF206826F056FA6B4B256848
:10C4D00003F1500103E00433994200F081801A789F
:10C4E000002AF8D19C78D8788442F4D26449654B0C
:10C4F0000A7028461D6029F0E9FE634A63491079F5
:10C50000634A644B1160C822642111FB00210022A0
:10C5100059609A60DA601A615A619A61DA6183F847
:10C52000202083F8212020F097FD5B4B9FED5B5A84
:10C530001B885B4A9FED5B6A55795B4C5B495C48A5
:10C54000086006EE903AF8EEE66A1388C5EE265AC1
:10C5500007EE103A53881279C4ED005A07EE903A6C
:10C56000B8EEC77A534BF8EEE77A1D725A7227EE8F
:10C57000067A67EE867ABDE8F04783ED017AC3ED6F
:10C58000007A17F0CFB963799B077FF41CAF71680D
:10C5900094F804A0304608F041FD3388BAEB133F0D
:10C5A00004D01436BE42FFF4FFAE18E773887068FB
:10C5B000AA1FC3F30B039A4204F10601A8BF1A464F
:10C5C00034F09EFDEDE700225A701A782348224984
:10C5D0000160022A7FF629AF00221A70204B2BE758
:10C5E000012283E7D8000C186468002C7FF404AFA4
:10C5F0001724147000E7304808F046FD2B689B04B0
:10C600007FF544AF2D4808F03FFD402008F03CFD89
:10C610003CE72B4808F038FD2B6831E7294808F043
:10C6200033FD2B6829E79A8AB2F57A7FBFF419AFF8
:10C630004FF47A729A8214E743F008032B6019E7EB
:10C6400040060008900100086C6E0020E0540408C9
:10C65000082F0408289C0020349C00202C52002025
:10C660003862002028520020C08F00206C63002018
:10C67000096000027C76002098240020303F0020D2
:10C68000981D0020CC240020A06B0020426E0020CA
:10C69000D023002020470020E8260020C0C9FB4806
:10C6A000EC24002017B7D138EC2600200C660020BF
:10C6B0003661023DE8650020016000020940000289
:10C6C0000920000208600002024000080080000803
:10C6D00008B517F03FF908F015FD17F023F9FFF73B
:10C6E00057FE0120BDE808402FF0D8BA38B50C4CF1
:10C6F0000C4DAC4206D261682046143408F08EFC22
:10C70000AC42F8D3084A094B094C1460002209498D
:10C710001A705A7008480860BDE838401EF074B9B5
:10C72000900100084006000828520020289C0020A4
:10C73000386200202C520020349C002008B5FFF7FE
:10C74000D5FF17F007F908F0DDFCBDE8084017F049
:10C75000E9B8054B10B59A68044C2178501C09B90A
:10C760009A6010BD0246F8E7981F00205528002067
:10C77000F0B50C2934D8DFE801F0893333335E3368
:10C780003333343333330700048C9689B2F802E034
:10C790001788734D24F480542404240C0484038CDF
:10C7A0008488818B23F4005321F4E6411B0409049F
:10C7B0001B0C46EA0E06090C43EA063341EA072140
:10C7C000A8429BB2A4B289B200F09E8005F58065B4
:10C7D000A84200F099809268848081830264038477
:10C7E000F0BD048C9589B2F802C0B2F800E05C4F4D
:10C7F00024F480742404240C0484038C8688818BA4
:10C8000023F400731B0421F073011B0C45EA0C0494
:10C81000090443EA0423090CB8429BB2B6B241EAC8
:10C820000E015CD04F4CA04259D092688680818323
:10C83000C2630384F0BD048C9589B2F802C0B2F8DB
:10C8400000E0474E24F010042404240C0484038CDC
:10C850008788018B23F0200321F4E6411B0409049F
:10C860001B0C45EA0C04090C43EA041341EA0E21AF
:10C87000B0429BB2BFB289B25DD03A4CA0425AD00E
:10C8800092688780018382630384F0BD048C97895A
:10C89000B2F802E01688324D24F001042404240C7E
:10C8A0000484038C8488018B23F002031B0421F091
:10C8B00073011B0C47EA0E0709043B43090CA8420D
:10C8C0009BB2A4B241EA060125D005F58065A842D5
:10C8D00021D092688480018342630384F0BDD589AE
:10C8E000148A578A23F4006343EA05254FF6FF3381
:10C8F0002B40958826F440563C4343EA052346EAFC
:10C9000004169BB2B6B290E7158A24F4804444EA38
:10C910008514A4B25FE7D689158A578A23F00803E5
:10C92000334324F4407496883D4323F004032C439E
:10C930003343A4B2CDE7D489158A568A23F0800305
:10C9400043EA04134FF6BF741C40938827F44067F2
:10C95000354344EA031347EA85079BB2BFB28FE72A
:10C9600000000140000401402DE9F04FC8220021E1
:10C9700083B08A488A4CDFF84C928A4D8A4E8B4F9E
:10C98000DFF8448235F0B9FC89488A49DFF83CE297
:10C99000DFF83CC200221359834200F0D580B3F186
:10C9A000804F00F0DC80AB4200F0E480B34200F046
:10C9B000E380BB4200F0E280734500F0E180634514
:10C9C00000F0E080434500F0DF80DFF808A2534527
:10C9D00000F0DC800AF5806A534500F0D9800AF542
:10C9E000806A534500F0D680AAF5983A534500F086
:10C9F000D3800AF5806A534500F085800AF5806A85
:10CA0000534508BF0D237FD01832B2F5907FC2D1B5
:10CA1000634C694E694F6A4D04F5907802E0183412
:10CA2000A0456DD0A379002BF9D023794FEA1319D3
:10CA300009F1FF39B9F1030F03F00F03EFD836F80E
:10CA4000190040FA03F2D207E9D54FF0010A0AFAB9
:10CA500003F3013B184034F00FF917F8093018447C
:10CA600015EBC002DBD055F83000DFF86CE1217A1D
:10CA700000F13F4303F57E039B0A1EF8033003F0E9
:10CA80001F0E5B09032B0AFA0EFA5FD0042B68D045
:10CA9000022B07D1DFF81CE1DEF844304AEA030339
:10CAA000CEF8443093880093B3FA83F3C3F11F03A5
:10CAB0009BB2DA0800EB820203F00703D2F820E011
:10CAC0009B004FF00F0C0CFA03FC2EEA0C0EC2F880
:10CAD00020E0D2F820E001FA03F343EA0E031362E8
:10CAE00069460023022218348DF804208DF80530A1
:10CAF0008DF806308DF8073023F080F9A04591D1EC
:10CB000003B0BDE8F08F0C2309EBC3034FF0010A1B
:10CB10001B7903F01F0B5B09032B0AFA0BFA09D0F0
:10CB2000042B0CD0022B7FF46FAF4B6C4AEA03034B
:10CB30004B6469E70B6C4AEA03030B6464E70B6B15
:10CB40004AEA03030B635FE70023DDE7DFF864E0F5
:10CB5000DEF840304AEA0303CEF84030A2E7012372
:10CB6000D2E7DFF850E0DEF830304AEA0303CEF8CF
:10CB7000303097E70223C7E70323C5E70423C3E761
:10CB80000523C1E70623BFE70723BDE70823BBE76B
:10CB90000923B9E70A23B7E70B23B5E7946F002011
:10CBA000085004080004004000080040000C004049
:10CBB00000000140003802402C51040828510408AC
:10CBC0007C830020605104080004014000100040F4
:10CBD0000014004000400140B84F040801490248D9
:10CBE000FFF746B9347000200018004001490248A0
:10CBF000FFF73EB90C7000200004014001490248D3
:10CC0000FFF736B90C7000200004014001490248CA
:10CC1000FFF72EB9E46F0020000C004001490248E4
:10CC2000FFF726B9BC6F00200004004002494FF016
:10CC30008040FFF71DB900BF946F0020F0B5046875
:10CC4000474DA30AAB426ED009D8B3F5801F66D01A
:10CC5000023DAB4258D14FF0480E012608E0414D4D
:10CC6000AB4264D03B35AB424FD14FF0980E032618
:10CC70004779B0004FEA970C00295CD06346022741
:10CC8000A5899F4083190CEB43032F4303F1040C48
:10CC9000354DBFB245F8231045F82C20A781EFF39E
:10CCA0001181502282F31288821905EBC2021369A6
:10CCB00063B313620433821905EBC202576917B1DB
:10CCC0001F6053690433821905EBC202976917B1DB
:10CCD0001F6093690433821905EBC202D76917B14B
:10CCE0001F60D36904330027CAB21F6082F3118822
:10CCF000304405EBC000036A5BB9A38923F001034C
:10CD00001B041B0CA381F0BDF0BDF0BD05EB0E03B1
:10CD1000D1E7A3899BB243F00103A381F0BD4FF09B
:10CD2000200E0026A4E74FF0700E0226A0E74FF079
:10CD3000C00E04269CE70223BF0803FA07F7A38965
:10CD4000094D9BB223EA070387190CEB470CA3811B
:10CD50000CF1040345F82C1045F823209FE700BF91
:10CD60000300100006001000946F002010B5036847
:10CD700082480139834282B089B200F0CA80A0F5AE
:10CD80008060834200F0C58000F58040834200F05F
:10CD9000B78000F58060834200F0B28000F58060CB
:10CDA000834200F0AD80764C188824686408B4FB98
:10CDB000F2F4013CA4B282B2B3F1804F0AD07148C0
:10CDC000834207D000F58060834203D000F5806085
:10CDD000834202D122F0700292B26B48834200F08B
:10CDE000A18000F58060834200F0A68022F44072AA
:10CDF00000F56C4092B283421A80D9621C854FD0F4
:10CE00005E4A93424CD001229A821A8892B242F032
:10CE100001021A80B3F1804F00F09880594A934282
:10CE200000F0968002F58062934200F0938002F554
:10CE30008062934200F0908002F58062934200F09D
:10CE40008D8002F58062934200F08A8002F5704284
:10CE5000934200F0878002F57052934200F0848084
:10CE600002F58062934200F0818002F58062934275
:10CE70007ED0A2F5983293427CD002F58062934234
:10CE80007AD002F58062934208BF0D2215D002A825
:10CE90004FF0012340F8043D22F020FD02B010BD08
:10CEA0000122002119869A821A88384892B242F0EB
:10CEB000010283421A80ADD10A46354B03EBC2030F
:10CEC00001A85C798DF80440012300228DF805301B
:10CED0008DF807308DF8062022F000FD1B2C08D0BD
:10CEE0002E2CDBD12B4B019301A822F0F7FC02B0D2
:10CEF00010BD294B019301A822F0F0FC02B010BD37
:10CF00001F4C18882468B4FBF2F4013CA4B282B22E
:10CF100052E71B4C18882468B4FBF2F4013CA4B21D
:10CF200082B257E701201A80D9621C8598821A883C
:10CF300092B202431A8071E701201A80D9621C85DF
:10CF400098821A8892B202431A8063E70122B4E7FA
:10CF50000222B2E70322B0E70422AEE70522ACE7E3
:10CF60000622AAE70722A8E70822A6E70922A4E7E3
:10CF70000A22A2E70B22A0E70C229EE70004014050
:10CF8000F08200200004004000100040000001403A
:10CF9000605104082C010001190100012B4B98423B
:10CFA0003CD0B0F1804F3BD0A3F57C43984239D0C0
:10CFB00003F58063984237D003F58063984235D0FB
:10CFC00003F58063984233D003F58063984231D0F3
:10CFD00003F5704398422FD003F5705398422DD03B
:10CFE00003F5806398422BD003F58063984229D0E3
:10CFF000A3F59833984227D003F58063984207D071
:10D0000003F58063984208BF0D2202D000207047CC
:10D010000C220F4B03EBC203187970470022F8E78C
:10D020000122F6E70222F4E70322F2E70422F0E706
:10D030000522EEE70622ECE70722EAE70822E8E706
:10D040000922E6E70A22E4E70B22E2E700000140BA
:10D05000605104082DE9F04F013085B0C3B203934D
:10D060000B4602918B4C8C4E002B00F09A803220A4
:10D070008A4D8B4FDFF82C922BF088FD4FF4FA7A13
:10D080004FF0100C4FF47A70D9F80430C3F3080352
:10D09000002B40F0DE80EFF31183002B40F0D980AD
:10D0A0002968A26800BF2B689942F9D1D7F800E03F
:10D0B00000FB0EF39B1AB3FBFEF300FB01314FF0B4
:10D0C000010E0191D9F80430C3F30803002B40F09E
:10D0D0008780EFF31183002B40F082802B68A168DA
:10D0E00000BF2A689342F9D1D7F800B000FB0BF2D9
:10D0F000521AB2FBFBF200FB0323019A9B1AB3F511
:10D100007A7FDFD3BAF1010ABED1039B002B40F036
:10D11000BD804FF47A7ADFF88C9150464FF0100CB6
:10D12000D9F80430C3F30803002B75D1EFF3118352
:10D13000002B71D12968A26800BF2B689942F9D1F0
:10D14000D7F800E000FB0EF39B1AB3FBFEF300FBE5
:10D1500001314FF0010E0191D9F80430C3F30803F7
:10D1600013BBEFF31183FBB92B68A16800BF2A68DA
:10D170009342F9D1D7F800B000FB0BF2521AB2FB80
:10D18000FBF200FB0323019A9B1AB3F57A7FE3D3EA
:10D19000BAF1010AC4D1029B013B0293002B7FF438
:10D1A00066AF05B0BDE8F08FEFF311888CF31288FD
:10D1B000A1682368DB0344BFC6F800E0A1682B68C0
:10D1C00032685FFA88F888F31188D7F800801A442B
:10D1D00000FB08F35B1AB3FBF8F300FB0233D2E762
:10D1E000EFF311888CF31288A1682368DB0344BF36
:10D1F000C6F800E0A1682B6832685FFA88F888F307
:10D200001188D7F800801A4400FB08F35B1AB3FBBF
:10D21000F8F300FB023370E7EFF311828CF312880E
:10D22000D4F808E02368D90303D501233360D4F888
:10D2300008E02B683168D2B282F311883A68194449
:10D2400000FB02F3A3EB0E03B3FBF2F300FB01318F
:10D250007FE7EFF311828CF31288D4F808E023689B
:10D26000D90303D501233360D4F808E02B68316873
:10D27000D2B282F311883A68194400FB02F3A3EB9F
:10D280000E03B3FBF2F300FB013118E718462BF055
:10D29000DFFA3EE710E000E0388500203C85002002
:10D2A0004085002000ED00E0204B5B68C3F30803DD
:10D2B00030B4BBB9EFF31183A3B91D4B1D4C1868F3
:10D2C000A16800BF1A689042F9D11B4B1C684FF44B
:10D2D0007A7202FB04F3591AB1FBF4F130BC02FB81
:10D2E00000107047EFF31182102383F31288114965
:10D2F0008C680B6813F4803F104B02D0012018603B
:10D300008C680B49D2B20D68186882F311880A4BF9
:10D3100019684FF47A72284402FB01F31B1B30BCDE
:10D32000B3FBF1F302FB0030704700BF00ED00E0FB
:10D330003C85002010E000E040850020388500207A
:10D340002DE9F84F8046FFF7AFFF254E2549DFF85E
:10D35000A0E0254A254D844610274FF47A74012019
:10D36000DEF80430C3F30803D3B9EFF31183BBB97C
:10D370000B68D2F808A000BFD1F800904B45F7D158
:10D38000D6F800B004FB0BF9A9EB0A09B9FBFBF9CD
:10D3900004FB0393A3EB0C034345E1D3BDE8F88FF3
:10D3A000EFF3118A87F31288D2F808B01368DB0311
:10D3B00044BF2860D2F808B00B68D5F800905FFA37
:10D3C0008AFA8AF31188D6F800A0994404FB0AF37C
:10D3D000A3EB0B03B3FBFAF304FB0933DAE700BF5B
:10D3E000408500203C85002010E000E038850020CA
:10D3F00000ED00E02DE9F04FDFF830C1474A484921
:10D40000484E494D8046102718F1FF38C0F08480FF
:10D41000DCF80430C3F30803002B5CD1EFF3118375
:10D42000002B58D10B68946800BF08688342F9D17B
:10D43000D6F800904FF47A7000FB09FEAEEB040EB4
:10D44000BEFBF9FE00FB03EEDCF80430C3F3080377
:10D450004FF47A740120FBB9EFF31183E3B90B6841
:10D46000D2F808A000BFD1F800904B45F7D1D6F80C
:10D4700000B004FB0BF9A9EB0A09B9FBFBF904FBAB
:10D480000393A3EB0E03B3F57A7FBDD2DCF804302F
:10D49000C3F30803002BDFD0EFF3118A87F3128860
:10D4A000D2F808B01368DB0344BF2860D2F808B094
:10D4B0000B68D5F800905FFA8AFA8AF31188D6F8DB
:10D4C00000A0994404FB0AF3A3EB0B03B3FBFAF3AC
:10D4D00004FB0933D5E7EFF3118487F31288D2F800
:10D4E00008901368D80303D501232B60D2F8089065
:10D4F0000B682868E4B284F31188D6F800A04FF4D2
:10D500007A7400EB030E04FB0AF3A3EB0903B3FBED
:10D51000FAF304FB0E3E97E7BDE8F08F10E000E061
:10D520003C850020408500203885002000ED00E08B
:10D5300030B4EFF31183102282F312880649074CAE
:10D540000A680748013200250A602560DBB20268DC
:10D5500083F3118830BC70473C850020388500205B
:10D5600010E000E00F4B1B88014643B90E4B0F4AF9
:10D570001B7810680BB981F0010107F023BA0C4B3E
:10D580005A691AB118B91A68106058747047094A74
:10D5900018681188084A92FBF1F20121026059745F
:10D5A000704700BF148500201685002018850020D4
:10D5B0001C8500203485002020A1070038B5264BAB
:10D5C0005C69636B73B1A36DA26BD2B1998A1A883F
:10D5D000C90592B201D5D20700D438BD4FF6F77213
:10D5E0001A8038BDA36D99891A88890692B2EBD545
:10D5F0009206E9D5E26AD2B19888216B80B2904751
:10D60000E1E799891A880D0692B2DFD51006DDD5BB
:10D61000A26A616A8A4219D0A1692569885C9880EA
:10D620000132B2FBF5F105FB1122A262CEE79B8825
:10D63000E2696169DBB28B54E269E068A36D013293
:10D64000B2FBF0F100FB1122E261BDE7DA6822F0E3
:10D650008002DA60BAE700BF843A002038B5264B72
:10D66000DC68636B73B1A36DA26BD2B1998A1A881F
:10D67000C90592B201D5D20700D438BD4FF6F77272
:10D680001A8038BDA36D99891A88890692B2EBD5A4
:10D690009206E9D5E26AD2B19888216B80B29047B0
:10D6A000E1E799891A880D0692B2DFD51006DDD51B
:10D6B000A26A616A8A4219D0A1692569885C98804A
:10D6C0000132B2FBF5F105FB1122A262CEE79B8885
:10D6D000E2696169DBB28B54E269E068A36D0132F3
:10D6E000B2FBF0F100FB1122E261BDE7DA6822F043
:10D6F0008002DA60BAE700BF843A002038B5264BD2
:10D700009C68636B73B1A36DA26BD2B1998A1A88BE
:10D71000C90592B201D5D20700D438BD4FF6F772D1
:10D720001A8038BDA36D99891A88890692B2EBD503
:10D730009206E9D5E26AD2B19888216B80B290470F
:10D74000E1E799891A880D0692B2DFD51006DDD57A
:10D75000A26A616A8A4219D0A1692569885C9880A9
:10D760000132B2FBF5F105FB1122A262CEE79B88E4
:10D77000E2696169DBB28B54E269E068A36D013252
:10D78000B2FBF0F100FB1122E261BDE7DA6822F0A2
:10D790008002DA60BAE700BF843A002038B5264B31
:10D7A0001C68636B73B1A36DA26BD2B1998A1A889E
:10D7B000C90592B201D5D20700D438BD4FF6F77231
:10D7C0001A8038BDA36D99891A88890692B2EBD563
:10D7D0009206E9D5E26AD2B19888216B80B290476F
:10D7E000E1E799891A880D0692B2DFD51006DDD5DA
:10D7F000A26A616A8A4219D0A1692569885C988009
:10D800000132B2FBF5F105FB1122A262CEE79B8843
:10D81000E2696169DBB28B54E269E068A36D0132B1
:10D82000B2FBF0F100FB1122E261BDE7DA6822F001
:10D830008002DA60BAE700BF843A002070B4EFF3E8
:10D840001186502383F31288836B1A68D20720D481
:10D850005D686DB9446A826A944217D08169114447
:10D86000D9600ED9A21A5A608462002280F85C2026
:10D870001A6842F00102F1B21A6081F3118870BC9B
:10D88000704701698A1A5A608562EEE7012380F8C1
:10D890005C30F3B283F3118870BC70472DE9F04F10
:10D8A000BC4B1E788BB0002E40F08180BA4BBB4C35
:10D8B0001D78BB4FDFF80CB305F00105A4F10A0990
:10D8C00054F80A0CB8B14FF0CC0808FB069806F0E3
:10D8D00079FC80B154F80A0C06F06EFC14F8023C96
:10D8E000024683B924283BD075B354F80A0C06F0DD
:10D8F00069FC0028EED10136032E04F1CC04DFD1FF
:10D900000BB0BDE8F08F012B2ED0022B33D0032BB0
:10D9100040D0042B00F06981052B00F05781062BC5
:10D92000E3D114F801ECBEF1000F00F0D881BEF194
:10D93000010F00F01B8201360023032E04F8023C85
:10D9400004F1CC04BCD1DBE7232A54F80A0C00F024
:10D950008281944B93F83A309342B8D1FBF738FC6C
:10D96000012304F8023CC0E74D2800F06781002342
:10D9700004F8023CB9E700233C2804F8023C00F01C
:10D9800057813E28B1D10122032304F8012C04F869
:10D99000023CAAE7C028EAD80021042304F8050CB9
:10D9A00004F8040C04F8061C04F8023C9DE77E4BC6
:10D9B00018680028A4D007F094FADFF80CA27B4D79
:10D9C000DFF8F891DAF8000006F0FCFB002897D0A9
:10D9D000DAF8000006F0F0FB09281BD03F2819D028
:10D9E0002B68002B67D1042800F0BA810C2800F0C6
:10D9F000CA807F28E6D0A0F12002D2B25E2AE1D808
:10DA00000BB92028DED05A1C09F803002A6017F051
:10DA1000A9F8D7E72C68002C5AD1654FA34607F523
:10DA20002078BBF1000F08BFBB4610374745F8D13F
:10DA3000BBF1000F00F04E81103FDBF800003A68A8
:10DA4000065D135D9E42204402EB040140F04081DC
:10DA5000661E4E4422460BB9FD2A5CD906F8013FEA
:10DA600001322A6010F8013F11F801EF9E45F2D013
:10DA70000AB15F4512D04F4817F07CF85F4508D3D4
:10DA80005BF8100B17F076F8092017F06BF8BB4520
:10DA9000F6D9494817F06EF82A680024944291D2CA
:10DAA000661E4E4416F8010F17F05CF82B6801341F
:10DAB0009C42F7D386E70C2865D00A2834D00D287D
:10DAC00032D07F2800F0BE80FF2B3FF67BAF92E77D
:10DAD000374E002706F52078BB4602E01036464553
:10DAE0000DD022463168484607F056FD0028F5D192
:10DAF000B346002FF2D1374610364645F1D13B46AA
:10DB00005F469B46002B98D1002F3FF45BAF29481E
:10DB100017F030F8B4E7511C202009F80200296002
:10DB200009F801300A46A4E717F0A5F82321234895
:10DB300034F0FAFB002800F01181A0EB0900286006
:10DB400090B1431E19F80310202940F02C8109EBF5
:10DB5000030243B112F8011D202903F1FF304FD118
:10DB60000346002BF6D12B604FF48072002148460B
:10DB700034F0C3FB074B1B78002B3FF4C1AE0E48BB
:10DB800016F0F8FF1EE70E4816F0F4FF0A4816F0EC
:10DB9000F1FF17E70D9C00200062002052AE00202C
:10DBA000981F00207C760020C8460020A843002053
:10DBB0001C420408E85A0408F05A0408A84200204D
:10DBC000F85A040824240408A442002014F8063C4F
:10DBD00014F8051C99426FD814F8043C83427FF472
:10DBE000C6AE062304F8023C9BE614F8043C04F895
:10DBF000030C5A40052304F8042C04F8023C74E694
:10DC00002B606A4C002204F5207809F8032002E01A
:10DC1000103444454CD0216848461AF01FF90028BA
:10DC2000F6D0444544D2E368984700232B609BE735
:10DC3000032204F8013C04F8022C56E6022304F8FF
:10DC4000023C52E6013B002259482B6009F80320B0
:10DC500016F090FFB6E6574B5749DB78574ADFF886
:10DC600088E11060003318BF01230B70544B554AF4
:10DC7000CEF80030544B3A614FF0400E012187F846
:10DC800018E0F86078617D765048197017F03AFC1A
:10DC90004F4816F06FFF4FF4006010F00FFB4D4B34
:10DCA00093F83A30232B3FF459AE14F8023C36E691
:10DCB000494816F05FFFB8E714F8041C08EB0300AE
:10DCC0005140013304F8041C04F8063C82720CE64F
:10DCD0002246CDE64148103F16F04CFFD0E69BE8C7
:10DCE0000F000DF1280C0DF1080888E80F004CF822
:10DCF00024ED14F8053C14F803AC06946246234462
:10DD00004FF0010C414606A8ADF822E00793ADF8AC
:10DD100020A08DF824C008F09BFA40B1029A304B45
:10DD200003924146A4F10A00029313F0AFF8DDF824
:10DD30000480002304F8023CB8F1000F3FF4DBAD8F
:10DD400054F80A0C13F064F9013654F80A0CC04771
:10DD5000032E04F1CC047FF4B3ADD1E52868EFE6DF
:10DD6000204819F0FFF80BB0BDE8F08F14F8053C1F
:10DD700014F8032C0694234407936E2A4FF00003F3
:10DD800008930993ADF820207FF4D5AD06A807F0DD
:10DD900082FC06A807F074FC06A807F071FC06A830
:10DDA00007F06EFCC7E503462BE700BF1C420408E2
:10DDB000205B0408289C0020D0280020A4420020DA
:10DDC000A81F00206D3901080D9C0020245B040869
:10DDD000F05A04087C760020045B0408E85A040822
:10DDE00080BA0020A8420020C84600202DE9F04F4C
:10DDF0002DED028B95B0064620F0B2FA9E4B1D78B1
:10DE000025B115B0BDEC028BBDE8F08F9B4B1B68B4
:10DE10005805F6D5DFF8B092D9F80020002A00F0B6
:10DE20002781974CD4F8283103F5F43348339E42C8
:10DE3000C0F01E81934F94F82C113B68C4F8286100
:10DE4000013184F82C11990701F1798713F0140F2F
:10DE500041F0178713F0080F94F82C3140F0C2817D
:10DE600013F0070801F0BA85282B874B029302F0C4
:10DE7000B1805E209047854B1B78002B6BD0804C87
:10DE8000834AD4F83431F31A934201F24384DFF821
:10DE90003CA29AF80080B8F1000F33D1DFF800926D
:10DEA000D9F8000006F08EF9C0B201280ED9022878
:10DEB000784F42F04F813B78002B42F02A82D4F811
:10DEC0003C31F31AB3F57A6F82F0D5827248076855
:10DED000002F40D09AF80030BBB9704BD9F8000041
:10DEE0001B689B781E3B012B4FF0020142F26882B7
:10DEF000043020F0EDF8012200238AF8002084F895
:10DF0000483126E0644807682FB3D4F8443140F61E
:10DF1000B732F31A93421ED994F84031002B02F025
:10DF20000F81013BDBB284F84031002B01F0978771
:10DF300017F8011B94F84821076094F849315848B4
:10DF40000A440133006884F8482184F8493106F016
:10DF50003CF9C4F84461534A029B12781B68012AB9
:10DF600003F101030C9301F0FF824F4B1B787BB14F
:10DF7000DFF85C91D9F8003053B1414C029BD4F8E2
:10DF80005C21D3F800B0ABEB0202632A01F21A82E3
:10DF9000DFF8408198F800A0BAF1020F01F03A874B
:10DFA0003C4F97F87430032B01F0DC843F4B1B7817
:10DFB00073B13F4D2B685BB1314CFFF775F9D4F865
:10DFC0006831039044F61F62C31A934200F26081E5
:10DFD000384B1B78002B7FD1374B1B7843B1284C33
:10DFE000D4F8B83203F50043E8339E4281F032831F
:10DFF000324B1B78002B3FF404AF214E304C314D97
:10E0000006F2C127206806F0DDF800283FF4F9AEDB
:10E01000206806F0D1F82B7880465A1E33B120686C
:10E020002A7006F0CFF80028F2D1EAE6032239463A
:10E03000781E34F048F996F8C03296F8C12286F876
:10E04000C38283F47F4383F0FF039B1A1FFA88F88F
:10E050009BB2B8EB132FD5D196F8C222DBB29A420D
:10E06000D0D1781E2EF050FD2B7818442870C9E7C7
:10E07000054B0293FFE600BF0D9C0020C08D0020E1
:10E08000F41F0020C85100203C850020DA520020F7
:10E090003F0D03001C000020405200203C52002095
:10E0A00038520020DB520020E8520020F0520020BD
:10E0B000F45200206053002071530020FA520020D7
:10E0C00000530020045300204852002044520020F6
:10E0D000EC9B0020BA3E0020604C2278002A41F0E0
:10E0E0003A82DFF8A49199F80040002C40F0AB8010
:10E0F0005B4D2878002842F08C805A4C5A4DD4F859
:10E10000B0222978594B93FBF1F313449E42FFF45C
:10E1100063AF94F8B432564AC4F8B062D75CFB07D8
:10E1200002F17482B80702F1E981790702F12A82CB
:10E130003A074CD54F4BDFF854810D930DF1500940
:10E14000A3F13D0249F8202D0021A3F1400203F87C
:10E15000401C02231121517093704846D8F80010DA
:10E1600007F0A8FA4846D8F8041007F0A3FAB8F860
:10E170000E30414903EBC3039B00053381FB0321B0
:10E18000DB17C3EBA10189B2484607F0AAFAB8F839
:10E19000103003EB8303590089B2484607F0A1FA17
:10E1A000364B1B789B0743BFB8F8081001F57A710E
:10E1B00089B24FF47A71484607F093FA0C9B98F8AD
:10E1C0001420591C0C9148461A7020F06FF894F8EE
:10E1D000B4322978013393FBF1F201FB123384F856
:10E1E000B432F9E613F0030A7FF43AAE5E209047AA
:10E1F000D9F8003014209847214B1F4AB3F9043056
:10E2000082FB03124FEAE378C8EBA2080FFA88F802
:10E210005FFA88F01FF0B0FFC8F307201FF0ACFFD3
:10E22000D9F800305E209847D9F800301C20984774
:10E2300050461FF0A1FF50461FF09EFF94F82C316E
:10E24000D9F800200CE60F4D2F6E002F41F09D866F
:10E25000044B89F80070C3F8B062BDE6CC520020D0
:10E2600068530020F41F002070530020A086010096
:10E270006C5300208C520020676666662452002092
:10E28000D45100207853002069530020A4A5002019
:10E2900094F86E31002B41F0EA85DF4B1B6803F0E8
:10E2A0000802002A48F603414AF60B404BF60F429B
:10E2B00049F6074704BF02460F4613F0040F4FF01C
:10E2C000190118BF17469B0684F86E1103D547F451
:10E2D000804747F0200712F0BDFBC7F3090900286B
:10E2E00042F0D282CD4B9B79002B42F09F82984620
:10E2F00064204FF0FF3A4FF0000C0C970D97ADF8EB
:10E300003CC0CDF842C0CDF846C0CDF84AC0CDF8EB
:10E310003890ADF83E80ADF840A08DF84E000CAFBF
:10E320000FCFDFF808E384F805C0AEE80F0097E8E8
:10E330000F00AEE807002EF8023B71464FF0010CCB
:10E340001B0CFE271F20C82201F81E39A770A271DE
:10E3500084F807C0E07094F87E01207180F0F1032A
:10E3600083EA0313DAB2130983F0E70343EA0223D3
:10E3700083EAC2031BB283EA0312D2B2C3F30723B8
:10E3800083EA121343EA022383EAC2031BB283F037
:10E39000C80282EA0212D2B2C3F3072383EA12133D
:10E3A00043EA022383EAC2031BB283EA0C0787EA2B
:10E3B0000717FFB2C3F3072282EA171242EA0722C5
:10E3C00000EB0C0382EAC7070EEB0C0084F87E31E9
:10E3D000278011F8013B7B4083EA0313DBB21A0963
:10E3E00082EA172242EA032282EAC3031BB29FB2E7
:10E3F00081422780EDD183F07C0383EA0313DBB2F3
:10E400004FEA131E8EEA172E8EEA032E8EEAC30EF3
:10E410000FFA8EFE1FFA8EF9DFF814C2A4F80090EE
:10E420005FFA8EFE4FEA192984F8289084F827E0D5
:10E430000CF5D37804F1220ADCF80000DCF80410B3
:10E44000DCF80820DCF80C3047460FC70CF1100C44
:10E45000D445B846F0D1DCF800003860704F9CF825
:10E46000043088F8043007F1270884F8CDE184F8F7
:10E47000CE9117F8011F286805F0A7FEB845F8D11E
:10E4800094F86F21002A41F05E856649029B087866
:10E490001B680A2184F86F11002801F09A86DFF8C2
:10E4A00094E10128BEF80010059142F2EE820228A4
:10E4B000BEF8028002F00082BEF804100491032826
:10E4C00002F0DD820428BEF806A002F0D3820528FF
:10E4D000BEF8087002F0C7820628BEF80AC002F033
:10E4E000BF820728BEF80C1001D0BEF80E2094F8A9
:10E4F0007EB10C938BF0300383EA0313DBB24FEA57
:10E50000131E494884F804B08EF07A0E4EEA032EAA
:10E5100000888EEAC303DFF820E1C0EB00208EFB09
:10E52000009E8644C0171BB2C0EB6E200690C3F35A
:10E53000072E83EA0310059BC0B24FF0000963F376
:10E540000F098EEA101305934FF0000E049B68F339
:10E550001F4967F30F0E4FF00008002763F30F0801
:10E5600061F30F07059BCDF834906CF31F4E62F3F7
:10E570001F474FF0000C9DF81820CDF83CE06AF3DF
:10E580001F48CDF8388010978DF844C08DF845208D
:10E5900043EA00230DF1300883EAC007B8E80F0012
:10E5A0003FB287F0C80989EA0919DFF880E084F8EA
:10E5B00005C05FFA89F9C7F30727AEE80F0087EABD
:10E5C000191747EA092398E8030083EAC9031BB235
:10E5D00083F023074EF8040B87EA0717FFB2C3F353
:10E5E000072282EA1712704642EA072282EAC70728
:10E5F00020F814190BF1010B4FF0230CFE21162209
:10E60000C82384F87EB1278084F807C00EF1020E7B
:10E61000A170E270A37111E0C8510020B851002030
:10E620009B210020709C0020B0510020FC1F002086
:10E63000F61F002050B100200308208010F8013B95
:10E640007B4083EA0313DBB21A0982EA172242EA0B
:10E65000032282EAC3031BB29FB270452780EDD12B
:10E6600083F0F40383EA0313DBB24FEA131E8EEA4E
:10E67000172E8EEA032E8EEAC30E0FFA8EFE1FFAB5
:10E680008EFCD64FA4F800C04FEA1C295FFA8EFE1C
:10E6900084F81EE084F81F907968BA683868FB68CF
:10E6A00007F5D37CACE80F0038697969BA6904F2E0
:10E6B000C518ACE8070004F2A71784F8C59184F8E0
:10E6C000C4E117F8011F286805F07FFDB845F8D1AF
:10E6D00094F87231002B41F04684C14F3B681922F7
:10E6E000980684F8722140F10E83BE4BDFF8008358
:10E6F0001B78990741F1868798F81430042B8CBF5A
:10E700004FF003094FF00209FEF7CEFDB8F81030C4
:10E71000B8F808200C9003EB83035B00ADF84A3097
:10E720004FF47A70D8F800308DF84C900E93B8F80A
:10E730000E1098F814E0D8F804308DF84DE000FB86
:10E7400002F24FF0000A4FF0FF300DF13009CDF822
:10E7500034A010920F93ADF848101190CC46BCE84D
:10E760000F00DFF890E2AEE80F009CE80F00AEE883
:10E7700007007246182122F81C39E17194F87E11C5
:10E7800084F805A081F0780383EA0313D8B2030963
:10E7900083F0F60343EA002383EAC0031BB283EA53
:10E7A0000310C0B2C3F3072383EA101343EA002324
:10E7B00083EAC0031BB283F0C80080EA001C5FFA42
:10E7C0008CFCC3F3072080EA1C1040EA0C2080EA8E
:10E7D000CC0000B280F0180383EA0313DBB2C0F36D
:10E7E000072080EA131040EA032080EAC30301F106
:10E7F000010CFE204FF01E0A4FF0C80BA0700EF166
:10E80000020E217184F87EC1238084F803A084F86D
:10E8100006B0184612F8011B414081EA0111C9B245
:10E820000B0983EA102343EA012383EAC10109B2F9
:10E8300088B272452080EDD181F0180181EA011182
:10E84000C9B20A0982EA102383EA012383EAC103D9
:10E850001BB29AB261492280DBB2120A049106927D
:10E86000059384F8272084F826308E4601F5D37B63
:10E8700004F1220ADEF80000DEF80410DEF80820B9
:10E88000DEF80C30DC46ACE80F000EF1100ED64579
:10E89000E346EFD1DEF80000CCF800009DF814301C
:10E8A000DFF854A184F8CC319DF8183084F8CD31CC
:10E8B000D3461BF8011F286805F087FC4A4B5B45CF
:10E8C000F7D1FEF7F1FCD8F800103B68B8F8082043
:10E8D0000591D8F80410069113F0140F4FF47A71D3
:10E8E00001FB02F141F074850F4694F87EB10C9063
:10E8F0008BF06A003D4BDFF804E1B3F90420109778
:10E9000080EA0010C0B2030983F0D50343EA002374
:10E9100083EAC0031BB283EA0310C0B2C3F3072328
:10E9200083EA101343EA002383EAC0031BB28EFB81
:10E93000020E05980D90D2174FF00008C2EBAE0200
:10E9400006980E9083F0C80C0F91ADF84A20ADF8F0
:10E950004480ADF84680ADF848808CEA0C1CCE4669
:10E960005FFA8CFCC3F30727BEE80F0087EA1C1789
:10E9700047EA0C2787EACC07DFF878C084F804B0B0
:10E980003FB2ACE80F0087F021039EE8070083EA5E
:10E990000313DBB2C7F3072787EA13170BF1010E46
:10E9A00047EA03278CE8070087EAC30384F87EE17F
:10E9B0004FF0210B4FF0FE0E1C27C8220CF10C0C5F
:10E9C00084F8058084F807B084F802E0ACF11C01FB
:10E9D000E7701846A271238012E000BFF61F0020E6
:10E9E000C851002024520020C1210020D451002011
:10E9F000A4A50020FC1F00209B21002067666666FE
:10EA000011F8012B424082EA0212D2B2130983EAC2
:10EA1000102343EA022383EAC20212B290B2614594
:10EA20002080EDD182F0680282EA0212D2B24FEA6F
:10EA3000121B8BEA102383EA022B8BEAC20B0FFA1C
:10EA40008BFB1FFA8BF3DB4F23805FFA8BFB1B0AD8
:10EA5000059384F8253084F824B007F5D37C04F1BD
:10EA6000220838687968BA68FB68E646AEE80F00A5
:10EA700010374745F446F4D13B88AEF800309DF896
:10EA80001430CD4F84F8CAB1D04684F8CB3118F891
:10EA9000011F286805F099FB4745F8D194F87EC11D
:10EAA000C64A84F804C08CF0EB0383EA0313D9B29E
:10EAB0000B0983F0C50343EA012383EAC1031BB2B8
:10EAC00083EA0310C0B2C3F3072181EA101141EABF
:10EAD000002181EAC00109B20CCA81F0C80787EAA7
:10EAE0000717FFB24FF0000EC1F307210D93CDF8C9
:10EAF00038E081EA17130C9299E8070043EA0723EC
:10EB000083EAC7030FFA83F8AD4B84F805E088F079
:10EB1000310783E8070087EA0717FFB2C8F3072326
:10EB200083EA171343EA072383EAC703277A607A45
:10EB3000A27AE17A94F80CE094F811801BB25F405D
:10EB400087EA0717FFB2C3F3072383EA171343EAE1
:10EB5000072383EAC7031BB2584080EA0010C0B203
:10EB6000C3F3072383EA101343EA002383EAC003B5
:10EB70001BB25A4082EA0210C0B2C3F3072282EAF3
:10EB8000101242EA002282EAC00212B2514081EA27
:10EB90000111C9B2C2F3072383EA111343EA012327
:10EBA00083EAC1031BB28EEA030E8EEA0E1E5FFAE1
:10EBB0008EFEC3F3072383EA1E1343EA0E23677B0B
:10EBC000A07BE17B227C83EACE031BB25F4087EA15
:10EBD0000717FFB2C3F3072383EA171343EA072398
:10EBE00083EAC7031BB2584080EA0010C0B2C3F3E7
:10EBF000072383EA101343EA002383EAC0031BB20E
:10EC0000594081EA0111C9B2C3F3072383EA111302
:10EC100043EA012383EAC1031BB25A4082EA02128B
:10EC2000D2B2C3F3072383EA121343EA022383EA2F
:10EC3000C2031BB288EA030888EA08185FFA88F85A
:10EC4000C3F3072383EA181343EA082383EAC803BC
:10EC5000A17CE27CDFF874811BB2594081EA01118A
:10EC6000C9B2C3F3072383EA111343EA012383EAFA
:10EC7000C1031BB25A4082EA0212D2B2C3F3072385
:10EC800083EA121343EA022383EAC2031BB283F02E
:10EC9000270787EA0712D2B2C3F3072787EA1217BA
:10ECA00047EA022787EAC2073FB20CF10103BAB272
:10ECB0005FFA87F94FF0310CFE200C2184F87E3189
:10ECC000C8234FEA122E228084F807C0A070E1709A
:10ECD000A37184F81490049F84F815E07968BA68E9
:10ECE000FB683868B7F810C0A8E80F0028F803CB15
:10ECF00084F8BBE184F8BA911AF8011F286805F07E
:10ED000064FAD045F8D194F87671002F41F026814D
:10ED10002C4B94F87E81B3F90010B3F90220B3F9BB
:10ED200004309FED296A677107EE103A029B1B6859
:10ED30000C9388F06A0383EA031306EE901AD9B2A3
:10ED40000B0983F0D50343EA012383EAC1031BB215
:10ED500083EA03115242C9B207EE902AC3F3072394
:10ED600083EA111343EA0123F8EEE77AF8EEE66A44
:10ED7000B8EEC77A83EAC1031BB267EE867A66EE05
:10ED8000866A27EE067A002083F0C80ECDED0E7A53
:10ED9000CDED0D6A8DED0F7A1090119012908EEAE4
:10EDA0000E1C0DF130095FFA8CFCC3F3072EB9E895
:10EDB0000F000DE0F61F0020BF2100205049002069
:10EDC000FC1F0020D451002088C3E43A9C2100207D
:10EDD0008EEA1C1E4EEA0C2E8EEACC0EDFF888C49A
:10EDE0000FFA8EFEACE80F008EF01E0799E80700C0
:10EDF00087EA071A5FFA8AFACEF3072787EA1A1713
:10EE000047EA0A278CE8070087EACA071C214FF067
:10EE1000050A4FF01E094FF0FE0EC82208F101034B
:10EE2000E17084F876A184F8079084F802E0ACF1F0
:10EE30001001A2710CF10C0C84F80480278084F876
:10EE40007E3111F8013B7B4083EA0313DBB21A09E0
:10EE500082EA172242EA032282EAC3031BB29FB26C
:10EE600061452780EDD183F0270383EA0313DBB2EA
:10EE70001A0982EA172282EA032282EAC3031BB23A
:10EE80001FFA83FCDFF8E483A4F800C05FFA83FE76
:10EE90004FEA1C2C84F825C084F824E008F5D379C7
:10EEA00004F1220AD8F80000D8F80410D8F8082095
:10EEB000D8F80C304F460FC708F11008D045B946B6
:10EEC000F0D1E04FB8F80030A9F8003007F124087D
:10EED00084F8CAE184F8CBC117F8011F286805F04F
:10EEE00074F9B845F8D194F877A1BAF1000F41F060
:10EEF0002F80D54B1B68052284F877219A0641F1B3
:10EF00007281D24ADFEDD27AD18907EE101AB8EEBB
:10EF1000C77A13F0140F27EE277A01F0F984CD4B4E
:10EF2000DFEDCB6AD3ED007AF8EEE77A67EEA67AEA
:10EF300094F87EC1C84BC94AB3F90410B2F906204F
:10EF4000C74FC8488DED0D7A8CF0220383EA031376
:10EF50005FFA83FE4FEA1E1383F0590343EA0E2340
:10EF6000B2F5FA6F83EACE031BB2A8BF4FF4FA6280
:10EF700083EA0318B2F57A7F5FFA88F8C3F3072EA5
:10EF8000B8BF4FF47A72A2F57A728EEA181E642323
:10EF900003FB02F34EEA082E87FB03278EEAC80E16
:10EFA000DA17C2EBA71280FB01300FFA8EF7CB17EE
:10EFB0004FF0000BC3EBA00387F0C8080DF1300938
:10EFC000CDED0E7AADF84220ADF84030CDF830B03E
:10EFD000CDF83CB0CE4688EA0818BEE80F005FFACC
:10EFE00088F8C7F3072787EA181747EA082787EA48
:10EFF000C8089D4FDEF800E084F804C00FC70FFA80
:10F0000088F888F04A0383EA0310C0B2C8F30723E4
:10F0100083EA10133A460CF1010143EA002383EA24
:10F02000C00342F810E900204FF04A084FF0FE0CF0
:10F030004FF0140E84F87E11C821607123800437CC
:10F0400084F8078084F802C084F803E0A1711846B0
:10F0500012F8011B414081EA0111C9B20B0983EA90
:10F06000102343EA012383EAC10109B288B2BA42FC
:10F070002080EDD181F0140181EA0111C9B24FEA7B
:10F08000111E8EEA102E8EEA012E8EEAC10E774BEB
:10F090000FFA8EFE1FFA8EFC1F464FEA1C2B5FFAFA
:10F0A0008EFE84F81DB084F81CE0596838689A68B0
:10F0B000DB68A4F800C007F5D37CACE80F00386922
:10F0C0007969B7F818800497ACE8030004F2A71731
:10F0D000ACF8008084F8C3B1B84684F8C2E104F209
:10F0E000C31B18F8011F286805F06FF8C345F8D155
:10F0F0005F4B604A1B781278013B12F00100DBB2D3
:10F1000014BFC0214021172B03D85B4A134493F846
:10F1100014A05A4B1A8893071ABF002341F010011C
:10F12000012312F4027F18BF022312F0100F18BF40
:10F13000062312F0200F18BF1023002841F0918100
:10F140004FF0030894F87EC10C938CF0460383EAD9
:10F150000313DAB2130983F0920343EA022383EA2A
:10F16000C2031BB283EA0310C0B2C3F3072282EAD0
:10F17000101242EA002282EAC00212B282F0C80EE5
:10F180008EEA0E1E00235FFA8EFE0320C2F30722D2
:10F190008DF834A08DF8378082EA1E128DF8353054
:10F1A0008DF836108DF8380042EA0E2899E80700ED
:10F1B00088EACE0E0FFA8EF8DFF8ACA0E37188EA89
:10F1C0000819AAE803005FFA89F9C8F3072888EA52
:10F1D000191848EA092181EAC90994F808808AF8CF
:10F1E00000200FFA89F988EA090282EA02185FFA18
:10F1F00088F8C9F3072282EA181242EA0822607AE4
:10F20000A17A94F80B90637182EAC80212B250405E
:10F2100080EA0010C0B2C2F3072282EA101242EA6A
:10F22000002282EAC00212B2514081EA0111C9B241
:10F23000C2F3072282EA111242EA012282EAC102E3
:10F240001EE000BF9B210020C8510020A4A5002083
:10F250000AD7233CCC510020D451002050B10020CB
:10F26000D34D621067666666FC1F0020F61F002003
:10F270006C6E00200062002034240408B25100208B
:10F2800012B289EA020989EA09195FFA89F9C2F317
:10F29000072282EA191242EA092294F80C80607B64
:10F2A000A17B84F804C082EAC90212B288EA02088B
:10F2B00088EA08185FFA88F8C2F3072282EA18126F
:10F2C00042EA082282EAC80212B2504080EA0010E4
:10F2D000C0B2C2F3072282EA101242EA002282EA96
:10F2E000C00212B2514081EA0111C9B2C2F3072231
:10F2F00082EA111242EA012282EAC102E17B94F819
:10F30000109013B281EA030282EA0212D2B2C3F36E
:10F31000072383EA121343EA022383EAC2031BB2E0
:10F3200089EA030282EA0212D2B2C3F3072383EA14
:10F33000121343EA022383EAC2031BB283F03202B0
:10F3400082EA0212D2B2C3F3072383EA121343EA1A
:10F35000022383EAC2031BB29AB24FF0FE085FFA9F
:10F3600083FE0920C8210CF1010C84F802804FEAC9
:10F370001228E070A17184F87EC1228084F8128086
:10F3800084F811E0049B186859689A68B3F80CB0C7
:10F390000AF5CC7CACE807000AF5D47A8CF8029028
:10F3A000ACF800B084F8B88184F8B7E117F8011F11
:10F3B000286804F00AFFBA45F8D1039BC4F8683105
:10F3C000FEF706BEDFF83C83BF4FDFF83CA34120C9
:10F3D0002DF01AFEB8F9022087FB0230D217C2EBDB
:10F3E000A00080B22DF0F4FDB8F9002087FB0230B8
:10F3F000D217C2EBA00080B22DF0EAFDB8F90420CC
:10F4000087FB0230D217C2EBA00080B22DF0E0FDE6
:10F410009AF80010D9F8000004F0D7FE94F8608143
:10F4200018F0010700F02885A84F3A68910640F1CE
:10F430008180A74ADFF8D4821278920740F1C4870E
:10F4400098F81420042A8CBF032302230393472037
:10F450002DF0DAFDD8F800002DF086FDD8F8040074
:10F460002DF082FDB8F80E209A49D9F80000A1FBD2
:10F470000232C2F347121146049204F0A6FE9AF833
:10F4800000003968049A11F0140F82EA00028AF829
:10F49000002040F0BA86B8F80820642000FB02F093
:10F4A0002DF062FD98F81470039BD9F8000043EA30
:10F4B0008707FFB2394604F088FE9AF80020D9F891
:10F4C0000000574039468AF8007004F07EFE94F838
:10F4D0006081B8F1000F2DD17F4F4F202DF094FDAA
:10F4E00038682DF041FD78682DF03EFD40462DF046
:10F4F0003BFD0121D9F8000004F067FE744A9AF838
:10F5000000701278D9F8000002F00108414687F037
:10F5100001078AF8007004F058FE9AF80020D9F824
:10F52000000088EA020211468AF8002004F04DFE2D
:10F5300094F86081694AC4F85CB108F10103DBB258
:10F54000A2FB0312D20802EB8202A3EB420384F86F
:10F550006031FEF71DBD624B6249186804F003FE7E
:10F5600000232370FEF7BDBD5F4F386800283EF4CE
:10F57000FCAC4FF0000ADFF898815C4CAB46554676
:10F5800004F020FEF8B1F5B94FF00109AA46386839
:10F5900004F012FE83B27E2B00F0518498F8012013
:10F5A000002A49D194F84C11B1B11B2B84F84C219D
:10F5B00000F01E840D2B45D0386888F8019004F0C7
:10F5C00001FE0028E3D1AA4650460CAA48495D46F0
:10F5D0001EF03AFAFEF7C9BC7D2B00F0F08594F8D6
:10F5E000502122B180F02003DBB284F8501194F84E
:10F5F0004B21062A10D8B4F84E1138681944A4F8E3
:10F600004E11A118013281F8543184F84B2104F0D5
:10F61000D9FD0028BBD1D6E7B4F84E2188F8019077
:10F6200013449BB21A0A52FA83F3FF2BA4F84E310B
:10F63000386802D12F4DA3E7386804F0C3FD0028D5
:10F64000A5D1C0E73868A4F84E2104F0BBFD00281E
:10F650009DD1B8E794F8BC32C4F8B862012B40F2EF
:10F66000738594F8BD222449981801EB800101327A
:10F6700002F00102CF6A84F8BD22BFB11F4D0D9583
:10F680000DF15009123DA52349F8205D802284F830
:10F69000103115233146484684F8112184F812317F
:10F6A000B847002840F0D18494F8BC32144A0133A2
:10F6B00082FB0312A2EBE37202EB42029B1A84F874
:10F6C000BC32FEF795BC00BF67666666C851002075
:10F6D000245200201F85EB5150490020CDCCCCCCCA
:10F6E000645300208C52002034520020F41F00206C
:10F6F0003E21002048210020342404081921002044
:10F7000056555555D4510020F09B0020A4A500204B
:10F710001C0000209E4A9F4B92F80BE0029AD4F8FE
:10F72000381110681B889C4A401A4FF47A71DFB276
:10F7300001FB0EF11B0A9777177588424FF00007FF
:10F74000D37753759770177180F0EA84934BDFF885
:10F7500070C21B689249934F0868DFF86892896805
:10F760003F688CFB038EDB17C3EB6E1303F5FA7354
:10F770009BB293761B0AD37689FB00A389FB01A970
:10F78000C017C917C0EBA300C1EBA90107F5EA43F5
:10F79000DFF834E210773033001282F820100912BB
:10F7A0001B12DFF828829EF800E0507782F82110C3
:10F7B0008CFB0790F917C1EB601182F823307A4B6C
:10F7C00098F814A083F81AA0783130371EF0020F91
:10F7D00082F8241082F8227000F09F84D8F800E0AC
:10F7E000724AD8F80400DFF8E8B182FB0E714FEAE4
:10F7F000EE77C7EBA151039182FB0092C117C1EBD9
:10F80000A25203990BFB01E101EB410149000F46B4
:10F810000BFB020B0497B9460BEB4B0B644F4FEA03
:10F820004B01059187FB099B87FB01194FEAA94909
:10F83000CDF81C90B8F80E900399B8F8088002EB48
:10F84000820209EBC90902EB8202089201EB8107EF
:10F850004FEA89020599039207EB8707049A0697F6
:10F86000CF17C10F0991049852494FEAAB4BD217F9
:10F870004FEADE7E83F809E0ABEB020E01FB1E02CD
:10F880000798069908F5FA78BAF1050F1FFA88FA71
:10F89000A0EB0708059F474883F815A04FFA8EF99B
:10F8A00009EB8109414600FB18789DF82400987304
:10F8B0000898414FDFF81CE149B201EB80018CFB55
:10F8C000020B4FEAE2720492039ABEF800E08CFB4E
:10F8D00008C087FB02C74FEAE27C049AC2EB6B12B6
:10F8E0000392364A1FFA89F91288ADF8102083F87E
:10F8F0000A90039A83F813E089B24FEAE8784FEA56
:10F90000112BC8EB6010CCEBA7174FEA1A284FEA6F
:10F91000192C4FEA222A9DF80C2083F810B04FEAE8
:10F92000202983F80BC0D973C7F3072C4FEA1E2197
:10F9300034BF4FF0320B4FF0330B1A739DF8102089
:10F9400083F80DA0587483F8129083F81680DF7145
:10F9500083F808C0197583F81BB01A77C4F83461AE
:10F96000FEF795BADFF87090D9F8000004F01EFC9D
:10F9700000283EF41BABD9F80000012104F013FC71
:10F980000222002387F8742088F80030FEF70EBBAF
:10F99000209A0020189A002008530020CC51002003
:10F9A000F04F0020D0510020345300206BCA5F6B11
:10F9B00083DE1B4340420F00D34D6210A04900205C
:10F9C0001F85EB516766666624520020A4A50020BF
:10F9D000806967FF30520020CC3F00205E209047B6
:10F9E000D9F8003002209847FF202DF013F8037853
:10F9F000FF2B00F0998490F901304FEAE3785FFA29
:10FA000088F8D8B21EF0B8FB40461EF0B5FBD9F816
:10FA100000305E209847D9F8003003209847FF2037
:10FA20002CF0F8FF0378FF2B00F07984B0F9083050
:10FA3000D8B2C3F307281EF09FFB40461EF09CFB84
:10FA4000DA4B1B78042B7DD0DFF88CB3B4F82E1181
:10FA50009BF80020DFF884A391FBF2F302FB131361
:10FA60009BB2BAF80010A4F82E314FEA03181FFA1F
:10FA700088F8642303FB01235200B3FBF2F348EA46
:10FA80000328C3F303225E20D9F800301FFA88F858
:10FA900048EA02089847D9F80030062098475FFAEC
:10FAA00088F01EF069FB4FEA18201EF065FBC04984
:10FAB000B4F82E214B7ABAF800A00132012BA4F839
:10FAC0002E2100F00C874A7B0AEB8A031FFA83FA87
:10FAD000002A40F0C084D9F800305E209847D9F859
:10FAE00000303A209847B34BA3FB0A384FEA581826
:10FAF0001FFA88FB5FFA8BF01EF03EFB4FEA1B20DB
:10FB00001EF03AFBD9F800305E209847D9F8003053
:10FB10003B209847642303FB18A39BB2A6480533F8
:10FB200080FB0320DB17C3EBA000C0B21EF024FB58
:10FB300000201EF021FBDFF8A88298F80630002B89
:10FB400040F051843B689F0640F11282DFF894A296
:10FB50009AF80030980700F1EA83DFF88C820027DA
:10FB6000BB46D9F800305E209847D9F80030012014
:10FB7000984758461EF000FB38461EF0FDFAD9F8AB
:10FB800000305E209847D9F80030092098470020BF
:10FB90001EF0F2FA00201EF0EFFAB8F8123098F8D2
:10FBA00014B0B3F5967F0AD994F82C2102F00F0215
:10FBB000072A04D842F20F7B9B4528BF9B46D9F801
:10FBC00000307B4F5E209847D9F8003005209847D9
:10FBD0003B7A002B00F06685ABF1200307EE903AEC
:10FBE0009FED767AF8EEE77AF6EE006A67EE877AAE
:10FBF000BEEE007AF5EEC07AF1EE10FA58BFB0EE24
:10FC0000667A77EE877AFDEEE77ACDED027ABDF976
:10FC100008B05FFA8BF01EF0AFFACBF307201EF0AE
:10FC2000ABFA9AF80020002392070A930B9300F195
:10FC3000658394F83031012B00F06083B7F9003010
:10FC4000DFED5F6A07EE103AB7F9023007EE903A3F
:10FC5000B8EEC77AF8EEE77A27EE267A67EEA67A4C
:10FC6000BDEEC77AFDEEE77A0CA88DED0C7ACDEDEE
:10FC70000D7A1EF0A3FA94F82C31D9F80020FEF783
:10FC8000F3B85E209047D9F80030302098474D4BAC
:10FC9000D3F800805FFA88F01EF06EFAC8F30720F0
:10FCA0001EF06AFA94F82C3113F003087EF4C8AA07
:10FCB000454AD4F82811454B9142186840F28F8389
:10FCC00080EAE073A3EBE0733A4A1BB282FB0312B3
:10FCD0004FEAE37ACAEB621A4FF0640808FB1A385D
:10FCE0000FFA88F80FFA8AFA5FFA88FB5FFA8AF24D
:10FCF000C8F30728CAF3072AD9F8003002925E2019
:10FD00009847D9F8003010209847029A10461EF004
:10FD100033FA50461EF030FAD9F800305E2098478A
:10FD2000D9F800302120984758461EF025FA404661
:10FD30001EF022FA3B68D9F80020FEF78BB8DFF8F6
:10FD4000AC809FED238A4FF0240A5E2090475046F6
:10FD5000D9F8003098471F4BF8EC016A9B8A07EEF0
:10FD6000103AF8EEE66AB8EEC77A0AF1010AC6EE72
:10FD7000877A5FFA8AFA67EE887AFDEEE77ACDED48
:10FD8000027ABDF908B05FFA8BF01EF0F5F9CBF3FB
:10FD900007201EF0F1F9BAF1270F02D0D9F80020A0
:10FDA000D3E73B68D9F80020FEF750B81D47002084
:10FDB000209A00201F85EB5167666666E4380E3F87
:10FDC0000050C347D05100203F4B4C00CC51002085
:10FDD00000007A44DC5100202E9A0020189A00205E
:10FDE000B851002024520020A4A500200C5200206D
:10FDF000386804F0E7F900287FF4DEAB386884F84F
:10FE00004A9188F8019004F0DDF900287FF4BFAB37
:10FE1000FFF7D9BBFDF748FAD14B1B68A0EB030BEA
:10FE200040F6B8339B4500F2BF81CE4B1A793A2A8F
:10FE300000F04284002388F80030FEF7B7B8386835
:10FE400084F84AA184F84BA184F84C9188F801A069
:10FE500004F0B8F900287FF49AABFFF7B4BB94F82C
:10FE6000481194F84931C0484A1CFEF76AB8013B72
:10FE700084F86E31FEF704BBBC4A1288D30513D454
:10FE8000D00600F1E682910600F11D85530600F1CF
:10FE90003C85100700F15485D10700F1588512F018
:10FEA000020F0CBF04270C27B149B24A0B78D27855
:10FEB00003F001030AB143F00203532003932DF032
:10FEC000A3F8AD4A128802EB820202EB8202900094
:10FED00080B22DF07DF800202DF07AF8A74AA849CD
:10FEE0001288D9F80000C2EBC212520081FB023125
:10FEF00011444FEAE278C8EB61285FFA88F841467E
:10FF000004F063F99AF80020039BD9F800001F431E
:10FF100088EA020800218AF8008004F056F9394680
:10FF2000D9F8000004F051F99AF80020D9F800003F
:10FF30007A40D2B211468AF8002004F046F994F8CB
:10FF40006081FFF7C6BA013A84F86F21FEF7C0BBA3
:10FF50000AF1FF3A84F877A1FFF72FBA013F84F83E
:10FF60007671FEF7C0BF013B84F87231FEF7CBBE5D
:10FF70001B077FF580AE834B93E803000CAB83E84F
:10FF8000030018461EF01AF975E60024DFF8108207
:10FF900027464FF0500A02E0DBB283F3118815F8D0
:10FFA00004B0601C594628442CF0DCFE002840F0C8
:10FFB00025810BF101031C44EFF311838AF31288AE
:10FFC0002A6E9442E8DB0022DBB22A6683F31188B2
:10FFD000FEF73EB94FF0000A5E201F6884F82CA19E
:10FFE0009047D9F80030DFF8BC8117209847504679
:10FFF0001EF0C2F8644BA3FB07239B0BA8FB031264
:020000040801F1
:100000005209C2EB0212A3EB8203D8B21EF0B4F87D
:10001000D9F800305E209847D9F80030182098476A
:100020005A4BA3FB07239B09A8FB03125209C2EBFF
:100030000212A3EB8203D8B21EF09EF850461EF0C7
:100040009BF8D9F80020FDF714BF0C9EAE424FF08C
:1000500000014FD941F2210015F8013B81EA032349
:100060005A0013F4004F80EA020192B289B208BF2D
:1000700011464A0080EA020311F4004F99B293B28C
:1000800018BF0B46590013F4004F80EA010289B2F1
:1000900092B208BF0A46530012F4004F80EA0301EF
:1000A0009BB289B208BF19464A0080EA020311F4E4
:1000B000004F99B293B218BF0B465A0013F4004F89
:1000C00080EA020192B289B208BF11464B0011F4D6
:1000D000004F80EA03029BB292B208BF1A46530057
:1000E00080EA030112F4004F9BB289B208BF19469F
:1000F000B542B1D1484605F018FB25490C9D25486D
:100100006D1A152DA8BF15252A4630F0F9FF224A91
:1001100094F8BC321570FFF7C9BA2D22DA761DE4C7
:100120001E4B02991B780968C4F83811013B012B5A
:100130003FF60CAB1021022391701371FFF706BB41
:100140001DF0FCFFFDF705BF0E4A02EB8302D76AE4
:10015000FFF793BA1DF0E2FF01233B70FDF7B6BE37
:10016000C03E0020A83E002038520020B25100209E
:100170000062002020470020189A0020B051002083
:10018000030820803424040873B2E745D34D62107D
:1001900004210020843C0020993C00201D470020C1
:1001A000E1E2020889888888C44AB2F862310021F5
:1001B0000133A2F8623188F80010FDF7F7BE386805
:1001C00084F8509103F0FEFF00287FF4E0A9FFF7C8
:1001D000FAB9014684460746824604908046059057
:1001E0000246FEF784B99FEDB67A13F0140F08BFEC
:1001F000F0EE477A7EF493AEFEF79ABE41463A207F
:100200002CF00CFD0743FFB2D3E6AE4A1068FFF7AF
:1002100047B9AD49AD4B0093A1F13F07AC4BAD4A97
:100220000B9101F8404C0CA8AB490A9705F054FB20
:100230000A9F7B1C0A933C700A9B2922591C0A9135
:100240001A700A9BEA22591C0A911A700A9BC8224A
:10025000591C0A910CA81A7030F014F800F101082A
:100260000CA942460A9830F04BFF0A9A02EB0803A9
:1002700001330A9302F808400A9B5A1C0A921C7028
:100280000A9B5A1C0A921C700A9B5A1C0A921C70E8
:100290000A9B5A1C0A921C700A9B5A1C0A921C70D8
:1002A0000A9B5A1C0A921C700A9B5A1C0A921C70C8
:1002B0000A9B5A1C0A921C700A9B5A1C0A921C70B8
:1002C0000A9B5A1C0A921C700A9B5A1C0A921C70A8
:1002D0000A9B5A1C0A921C700A9B0122991814A8A6
:1002E0000A911A7050F8283DDB1B3B701DF0DEFFB1
:1002F000724B2C70C3F8B062FDF76EBE98E80C002C
:1003000001210AA884F830110A920B931DF056FFC0
:10031000B1E4C4F83C6187F80080FDF7D7BD4FF029
:1003200000084046FFF787BB4046FFF76BBBDFF88E
:10033000C081D9F80030694F5E209847D9F8003065
:1003400011209847B8F80E204FF4F36B0BFB02F224
:1003500087FB0237D217C2EB6737F8B21DF00CFFEC
:10036000C7F307201DF008FFD9F800305E2098473A
:100370001920D9F800309847B8F80E30584A0BFBCE
:1003800003F382FB0301DB17C3EB611382FB032141
:10039000DA17C2EB6112642101FB1233D8B21DF0EF
:1003A000EBFE00201DF0E8FE9AF80030B8F8087067
:1003B00099077FF5D4AB5FFA87FB3F0AFFF7D1BB04
:1003C00003F0F1FEFDF797BD01230393FFF73FB85C
:1003D0003C4B1F6807EB87077F00FEF786BAC346D2
:1003E000C246424688E4D9F80030DFF808B1DFF8A9
:1003F00008A15E209847D9F8003028209847DBF8FC
:1004000000308AFB032ADB17C3EBAA0A5FFA8AF0E3
:100410001DF0B2FECAF307201DF0AEFED9F8003081
:100420005E209847D9F8003004209847B8F8083083
:10043000002B40F04B82DBF8083083F310085FFAA2
:1004400088F01DF099FEC8F307201DF095FEFFF718
:1004500079BB342728E59BF800309AFBF3FAFFF7C5
:100460003ABB204AD278002A0CBF4FF004084FF064
:100470000508FEF767BE0123D9F800003B7003F0C2
:100480009BFE0746D9F8000003F096FE7F067DF438
:100490001DAD8A2800F043828E287DF417AD9AF8AE
:1004A0000030002B7DF42EAD0F48104B03602D2340
:1004B00084F840310768FDF70DBD00BFF41F002030
:1004C00000000000CC5100208C5200202E9C002007
:1004D000785B0408805B04088C5B040889B5F81419
:1004E0001F85EB5120470020405200200853002078
:1004F000A4A50020F04F002067666666CF4AD04B67
:100500000D920DF15008A2F13D0048F8200D198818
:10051000DFF85493A2F1400300204FF00A0E02F8D6
:10052000400C082283F801E040469A7005F0D9F8A3
:10053000D9F80030C349DA1781FB0313C2EBA303D8
:1005400099B2404605F0CDF810F092FAD9F808902B
:100550000C9B4FEA1942591C0C911A700C9B4FEAE4
:100560001922591C0C911A700C9B5A1C0C9283F87E
:1005700000900C9B5A1C0C92187040461DF096FE81
:10058000FDF7D3BDAD4B0D93A3F14009002221210E
:10059000A3F13D0A03F8402C89F8021089F80120E4
:1005A000CDF830A023F026FAA74BA84A1B88A8490B
:1005B00000280ABF11464FF003084FF004085A05FF
:1005C00000F19F81D80700F1BE8103F00203A14A28
:1005D000002B1CBF4FF00308114642469E4830F0E6
:1005E0008FFD0AEB080314A89C4A013340F8203D14
:1005F0009B1A00220AF8082089F801301DF056FEE7
:10060000FDF796BD4FF00109FEF77EB8DFF86C925A
:100610009FED938AB9F90230884A0D9207EE903A1D
:10062000F8EEE77A0DF1500867EE887AA2F1400300
:10063000FDEEE77AA2F13D0148F8201D02F8400CDA
:100640000822CDED027A5A701E229A70BDF8081069
:10065000404605F046F8B9F9003007EE903AF8EE5A
:10066000E77A404667EE887AFDEEE77ACDED027ACA
:10067000BDF8081005F035F8B9F9043007EE903AE6
:10068000F8EEE77A404667EE887AFDEEE77ACDED40
:10069000027ABDF8081005F024F840461DF006FE69
:1006A000FDF740BD5FFA8BF01DF066FD4FEA1B20A1
:1006B0001DF062FDFFF7B5BA99780393184614F060
:1006C0002BF900287FF4B6AB5D49664F664A09886E
:1006D0006648674CF961DFF8A89111680368926871
:1006E000F962B4F86211C7F86CB0FB63FA64D9F828
:1006F0000000F965FBF770FA834600287DF451ACE1
:100700005146D9F8000003F04EFD039B94F8642194
:10071000DB780493642A4FF0040387F8743040F0C8
:10072000198194F86531072B08BF84F865B194F8F6
:100730006521504B079207EB021A0393DAF8041075
:10074000069108462FF09EFDDAF8083005935FFA0F
:1007500080FA18462FF096FD5FFA80FB454B079A0A
:1007600006990AEB0B000830D87122F00F0098723E
:1007700002F00F020BEBCA005A739873524603F152
:100780000F0030F0BDFC059B19463B4B0AF10900F8
:1007900018445A4630F0B4FC3648C37903F1010AD4
:1007A000CBB1013B5FFA83FC0CF1080CDFF8D4E01D
:1007B00084440023073010F8012B5A409300D108DD
:1007C00083EA420301F0180153404EFA01F253400C
:1007D0008445DBB2EFD1284A04980AF8023030F0A1
:1007E0006BFC94F865310022013384F8653184F89C
:1007F0006421039BDDF80CA09B785BB11AF805100F
:10080000D9F8000003F0E1FC01359AF80230EDB2AE
:10081000AB42F3D894F864310322013384F8643195
:1008200087F8742088F80020FFF79EB80E4B8046AA
:10083000B3F900A06420FDF75EBD00BF8C5200201C
:10084000189A002067666666B25100205C5B040857
:10085000645B0408745B04084F5200204D52002072
:1008600058A08B411C000020F04F0020CC510020EC
:10087000F41F0020BCA50020C2A50020D4510020F8
:10088000CC3F00200007090E854B864A1B889279D1
:1008900003EB830303EB83034FEA83081FFA88F813
:1008A000002A40F0FA804FF0FF330FFA83FA10F07D
:1008B000DFF840B2FDF71FBD114694461746924639
:1008C0000492FDF714BE2427FFF7EEBA10F0D0F81B
:1008D0001DF052FC00201DF04FFCFFF733B9D9F892
:1008E00000305E209847D9F80030392098475FFAE9
:1008F0008AF01DF041FC4FEA1A201DF03DFCFFF785
:100900001AB94FF00308684967E61027FFF7CCBA19
:10091000138907EE903AF8EE677AFEF709BB634B4E
:100920001B6898067DF5D2AA9AF80030002B7DF45A
:10093000E9AA5F485F4B03602D2384F84031B9E595
:100940002027FFF7B1BA5C494FF0040845E60827B5
:10095000FFF7AABA97F8753058481A0704BF013351
:10096000DBB2072B28BF01234FEA031B07EB0B0267
:100970005FFA8BFA92F810E0514A039200EB0E01F5
:100980000022087A4E498A7201F10D0207EB0B0131
:100990004AEA0E0E012882F800E0C96802F1010C53
:1009A0000DD90238C0B200F1020E9644624602F838
:1009B000011B72454FEA1121F9D101308444BB4437
:1009C00021F0600201339BF81110DBB20A43082BBF
:1009D0008CF800200CF1010249D04FEA031B07EB11
:1009E0000B00384990F810E034487044511A007AEE
:1009F00001EB000C0AF1100ABCF1130F5FFA8AFA3E
:100A0000C4DDC9B28A1DD2B2039842F0400E80F80C
:100A100007E002F1010ADFF8B8E0CAB105315FFA78
:100A200081FB0BF1080B83440EF1010C00221CF832
:100A3000010B5040820082EA4002C1084240224835
:100A400001F0180140FA01F14A40E345D2B2EED17B
:100A500004980AF80E2087F8753030F02DFBC8E6B0
:100A60001146FDF744BD11469446FDF740BD1549BA
:100A7000511AC6E7114694461746FDF738BD114690
:100A8000944617469246FDF732BD114694461746E6
:100A9000924604929046FDF72ABD0C4B1B6804E772
:100AA000189A0020B8510020685B0408C851002043
:100AB00040520020345300206C5B040834240408A6
:100AC000BCA50020C9A500200007090EF04F00209A
:100AD000C2A500202DE9F047C44B1C6862072DED2C
:100AE000028B03D4BDEC028BBDE8F087C04D2B78A0
:100AF000002BF7D06E6846F2A713861B9E42F1D9F1
:100B0000DFF850936860B9F80070DFF84C83002F6D
:100B100040F0A68198F80620AB689FEDB60ADFED9D
:100B2000B60ADFF8F492013AB3FBF2F307EE903A1B
:100B3000F8EE677AB7EE008A27EE800A30F0E8FC1C
:100B4000DFEDAE7A38EE400A20EE270A30F018FCCE
:100B5000B8F80830DFEDAA6A07EE103AEB68C01A61
:100B6000B8EEC77A07EE900AA7EE668AB8EEE70AF3
:100B7000D9ED097AF8EEE77A20EE080A67EEA67A50
:100B8000A7EE270A30F0FCFB9E4BC9F82400024672
:100B90001860A30740F1AA81DFF8C0E29A4CDEEDAD
:100BA000007A9FED9A5A2168F8EE677A27EE855A07
:100BB000002900F0BB81964B07EE101AD3ED026AB4
:100BC000B8EEC77AF8EEE66A86EE878A914991ED2B
:100BD000004AB8F80C10D5ED054ADFED895A95EDBD
:100BE000066A67EE847A06EE901A67EE887A8A497A
:100BF000B6EE004AF8EEE66AF0EE643AE7EE843AC2
:100C000066EEA56A91ED097A7E49F7EE005A75EE17
:100C1000E65AB8EEC77AA3EE856A77EEA47A27EE95
:100C2000257AC5ED057AF0EE477AE6EE267ABDEE36
:100C3000E77AC5ED067A81ED007A784909781229BC
:100C400000F05B8100211960596099602160CEF845
:100C50000010002F7FF446AFE869EA61121A07EE30
:100C6000102ADFED6F6A6F4B07EE906AB8EEC77A15
:100C7000F8EE677A27EE267A40F2DC52C7EE276A52
:100C80000A21FDEEE67A17EE900A9042A8BF1046C0
:100C90009842B8BF184604F05BFFB8F80A309FEDE1
:100CA000586AD5ED056A07EE103AB8EEC77AF7EE46
:100CB000007AE7EE467A05EE900AF8EEE55A66EE1F
:100CC000866A67EEA57AE7EE267AB0EE670AC5ED8A
:100CD000057A30F055FB0521064604F039FF524AEB
:100CE0005249B2F90040086084EAE473A3EBE4736C
:100CF000B3F5487F74DAB2F9022082EAE273A3EB1B
:100D0000E273B3F5487F6BDA494B1B78002B40F058
:100D10001181484B3B4A1B68126847489B1AB3F540
:100D2000FA7FA8BF4FF4FA739842B8BF18460A2159
:100D300004F00EFF414B1C68637A00FB03F00028AF
:100D4000B8BF7F30C211B2F5967F3D4BA8BF4FF4BC
:100D500096729A42B8BF1A463A48E37E076895ED04
:100D6000087ADFED396A911B01FB03F3227F344ED1
:100D7000002B01FB0272B8BF1F335B11B2F5C81F15
:100D80003249A8BF4FF4C812B3F5967FA8BF4FF4FD
:100D900096738A42B8BF0A46617F026007EE901AD6
:100DA00037EE087AF8EEE77A27EE267AB34267EE56
:100DB000877AB8BF3346002AB8BF02F5FF52FDEE6E
:100DC000E77AB8BF1F3203EB623317EE902A962AF8
:100DD0006FF09501A8BF96228A42ACBF9F1A5F1A96
:100DE0001B4A85ED088A17607CE600BFC8510020C9
:100DF000B822002008942537B1DC423ED048874A0B
:100E00006F12833ACC51002020660020BD37863512
:100E1000106600209C6B0020006C00203C99002094
:100E20000024744924FAFFFFD4510020D05100203F
:100E3000E4260020DC2600200CFEFFFF28520020C4
:100E4000D4FEFFFFD42600200000003B0000E7FF97
:100E5000CC2600206EBA0020886100201C6600208D
:100E6000374998F806A00A68AB689FED360ADFEDAF
:100E7000360A002A0AF1FF3AB3FBFAF39246B8BFEA
:100E800002F1070AA2EBEA0203EB020ABAF1000F31
:100E90005346B8BF0AF10703DB1007EE903AF8EEAD
:100EA000E77AC1F800A027EE800A30F031FBF7EEB8
:100EB000007A77EEC07A9FED257A2B6967EE877A04
:100EC0009A4518BF07F1FF33FDEEE77A14BF9FB2D2
:100ED00000274FF00003C5ED037A18BFC5F810A036
:100EE000A9F800706B61AB61002252E69FED188A91
:100EF000DFF870E0174C184B9FE695ED057AD5EDBD
:100F0000067ADFF864C02068996891FBF0F1BDEEC5
:100F1000C77AFDEEE77A17EE100A17EE909AACF852
:100F20000200ACF80010ACF804908BE69FED088A44
:100F3000094B4BE6094A0A4B12681C680CE700BFD4
:100F40009400002008942537B1DC423ED048874AFF
:100F5000000000002066002010660020E02600202F
:100F6000285200201C660020409900202DE9F843FB
:100F7000304B1B685B0701D4BDE8F8832E4C2F4D26
:100F800094F82490B9F1010F48D1EB6928469847AD
:100F90002B69284698472B6A04F12C0004F128019C
:100FA0009847274B276B9B79A668E06A07F10108F1
:100FB0009845636B08BF84F8009003F1010208BFF5
:100FC0004FF00008032A1FD01E49626394F83820AE
:100FD00041F82300FAB904EB870704EB8803F863B0
:100FE000DA6BAB89C4F83080B61A30440022A060B6
:100FF00084F82420002BBFD0134A0A2B1268B8BFF4
:101000000A231361BDE8F8830E4B01229860002388
:1010100084F8382063632EF09BF8DCE76B69284680
:101020009847AB69284698470122EB8984F8242029
:10103000E0E700BFC8510020B8220020006C00206B
:101040008861002094A50020A8610020F8B5534BCA
:101050001B681C0700D4F8BD514C524E524D7368AA
:1010600004F1FC01074630469847B4F9FC00B4F996
:10107000FE20B4F90031317E286028466A60AB60FA
:101080001BF06CFF494A137859073ED4D4F8040189
:10109000474B1B7883B1474B2968B3F90AC0B3F9B2
:1010A0000CE0B3F90E606A68AB68A1EB0C01A2EB2F
:1010B0000E029B1B85E80E000028CCD03E4B381A50
:1010C00098423FD9B4F91451B4F91011B4F9087128
:1010D000B4F90A21B4F91261B4F90C313548394434
:1010E00032442B4401EBD17102EBD27203EBD37388
:1010F0005B1049105210002541818281C381C4F8E0
:101100000451BDE8F840FBF7E3BA2C4EB5F90000F6
:10111000B5F90410A4F8080123F0040313700022A9
:10112000B5F90830A4F81001C4F804713260B28037
:10113000A4F80A11A4F81211A4F80C31A4F814317F
:101140003846A5E7002003F058F82B68B4F90821C9
:101150009342B4F91021B8BFA4F808319342C8BF34
:10116000A4F81031B4F90A216B689342B4F9122142
:10117000B8BFA4F80A319342C8BFA4F81231B4F939
:101180000C21AB689A42B4F91421C8BFA4F80C3101
:101190009A42BFF660AFA4F81431F8BDC8510020E0
:1011A000B8220020C44E0020589C00202452002069
:1011B000E44E00204C6E00207FC3C901566E002013
:1011C0002DE9F047C74C636820469847002800F097
:1011D000C380C54B1B780122042B84F83C2000F00F
:1011E000BD80B4F91610B4F91820B4F91A3021638F
:1011F0006263A363BD4B1B88002B69D0BC4DD4ED4B
:101200000C7AD5ED004A95ED050A95ED015A95ED5C
:10121000067AD5ED035A95ED026AF8EEE76AD5ED48
:10122000047AA4EEA60AA5EE267A67EEC07AA5EEA9
:10123000C07AE6EE267A85ED057AC5ED067A30F0BD
:101240009FF8D4ED0D6AD5ED094A95ED0E0A95ED9E
:101250000A5A95ED0F7AD5ED0D7AD5ED0C5A95ED2C
:101260000B6A2063F8EEE66AA4EEA60AA5EE267ADB
:1012700067EEC07AA5EEC07AE6EE267A85ED0E7AA4
:10128000C5ED0F7A30F07CF8D4ED0E6AD5ED124A38
:1012900095ED170A95ED135A95ED187AD5ED167A56
:1012A000D5ED155A95ED146A6063F8EEE66AA6EE80
:1012B000A40AA6EE857A67EEC07AA0EE657AE6EE1D
:1012C000867A85ED177AC5ED187A30F059F8A06363
:1012D000884FA17F88481BF041FE3B88002B40F0DF
:1012E0008480864ED6F81851854B1B685B0743D423
:1012F000B5F90070216B636BA06B824A824E92ED50
:10130000026AD2ED006AD2ED015AC91B2163B5F918
:101310000270DB1B6363B5F904703568C01B07EE10
:10132000900AB8EEE75A07EE901AB8EEE77A07EEA1
:10133000903AF8EEE77A36EE056A36EE877A77EE7F
:10134000A57A0135A06382ED026A82ED007AC2EDD2
:10135000017A3560BDE8F087BDE8F0876B4BB4F9E2
:101360001600B4F91810B4F91A20188020635980B7
:1013700061639A80A2633DE7B6F82821322A00F023
:101380008880002A66D196F84631002BB0D060489C
:10139000D6F838215F4980FB0273D217C2EB2312C3
:1013A0002A80D6F83C2180FB0273D217C2EB2312AD
:1013B0006A80D6F84031A78A80FB0302DB17C3EBB3
:1013C0002213DB1BAB800023CB6086F8463112F082
:1013D000C1FA03F097FE12F0A5FAFAF7D9FF01203F
:1013E0002AF05CFCD6F8185182E7444E226BD6F8FE
:1013F0001851B3F5C87F4FF0000323632B80398861
:1014000018BFD6F81C01B7F8008008BF0020B1F55E
:10141000C87F18BFD6F82031616B02440B4400200E
:10142000B8F5C87F6063C6F81C21C6F82031688013
:1014300052D0D4F838E0D6F82411A0637144B8F142
:10144000010FA880C6F8241168D008F1FF38A7F86A
:10145000008049E7D6F83801236B00210344C6F821
:10146000383121632980D6F83C01636B6163034402
:10147000C6F83C316980A36BD6F84001A1630344F0
:10148000012AC6F84031A98075D0013AA6F8282172
:1014900079E72B8820491F48276BA6F82C310023B9
:1014A000B5F802E0B5F804C0C0684B608B602363F8
:1014B000C6F838712B80616BC6F83C1163636B8092
:1014C000A16BC6F84011A363A6F82EE1A6F830C1BF
:1014D000C6F83401AB80D8E7A36BC6F82431A0630B
:1014E000A880B2E7DC5100203C990020944A0020FB
:1014F000984A002070BA00200C520020B822002028
:10150000C08D0020DC650020D865002040990020B7
:101510001F85EB513C6E0020F0230020DFF804C152
:10152000DFF8F0E0C8328CFB02A9C833D217C2EB57
:10153000E9128CFB03A9DB17C3EBE913C8316B80FD
:101540002A808CFB013CA28ACB17C3EBEC139B1ABD
:10155000AB80CEF80C0012F0FDF903F0D3FD12F0D1
:10156000E1F9FAF715FF40462AF098FBB7F800803A
:10157000D6F8185169E7254B86F844111B6886F8A0
:10158000452113F4003334D119462148475C0B2F11
:1015900001F10C0110D00133182BF7D1B6F82C1142
:1015A0001C4B2980B6F82E71B6F83001D6F83411EC
:1015B0006F80A880D96068E7174FD7F800C059003E
:1015C000BCF1000F09D001EB030E00EB8E0E9CF86E
:1015D00001C09EF801E0E645E0D20B44DFF848E0A8
:1015E0000E4900EB830000233860AEF800300B603A
:1015F000D4E70B4B1B78032B01D00B46C5E72AF031
:101600000BFAD6F81851B6F82821C7E79C450020F8
:10161000844504083C6E00206027002068270020D5
:101620001D4700201F85EB51642700202DE9F04F56
:101630009F4BA04A1C7897B000F59C412031814611
:1016400009911160002C00F0FE849B4A12689042C0
:1016500040F28380994A089216689949994ADFF8BE
:10166000A0A20791013C04921C7006F48056002E43
:1016700040F08180944B1B78022B00F04B87042BA9
:1016800000F03A87012B00F0EE86904B99459AF8CE
:10169000023000F2AC83002B40F0AD838C4B0993F9
:1016A000089B1E6816F4805740F09B84DFF8549224
:1016B000049BB3F90610079B5C8BA142B4BF0024C6
:1016C0000124844B1B6813F080535ED0099A127872
:1016D00012F001025FD00798408C884241F3B1803C
:1016E000002C5ED17C4D95F8D411002959D17B484E
:1016F0007B49006890F82D0000250D604D608D60DD
:10170000784900284ED10870002A4FD0F1064DD5F7
:10171000754A1278D20649D4002F47D1002B45D103
:10172000750243D4714B1B78002B02F09480704BF0
:101730009B78002C42F09F803BB16E4A6E4B126842
:101740001B689B1A002BC2F2AD801020624D2AF05C
:101750007FF9012385F8D53128E0584B08931E689E
:10176000574A584B079206F480560493DFF890A12D
:10177000002E3FF47FAF0021564804F0BAFC002849
:101780007FF478AF0DF088FB74E770029ED4099A5D
:10179000127802F00102504D002185F8D411002C7E
:1017A000A5D0504901200870002AAFD1534B1A78B8
:1017B000002A40F0B3800799049D488BB5F900706A
:1017C000898BB5F90250B842B4BF8026002646F096
:1017D0004003B942D8BF33469B0843F08006A84275
:1017E000B8BF3346049F43F04006A942C8BF334602
:1017F0009B08B7F90450B7F9066043F080078542AB
:10180000C8BF3B4643F040078D42B8BF3B469B08EC
:1018100043F08007304D8642C8BF3B4643F0400747
:1018200095F8D6E18E42B8BF3B469E4501F06282F4
:10183000A5F8D82185F8DA212C4985F8D6310E781B
:10184000002E01F04E815F2B01F0D7816F2B01F04C
:101850001782099B1B78DB0760D495F8DA11002901
:101860005CD1B5F9D831322B58DD95F8D62101205D
:10187000572A85F8DA0101F07E85089B1B685C0712
:1018800041F19C805A2A41F0998095F84531002B0E
:1018900041F0D18795F8DC3183F0010385F8DC3124
:1018A000002B42F011800C202AF0D2F801F0B9B9D7
:1018B000C83E0020783D0020C43E0020C08D00209E
:1018C0005076002050B100207E4E0020404B4C004E
:1018D00000620020846C0020B822002028520020E2
:1018E000E86B00208426002024520020981D002050
:1018F0005C6E00203C8500206C270020CF9C0020DF
:1019000020470020803F00200F202AF0A1F8B5F8E2
:10191000D83185F8DA41FA3BA5F8D831089BB14AAD
:101920001B680692B04C5F0700F174840DF1500BF8
:10193000DFF8DC820A940023CBF804304546149388
:10194000192740F6330340F28336049C02E0043545
:101950004D4522D0A878E978884217FB006EF6D270
:101960006878043017FB016134F910009842A8BF71
:101970001846B0F5617FB8BF4FF461707045E6DD81
:101980008842E4DC29782729E1D8584604350593B4
:1019900004F0A0FB4D45059BDCD1944B944A1B7889
:1019A0000A9C9BE8030082E80300002B40F01581AD
:1019B000904B1F78002F00F0B78301218C4804F072
:1019C00098FB002840F048819AF80330002B40F043
:1019D000438123881DB225F00105AEB2B3422680B3
:1019E00000F0BD85844D02270E204FF014094FF002
:1019F000FF082F7085F8019085F802802AF028F8FA
:101A000039467B48268804F074FB002841F0C680E4
:101A100026F002039BB2B34223800AD0764B1421F6
:101A2000FF2202250E201D7059709A702AF010F8BE
:101A30002688DFF8E0B1DFF8E0A19BF80010DAF8C3
:101A40000400B50708BF81F00201C1F3400102F0B4
:101A5000B9FF2421664804F04CFB30B9099A137889
:101A6000590744BF23F004031370069B1B6813F04F
:101A70000A0F1DD005215E4804F03BFB002800F052
:101A8000B68625886F0741F141805948062104F048
:101A900030FB002800F098866E0641F12F80072168
:101AA000534804F026FB002840F0B485069B1B68D1
:101AB0009D0600F10A8326884D480C2104F019FB8D
:101AC000002800F0E48046F48073B342238009D0FC
:101AD000494B02251421FF220E201D7059709A7067
:101AE00029F0B6FF454B1B78082B00F0DC800E2B4D
:101AF00000F0D980089B1B685D0548D5404B1B79D9
:101B0000002B00F08D801421394804F0F2FA0028EF
:101B100040F08B801CF024FC012029F0A3FE00285B
:101B200035D0DFF8F88000254FF0CC0902E0DDB2B7
:101B3000022D2CD809FB05F76B1C58F80760002E06
:101B4000F5D1032290F9023002960192C2782D4914
:101B500051F822200092184632463346012129F0DE
:101B600077FA034605EB450000EB0010059353B1EF
:101B7000314608EB8000CC2230F0BFFB059B48F8D3
:101B800007300135EDB226F05DFB0028D0D1099B6E
:101B90001B78D80740F19A809BF800101A4A1B4D19
:101BA000DAF80000012301F0010113702B7002F03C
:101BB00009FF069B1B685A0700F1FC8017B0BDE8BF
:101BC000F08F98F8022098F803309A42C0F0B2865D
:101BD00008F1040845453FF4EBAE98F800102329BE
:101BE000F6D1EEE7C8510020B2510020E48F00206A
:101BF000846C00200D9C0020CC4600206C6E0020E0
:101C0000209A00206C4A0408F0260020016200207F
:101C1000303F0020048500200885002048AE0020C9
:101C2000099B1B78D9077FF575AF4FF40F702DF026
:101C300079FC0028ABD00FF0DFFA4FF40F702DF0D5
:101C400007FC0028A3D00FF0D7FA4FF40F702DF047
:101C5000FFFB0028EFD19AE7069B1B689A077FF5E8
:101C6000B8AE2688F3073FF5D3AE46F001039E4297
:101C700023803FF4CDAEB44B1421FF2202250E2069
:101C80001D7059709A7029F0E3FE2688C0E626F48C
:101C900080739BB2B34223807FF41AAFAB4B1B78A7
:101CA000082B7FF424AF228822F040039BB29A4293
:101CB00023803FF41FAFA44B02251421FF220E20E6
:101CC0001D7059709A7029F0C3FE13E7A04B1E785F
:101CD000002E65D19F4B1B68002B61D0DFF8C082BE
:101CE000DFF8C09218F8030C99F804704146A8F187
:101CF000030521F055FE002800F0BB85002F40F0C1
:101D00000C8605F10801687921F04AFE002841F0AF
:101D100000859149A87A21F043FE002800F0BC8597
:101D2000022F41F019858D49E87B21F039FE00280A
:101D300041F00E858A49287D21F032FE002800F00E
:101D4000BC85042F41F0F5848649687E21F028FE89
:101D5000002841F0EA848449A87F21F021FE002870
:101D600000F0BC85062F41F0DC84804995F8230003
:101D700021F016FE002841F0D0847D4995F8280016
:101D800021F00EFE002800F0BC85082F41F0BD8434
:101D9000784995F82D0021F003FE002840F0BC851D
:101DA000754B01221A702DF059FF069B1B685A07CC
:101DB0007FF504AF032021F02BFE002800F0B2874E
:101DC000238813F008047FF4F9AE08200CF05EFAC3
:101DD000049E6A486A4D6B496B4A6C4BF6880068F2
:101DE0002E80086014601C6017B0BDE8F08F13B936
:101DF00001238AF80230664B09931B201D789AF85C
:101E0000214021F005FE012C05F00108814600F07B
:101E10000F8705F0020305939AF820305D4EDFF836
:101E200088B15D4F052B00F2CF80DFE813F0BF00D3
:101E300082000600FD00FF00F200012C04BF052314
:101E40008AF82030B8F1000F12D0079B3088B3F920
:101E500018100022134661F30F0260F31F4261F372
:101E60000F03049861F31F4303600323426005934B
:101E70004A4DDAF814202B689A4280F0228647F205
:101E800030520323CAF81C208AF8203002200CF0BC
:101E900015FA0DF001F82A68DAF81C301344042210
:101EA000CAF818308AF82020012C40F080872B686F
:101EB000DAF818209A4280F087809BF8000018B961
:101EC00021F0A6FD00287FD13B6823F002033B6090
:101ED0002A687388642101FB03234FF48060002289
:101EE000CAF810308AF820208AF803200CF0B6F9DE
:101EF0009AF8203096E721F091FD012807D1274D6F
:101F000073882A68642101FB0323CAF81030B9F1F1
:101F1000000F02D0B379002B7DD1012C54D01F4D7E
:101F2000DAF810202B689A42C0F0498701238AF81A
:101F30002030012C6DD0F379012B79D021F0EEFC0B
:101F40009AF820306EE700BFCC4600206C6E00206F
:101F500001620020046200209C460020A14600206F
:101F6000A6460020AB460020B0460020B546002023
:101F7000BA460020BF460020F0260020CC510020A9
:101F8000D0260020DC260020D4260020CC260020ED
:101F900000620020A06B0020205200203C85002021
:101FA0009246002094000020981D0020B8F1000FF8
:101FB000A1D14FF48060B9F1000F00F0EE820CF077
:101FC00065F90023CAF81030059B002B3FF468AB7D
:101FD000184629F03DFD089B1E6816F480573FF413
:101FE00065AB1D219E4804F084F800287FF45EABA9
:101FF0009C4B03F1500903E00433994500F09786A8
:102000001A78262AF8D19978DA789142F4D2FFF733
:102010004FBB954D5CE721F081FC03224FF47A73AE
:102020008AF82020CAF81C308F4D2FE78E4D3BE7F1
:1020300021F074FC032240F6B8338AF82020CAF855
:102040001C30894D22E7894F3B78002B01F04A82F2
:10205000874BDFF85082DFF850B2DFF850A20793C9
:1020600045465E46049099460EE019F804109847DC
:10207000032C28DC88B93B782AF8020F01349C42F3
:1020800005F1040580F21881072CE1B23046DBF837
:102090000430EADD984700B2EDE738F824206B8879
:1020A000801A4FF47A719B1A01FB00F040F6CA02C5
:1020B00090FBF3F00844904240F2EE23A8BF104694
:1020C0009842B8BF184600B2D5E76A4B1B7898070C
:1020D00004D5694D2B7D042B00F27C86268816F0F2
:1020E000300F3FF4E9AC10200CF0B8F820200CF0D1
:1020F000B5F8624B268800221A70614A6148624F27
:10210000624D00211160624A3960002329604160FC
:102110008161036083604361C361136051609360B8
:1021200053619161D361C7E4DFF884B1DFF8848142
:10213000584D0BF15A064FF0010959461BF8010C96
:1021400021F02EFCF8B19BF804009BF802309BF8BC
:1021500003E000EB400105EB8101013BD1F8E421F4
:1021600003EB4303434493420DD095F8102281F8CA
:10217000E0E109FA00F022EA0000C1F8E431C1F818
:10218000E87185F810020BF1060B5E45D5D1424986
:10219000354A424B424D09681B78D2F800900A91AB
:1021A0000593A5F5F07B00266B6863B31F7857B3E2
:1021B000AA68A9EB0202002A0ADB9BF8102201217F
:1021C000B14022EA010209F5FA718BF81022A960E8
:1021D000059AC2B12A7859780432D2B2002940F067
:1021E000368307990498098B30F9122001F1C80051
:1021F000824240F3AE859BF810129A7841FA06F3BA
:10220000D80740F14E860136042E05F10C05CBD1DE
:10221000FFF7D3BB1F4D95F8DC315BB1099B1B78F1
:10222000DE0707D5049BB3F90620079B5B8B9A4218
:1022300000F3298611210A4803F05BFF002800F013
:10224000EE8295F844312BB995F8453113B9322314
:10225000A5F82831012385F84431FFF767BB00BF9B
:10226000846C0020303F00203C850020F43F00209B
:102270005076002024520020A4A500205C490020B4
:10228000484A0020F8490020582600204C2700200A
:10229000204A0020B82200202C52002014470020A1
:1022A0009824002008400020709C0020FE2300207D
:1022B000A945002070240408DDF81090B84AB949F7
:1022C00008921268A1FB091B42F2010111404FEA7A
:1022D0009B1B0F9100F0A082B34DB448B44CB5499C
:1022E0002E780078267008701EB1B2490E7886F0FC
:1022F0000106B14D0F2185F86C11002B00F02384ED
:10230000AE4B079C0E93B4F824E0B4F826C0079CAB
:10231000CDF82CC01846248B0078A94B1294A94CF8
:102320000D9004940446A3FB00035B0803EB4303F6
:10233000E31ADBB295F86D810A9302F4805205F539
:10234000B8700BF59673119597F800A0DFF8BCC232
:102350009C4C0C917546DDF83CE0139200210693ED
:102360000596CDF84090059B002B00F04D83964BD1
:1023700033F911301FFA83F9A9454FEA410203D31B
:102380000B9EB14540F284835CF821309B4580F080
:102390004483A35EBEF1000F40F0598301315145E3
:1023A000A35200F10600DEDB0C9A119D874B85F8E5
:1023B0006C210F2A0CBF01220022DDF8409085F825
:1023C0006D811A7000F0C6837848DFF844A279491D
:1023D0007F4D0122027004200A700BF06FFF2B6802
:1023E000DAF80810DAF80420CAF80C305B1A9342C5
:1023F00084BF00238AF821303C78089B1E68002C9B
:1024000001F07880079A734DB2F824E0178B6D497C
:1024100016F48056284640F0D28332460EE04378C8
:1024200003EB830303EB830303F2EE239BB201323E
:10243000A24221F8023B00F102000ED015F8123042
:10244000002B00F02983022BE9D001320B8821F800
:10245000023BA24200F10200F0D10E9A1378013340
:102460001370FFF704B9544DD5F8D031A9EB03032D
:10247000002BFFF60AA9584A584B527C079933F8AB
:1024800012308A7DDFED566A9FED566AC97D9BB298
:1024900007EE102A07EE903AB8EEC77AF8EEE77A20
:1024A00027EE267A67EE867A099AC5F8D021C7EE1C
:1024B000876A40F2FF32FCEEE67ACDED057ABDF890
:1024C0001430934228BF134609B1D31A9BB2464831
:1024D000464D0178464C35F81160226825F81130D8
:1024E000921B13440131434D236001F00F021B097D
:1024F00002702B80FFF7C9B8FAF7D6FE3E4B3F4A71
:102500001B68C31A93427FF7C0A83A4B00221A8077
:10251000FFF7BBB8079A0499537DD27D013B31F98F
:1025200013301AB1C3F53B6308331BB2A3F57A73BA
:1025300007EE903A9FED327A2E4AF8EEE77A40F2B3
:10254000FF3167EE877AFCEEE77ACDED057ABDF8CC
:1025500014308B4228BF0B461380FFF796B8022138
:10256000284803F0C6FD00283FF452AA2580B7078B
:102570003FF55FAA46F00203B34223803FF459AA15
:10258000214B02201421FF2218700E2059709A70DE
:1025900029F05EFA2688FFF74CBA0BF05FFE10E5D3
:1025A000C08D0020D34D6210543D0020EC0000206F
:1025B00014470020ED000020B8220020E53E002056
:1025C000ABAAAAAA50B1002000240020DE9C002063
:1025D0003C8500203C4000208C850020AC850020FC
:1025E0000000C842000080447F4E0020844E00203E
:1025F000804E0020B05100200025002060E316002E
:102600006F12833F846C0020CC460020E83E0020FF
:1026100020470020CD4AB2F90030002BB8BF5B4202
:10262000B3F5E17FBFF642AAB2F90230002BB8BF82
:102630005B42B3F5E17FBFF639AAC54B93ED096A5A
:10264000D3ED076A93ED057AD3ED037A76EE866AC9
:1026500077EE877A76EEA66AB7EE007A37EE666A8C
:1026600077EEA77AB0EEC66AF0EEE75AB4EEE56A06
:10267000F1EE10FAB4BFB0EE655AB0EE465AB5EEC0
:10268000405AF1EE10FA40F0CF839FEDB27AB4EEEB
:10269000E56AF1EE10FA44BF9FEDAF6A36EE477A75
:1026A000B7EE006AF4EEC66AF1EE10FAC8BFDFEDCD
:1026B000AB6AF5EEC07AC8BF36EEC77AF1EE10FA13
:1026C00048BFB1EE477AF6EE007A27EE677ADFED83
:1026D000A27A77EE276ABDEEE66A16EE103A20334C
:1026E000402B40F26786DFED9E6A9E4ADFED9C7AC2
:1026F000C2ED006AFDEEC76AC2ED017A16EE903AAD
:102700002033402BC2ED027A49D8DFED947AB4EE43
:10271000E77AF1EE10FA41F38A809FED936ADFEDDC
:10272000936A01E0B0EE677AB4EEE67AF1EE10FA61
:1027300077EE467AF6DC9FED8E7AF4EEC77AF1EE0C
:1027400010FA41F170809FED886ADFED8A6A01E03E
:10275000F0EE477AF4EEE67AF1EE10FA37EE867A8A
:10276000F6D4DFED7D7AB4EEE77AF1EE10FA40F3BD
:10277000A386DFED7A7A37EEC77A27EE076ADFEDB8
:102780007E5ADFED7E6ADFED7E7AE6EE256A67EE41
:10279000065AE6EE267AA5EEA77AF0EE477A794B4E
:1027A000C2ED037A1B6813F4003340F06286764969
:1027B0001A46C85C0A2803F10C0300F08385013235
:1027C000182AF6D1FFF772B925F040039BB2AB424D
:1027D00023803FF464A96D4B02251421FF220E20B3
:1027E0001D7059709A7029F033F9FFF758B9238892
:1027F00023F00405ADB2AB4225803FF446A9634BFC
:1028000002251421FF220E201D7059709A7029F0A4
:102810001FF92588FFF739B95D490E7864E595F809
:102820004531002B3FF482A8099B1B7813F001036C
:102830007FF47CA8012285F8453185F84621FFF711
:1028400075B8544D012185F8D411FEF7AABF0129AE
:1028500000F052859BF810220123B3400136134348
:10286000042E8BF8103205F10C057FF49DACFFF7B8
:10287000A4B808F10501687921F092F800283FF426
:1028800048AA012F40F0458705F10D01A87A21F0F3
:1028900087F8002840F060873F49E87B21F080F806
:1028A00000283FF447AA032F40F052873B49287D78
:1028B00021F076F8002840F03C873949687E21F005
:1028C0006FF800283FF447AA052F40F02E873549BE
:1028D000A87F21F065F8002840F02387324995F859
:1028E000230021F05DF800283FF447AA072F40F0AD
:1028F00014872E4995F8280021F052F8002840F05E
:1029000004872B4995F82D0021F04AF800283FF460
:1029100047AA092F3FF444AA0926334603EB830351
:102920001D44244B6978AA7889F8046019705A709C
:10293000FFF736BA204803F0DCFB00283FF438A844
:10294000142029F085F8FFF733B800BFD4510020D8
:1029500090140020A7DFA834DB0FC93FDB0F4940EC
:1029600000000000A0000020DB0FC940E4CB1641AE
:10297000DB0F49C0E4CB16C192E741B99730083C60
:1029800015A82ABE9C45002084450408CC4600209A
:1029900014470020B8220020A1460020A6460020AF
:1029A000AB460020B0460020B5460020BA460020C5
:1029B000BF46002008620020846C00205D2A00F0E1
:1029C00075825B2A00F092855E2A00F0FC85562A0B
:1029D00000F05086972A00F0B086A72A00F0E7851D
:1029E000B14C23889B0740F09785A2F1B703072BD2
:1029F00000F28682DFE813F07E0284028402840201
:102A0000780284026A026A02002D3FD05CF821300D
:102A10009B454FEA4102FFF4BCACA44BA34E9B5C28
:102A200006EB0209002B00F0AD80022B47D199F88C
:102A3000013003EB830303EB830303F2EE239BB22A
:102A4000032933DD1BB2BEF1000F3FF4A7AC0A9E91
:102A500020F81630B8F1000F03D10D9E022E7FF63C
:102A60009DAC4388B0F80090B0F804804B44984483
:102A70008F4B0FFA88F883FB08638E4EA3EBE87345
:102A800026F802801BB24FF0010887E42B464A006B
:102A9000069E4CF821607DE4D3B2022B04D9032BAF
:102AA0007FF4D3AC7346C2E43B46C0E4012606FA89
:102AB00001F90C9E26EA09061BB20C966AE4A35A99
:102AC000BEE77D4B1B78002B7FF4D9A9B8F1000F2E
:102AD0003FF4D5A9012C7FF477AA9AF82030FFF7AC
:102AE000A1B93146754803F004FB002800F0A4802A
:102AF00085F8DB610CF000FEFEF7ABBE45F040034D
:102B0000AB4223807FF467AEFEF7C9BF45F00403F4
:102B10009D4223800AD06A4B02251421FF220E20F9
:102B20001D7059709A7028F093FF2588654B664A8E
:102B3000B3F90430654982FB0302DB17C3EBA20340
:102B40000B80FEF7A2BF624B624A0E9201221A70FE
:102B5000614B04931B21594803F0CBFA00287FF402
:102B600033ACDFF88CA15D4DDAF80C202B68CAF885
:102B700008309B1AC82B00F2C184089B1E6806F41B
:102B800080566AE4CBB2022B40F2B383032B96D17A
:102B9000129B139E002E08BF2B4651E726F001031F
:102BA0009BB2B34223803FF4E2AC0E202F7085F835
:102BB000019085F8028028F04BFF2688D7E4002298
:102BC0000FE0437803EB830303EB830303F2EE236D
:102BD0009BB20132A24221F8023B00F102003FF415
:102BE0003CAC15F812301BB1022BEAD00B88F0E791
:102BF000D3B2032BFAD83B46EBE7B2F5FA7FFEF6E9
:102C00008DAE95F8DA31002B7EF488AE099B1B78E7
:102C1000012213EA020485F8DA213EF475AE0CF0C5
:102C20003BF92F4B0693089B1F4C1B68FEF77BBE9E
:102C300000230593FFF7F0B8099B2A4A1B78106020
:102C4000D8077EF50AAE284B1B78002B3EF466AE03
:102C50009AF80330002B7EF461AE95F8DB31013336
:102C6000DBB2032B85F8DB317EF658AE1F4B5B7869
:102C700013B9002C7EF452AE0CF00EF9FEF7E9BD4C
:102C8000B2F5FA7FFEF64AAE95F8DA21002A7EF414
:102C900045AE099B1B78012185F8DA11D90700F1AF
:102CA00018840CF029FDBCE7B25100203C40002004
:102CB000565555557024002074260020846C002041
:102CC000CC460020D451002067666666684A002022
:102CD000DE9C0020E53E002050B100203C85002015
:102CE000C851002070270020144700205C6E00208F
:102CF00020470020C44AC5491068B5F9D821C669E3
:102D000081FB06018911F617701A00F5FF407F302C
:102D100082423EF791AD891B0A4412B2A5F8D82130
:102D2000FEF78ABD08200BF099FAFEF747BFB84AB4
:102D3000079BD488049A1B8BB2F906101A1B914288
:102D400040F39E8023449942B4BF00240124FEF73F
:102D5000B8BCC8398A425ADA9BF810129A7841FAFC
:102D600006F3D9073FF54FAA524201200B9228F0F3
:102D700095FF7B1E0B9A162B00F29981DFE813F06A
:102D800022023802090261024E027502F401DF01DB
:102D9000C801B1019A019701610287017502F4012E
:102DA000DF0170012E0118018A020001EA002A6881
:102DB000DAF81C301344CAF81830FFF705B920F0D0
:102DC000ADFD032240F6B8338AF82020CAF81C3043
:102DD000FFF75CB80A2020F01BFE26880746002873
:102DE00000F03083F10640F12F848A4D95F8187277
:102DF000002F7EF461AE0D2028F02AFE012385F815
:102E000018322688002F7FF478A9FEF755BE9BF86C
:102E100010320122B24023EA020309F5FA728BF85C
:102E20001032AA60FFF7EFB9B4EEE56AF1EE10FADE
:102E30008CBFB0EE654AB0EE464AC4EE054A9FED3F
:102E4000762A9FED765ADFED761ADFED762A9FED32
:102E5000763ADFED763A9FED764AA4EE825AE4EEBA
:102E6000E12AA4EE857AA4EEA23AB0EE475AB0EE7B
:102E7000637AA4EE837AA4EE874A84EE057A06E4A8
:102E80000124FEF71EBC00216A4803F032F9002835
:102E90007FF4D0A9322385F8DC01A5F82831FFF7AB
:102EA000C9B9002A0CBF012002205FE7624B002253
:102EB00001206249624C0B60624B2270069328F03D
:102EC000EDFE089B604C1B68FEF72DBD5F4A604914
:102ED0005B4B116002225A705A4B069320F0FCFDA6
:102EE000089B1B68FEF71FBD584A5A491160544B96
:102EF0000022F0E7554A58491160514B0122EAE798
:102F0000792A00F087847A2A00F07D849E2A00F0D6
:102F100072849D2A00F06784AE2A00F05C84AD2A9A
:102F200000F05184EF2A00F04B84FD2A00F0368433
:102F3000FB2A00F0E884FE2A00F0E284F72A00F081
:102F4000DC847B2A00F01F84089B3E4A1B680692A3
:102F5000FEF7E9BCDBF81402DFF8008190F83610C8
:102F600098F8023011446429A8BF642121EAE17174
:102F700080F83610002B40F089841FF05DFE69E474
:102F8000DBF81402DFF8D48090F8371098F802309C
:102F90001144FE29A8BFFE2121EAE17180F8371013
:102FA000002BEAD0162020F07DFDDBF81402E4E7C8
:102FB000DBF81402DFF8A48081781144C829A8BF87
:102FC000C82121EAE171817098F80230002BD4D039
:102FD000142020F067FDDBF81402CEE7DBF81402C2
:102FE000DFF8788041781144C829A8BFC82121EAB8
:102FF000E171417098F80230002BBED0132020F010
:1030000051FDDBF81402B8E7A8610020D34D62102F
:10301000846B0020B822002099FB243F69A2163E51
:1030200039094E3DE3B59E3E88FA163E45FE7F3F88
:10303000A7DFA834846C00203862002028520020CA
:10304000289C0020C8510020B25100202C520020A2
:103050004C9C0020349C0020409C002058630020A1
:10306000DBF81402DFF8DC8501781144C829A8BF19
:10307000C82121EAE171017098F80230002B3FF479
:103080007CAF122020F00EFDDBF8140275E7DFF8AC
:10309000B4850A9898F80230417911446429A8BF90
:1030A000642121EAE1714171002B40F00384DBF8D7
:1030B000140262E7DBF81402DFF88885017A98F8D9
:1030C00002301144C829A8BFC82121EAE171017268
:1030D000002B3FF452AF0B2020F0E4FCDBF814028D
:1030E0004BE7DBF81402DFF85C85C17998F8023011
:1030F0001144C829A8BFC82121EAE171C171002B80
:103100003FF43BAF0A2020F0CDFCDBF8140234E79B
:10311000DBF81402DFF82C85817998F8023011442D
:10312000C829A8BFC82121EAE1718171002B3FF4B1
:1031300024AF092020F0B6FCDBF814021DE7DBF811
:103140001402DFF80085417998F802301144C8294B
:10315000A8BFC82121EAE1714171002B40F0B7837B
:10316000112F7FF429AF08E7DBF81402DFF8D484CD
:10317000017998F802301144C829A8BFC82121EA72
:10318000E1710171002B40F0B083102F7FF42AAF62
:10319000F3E60A99DFF8AC840F791744642FA8BFCF
:1031A000642727EAE7770F7120F096FC98F8023041
:1031B000002B3FF47CAF0320394620F073FCDBF892
:1031C0001402DAE60A98DFF87C8401781144FA29BF
:1031D000A8BFFA2121EAE171017098F80230002BB2
:1031E0003FF465AF012020F05DFCDBF81402C4E67B
:1031F0000A98DFF85084817811446429A8BF6421BB
:1032000021EAE171817098F80230002B3FF44FAF52
:10321000022020F047FCDBF81402AEE60A98DFF843
:103220002484C17998F80230114481F30801C171F6
:10323000002B3FF43CAF052020F034FCDBF81402F7
:103240009BE60A9BDFF8FC83997998F80200114409
:103250006429A8BF642121EAE1719971002840F036
:103260003E830D2F7FF415AF21E7DBF81402DFF862
:10327000D483C17898F802301144C829A8BFC82166
:1032800021EAE171C170002B40F004830F2F7FF41D
:10329000EBAE72E60A98DFF8AC8341781144B1F5E1
:1032A000967FA8BF4FF4967121EAE171417098F8BA
:1032B0000230002B3FF4FBAE152020F0F3FBDBF8CF
:1032C00014025AE6C24D2E6853003EB1981801EB25
:1032D000800076784078B042BEF4E8AB1A44BD4E28
:1032E000BD48002301EB8201296033800360FEF7B3
:1032F000DDBB129BFFF7A4BB049931F9122099782A
:10330000B2F5617F4FF4966393FBF1F3C0F2B9809D
:1033100040F633019142A8BF11460C2FA1F561710F
:1033200091FBF3F100F02382182F7FF493AAC9B226
:10333000C8290B46A8BFC823DBF81402C27DDFB240
:1033400097423FF487AA9A1ADFF8F882C77548BFF8
:103350000732D71098F802300137FFB23BB9002F7F
:103360003FF478AA384628F099FCFFF773BA182082
:1033700020F098FBF3E7994B99491A684FF47A7358
:10338000B3FBF2F3C3EB431203EB8202089B1B680F
:10339000D2001F06A1F8A82000F1FA80914A0692F7
:1033A000126855077EF5BEAA8F4A904C0A211180FB
:1033B000FEF7B9BAB4EEE77AF1EE10FA40F3E08125
:1033C000DFED8B5A9FED8B6A01E0F0EE676AF4EE59
:1033D000C66AF1EE10FA76EEE57AF6DCDFED866A83
:1033E000F4EEE67AF1EE10FA40F1C781DFED805A93
:1033F0009FED826A01E0F0EE667AF4EEC67AF1EEB5
:1034000010FA77EEA56AF6D4DFED7D7AF4EEE76A7E
:10341000F1EE10FA40F3B080DFED7A7A77EEE66AEB
:1034200066EEA65A9FED785A9FED786ADFED787ABE
:10343000A5EE856A26EEA55AE5EE867AE5EE276AC0
:10344000FFF753B9F20600F152810B2020F0E0FAA9
:10345000002840F01E81B30600F182816D4D95F881
:103460001832002B3FF4C7AC002F7EF446AEFEF7B7
:1034700023BB694B1B78032B00F07B810023FFF7F4
:1034800096B90C2F40F03B8100273946634B0B91D6
:103490005B78BB423FF4DEA9DFF8A88138460DF027
:1034A000C5FA98F802300B991BB1C9B20C2020F074
:1034B000F9FA0137FFB252E7DFED597AB4EEE77A55
:1034C000F1EE10FA44BFDFED4C7A37EEC77AFFF722
:1034D00054B95449089B0A60424A1B680692434CFF
:1034E000FEF721BA504A0792FEF7E8BE4F4B012281
:1034F0000220DEE406F48056FEF7AFBF4C4A089B7C
:103500001E68136823F004031360012306F4805639
:103510008AF82130FEF7A1BF0023BB2A149300F0E4
:103520009781B72A00F09081BE2A00F07A81BD2AE7
:103530007FF4E6AC4FF6FE713E4A2A48D6890690E3
:103540009089334401449181D38110F003FA01F052
:10355000D9FD10F0E7F9F8F71BFF012028F09EFBDA
:10356000B5F8D821089BFA3A00211B68A5F8D821A4
:1035700085F8DA11FEF7D7B9DFED297AF4EEE76ABC
:10358000F1EE10FA44BFDFED1C7A77EEE66A47E70A
:10359000294A127896077FF501AF284A127D042A3E
:1035A0007FF6FCAE17F0C0FA089B1B68F6E62249CE
:1035B000089B0A780B481B68069042F004020A70C8
:1035C0000A4CFEF7B0B91E4B0222032071E400BF83
:1035D000602700206427002068270020B08D00208D
:1035E000C0850020C85100206EBA0020B2510020D2
:1035F000DB0FC940E4CB1641DB0F49C0E4CB16C159
:10360000DB0FC93FDB0F494092E741B99730083CD7
:1036100015A82ABEB82200201D470020289C0020A3
:10362000DB0FC9BF70270020507600208662002083
:10363000205200203C6E002024520020A4A500202F
:10364000D46200205863002010200AF01FFE2020C2
:103650000AF004FEAD49081F22F0E2FDAC4B022245
:103660001A70AC4D95F81832002B00F02A8126888C
:10367000FEF743BD10F06EF901F044FD10F052F971
:10368000F8F786FE012028F009FB95F8D621FFF710
:10369000A1B9A14AA14B528993ED007A07EE902A75
:1036A000F8EEE77AB0EEC77AB4EEE77AF1EE10FA08
:1036B0007FF5D1AE93ED017AB0EEC77AF4EEC77A1A
:1036C000F1EE10FA7FF7C7AEB3063FF5C7AE202084
:1036D0000AF0DCFD95E80C0091490A60084641F8C3
:1036E000043F22F09DFD8A4B01221A70B9E7102099
:1036F0000AF0B4FD864B26881F700127A5E6182F17
:103700007FF4A8A800210B4616E608263346FFF7EB
:1037100005B901263346FFF701B907263346FFF7FF
:10372000FDB806263346FFF7F9B805263346FFF7FE
:10373000F5B804263346FFF7F1B87A497A4A089B70
:1037400006914FF4C8711B681180784CFEF7EBB8F6
:1037500003263346FFF7E2B802263346FFF7DEB80A
:1037600020200AF07BFD6A4B00221A7079E7CFB265
:103770008CE628F051F9FEF799B9F0EE676A43E656
:10378000F0EE667A2AE64FF4FA6102200CF0DAFDD8
:10379000644B0693089B1B68FEF7C5B80021012007
:1037A0000CF0D0FDB5F8D821089B5E491B68069146
:1037B000963AA5F8D821002285F8DA21FEF7B3B8A9
:1037C00000210846ECE7FF2100201CF062FB95F881
:1037D000D621FFF7A7BB012100201CF05AFB95F86A
:1037E000D621FFF79CBB0021FF201CF052FB95F86F
:1037F000D621FFF791BB002101201CF04AFB95F870
:10380000D621FFF786BB4A4A137A43F001031372AD
:10381000FFF79ABB464A137A23F001031372FFF7AE
:1038200093BB022188E6B0EE677AFEF79ABFF0EE0E
:10383000477AFEF780BF3B4B85F8451185F8460176
:1038400006933A4CFEF7E7BC19464FF6FE7373E653
:103850001946022370E6002C3DF477AF2D4D95F804
:10386000D531002B3DF4A2AF28F0D6F8002385F81F
:10387000D531FDF79BBF002BF0D02E492E4A0968A9
:103880004FF47A7000FB03131360E7E7172020F072
:1038900009F90CE40F200B9220F004F9DBF8140274
:1038A0000B9AF3E41B4D0BF0F7FA002385F8D531A2
:1038B000FDF77CBF0E2020F0F5F8DBF81402FFF7CF
:1038C0005CBB0127FFF797BA0B20FDF7EDBF112076
:1038D0000B9220F0E7F8DBF814020B9A40E40D207D
:1038E0000B9220F0DFF80B9ABBE410200B9220F033
:1038F000D9F8DBF814020B9A47E4002104204FE7C3
:10390000002103204CE70021022049E75449002010
:103910005C490020B8220020EC490020309A0020A9
:10392000E4240020C851002070BA0020B2510020C9
:10393000744A00203C8500206C2700200A4B30B5DB
:1039400003F1180493F900205D78072AC8BF143AE0
:10395000811804330D7313F8025C855413F8012C9D
:103960000A76A342EED130BDB824040803682DE9DD
:10397000F041DF691FB13B46BDE8F0411847002A1E
:10398000164611DD04460D460E4400E023689B6890
:10399000204698470028F9D0236815F8011B1B68BA
:1039A00020469847AE42F1D1BDE8F08100232521A1
:1039B0002422017042708370C37070471523037016
:1039C0001623C370172383713A2383703B234371FB
:1039D0003C2303727047002870B51EDB092804469B
:1039E00020DD012303EB83035B00B0FBF3F2092A24
:1039F000F8D87BB10D4EB4FBF3F00928CCBF5722A9
:103A00003022A6FB03E5024403FB1044EB0801F857
:103A1000012BF0D100230B7070BD2D230B704042A1
:103A20000131DBE7303001F8010BF3E7CDCCCCCC32
:103A3000884230B44FF001042ED301FB04F4B0FBF4
:103A4000F4F58D42F9D284B1AAB901E0B0FBF4F5E6
:103A5000092DCCBF572230222A4404FB150003F85D
:103A6000012BB4FBF1F4002CF0D100221A7030BC11
:103A70007047B0FBF4F5092DCCBF372230222A4421
:103A800004FB150003F8012BB4FBF1F4002CF0D17A
:103A900000221A7030BC70470546002AEBD1D7E7E8
:103AA0002DE9F04714461D46064600234FF47A726E
:103AB000204629462DF090F8DFF848814B4A4C4FBC
:103AC00088FB00310144C31782FB002EC3EB611158
:103AD00088FB012887FB00278644464AC3EBEE2E6D
:103AE000C1EB011C82FB0E29A0EB8C0C0744424A5F
:103AF00086F806C0C3EB27474FEAEE7C08EB010AC5
:103B0000CCEBA90C82FB07824FEAE1780CEB4C0C62
:103B1000C8EB6A18AEEBCC0EC8EB0818DFF8E8C0AB
:103B200086F804E0A1EB880171718CFB0010F91795
:103B3000C1EBE21240F2B55101FB1272C3EBE0504F
:103B4000B2F5896F4FEA80073FDA40F2DA239A42F2
:103B500043DCB2F5B77FB4BF4FF0000C4FF0010C5F
:103B60004FEA4C08254B08EB0C0103EBC1031FFA8D
:103B70008CFED88D224908EB0C0301EBC3011631F2
:103B80000B2301E031F8020D82421BDA013BF9D12F
:103B90001A4BC44403EBCC0C0123BCF81800B370DF
:103BA00007F2B2770132121ABE44F270A6F800E0B2
:103BB000204629464FF47A7200232DF00DF8328109
:103BC000BDE8F0870133DBB2E9E74FF0030EF446BE
:103BD00040F296504FF00608CCE74FF0020EF44644
:103BE00040F229404FF00408C4E700BFC5B3A291DA
:103BF00007452EC2ABAAAA2A73B06D16B8240408D2
:103C0000D024040889888888792D031103685A1CF8
:103C10000260197070472DE9F047089C2578002B49
:103C2000804689460CBF4FF0200A4FF0300A661CD0
:103C300035B3002A29DD334601E0024698B113F876
:103C4000011B501E0029F8D1971E60B13D46013D71
:103C500051464046C8476B1C002BF8DC257827EA04
:103C6000E770013055B1041B29464046C84730195A
:103C700016F8015B002DF7D1BDE8F087BDE8F087AD
:103C8000002A04DC2846BDE8F0870020EBE7571E39
:103C9000DCE783684268D0ED037A00EB83010133EF
:103CA000934281ED040A836004BF0023836000EB2C
:103CB000830393ED047A036870EE277A9A42C0ED8D
:103CC000037A77EEC77AC0ED037A0CDA013307EE98
:103CD000103AF8EEC76AB7EE007A87EEA60A0360DC
:103CE00030EE070A704707EE102AB8EEC77A87EE63
:103CF000870A704790ED057A90ED004AD0ED066A8C
:103D0000D0ED014AD0ED047A90ED035AD0ED025A7D
:103D1000A4EE007AB0EE406AB0EE470AB0EE667AE2
:103D2000A6EE247A67EEC07AA0EE457AE6EE257A12
:103D300080ED057AC0ED067A7047D0ED057A90EDFA
:103D4000013AD0ED003AD0ED064A90ED024A90EDEE
:103D5000077A90ED035A90ED086AD0ED045AC0ED51
:103D6000067AF0EE406A27EE830AC0ED056AA3EEFC
:103D7000A60A80ED087AA4EE240AA5EE470AA5EE6D
:103D8000C60A80ED070A7047D0ED007A90ED017AFF
:103D900030EE670AE7EE007AB0EE670AC0ED007A0F
:103DA000704770470A44914214D030B40139551E0F
:103DB00041F2210211F8014F082380EA0420040493
:103DC0004CBF82EA40004000013B80B2F7D18D42F7
:103DD000F0D130BC704730B50446806D6171838985
:103DE000A26823F400531B041B0C838185B0A379C4
:103DF000009213F0040230D04FF4805213F002030B
:103E0000ADF804205CD1ADF806304FF48063002299
:103E1000ADF8083011F00103ADF80C2028D1ADF851
:103E20000A3008238D07694648BFADF80A301BF0F9
:103E3000EBFDA279A36DD10724D412F0080F9A8A62
:103E40001BD122F008021204120C9A829A8992B2B3
:103E500042F400529A8105B030BD13F00203ADF870
:103E600004202AD04FF400551346ADF80650CEE793
:103E70000423ADF80A300C23D4E792B242F00802D2
:103E80009A82E3E710498B4215D0A1F548418B4255
:103E90000FD001F580618B4209D00C498B42CCD107
:103EA00005200121F5F7DCFCA279A36DC5E703200D
:103EB000F7E70220F5E70020F3E7ADF80630A6E7C4
:103EC0004FF400539FE700BF001001400014014071
:103ED00010B50446806DA160838923F400531B0450
:103EE0001B0C8381A37984B013F00402009135D0B8
:103EF0004FF4805213F00203ADF804205CD1ADF80A
:103F000006304FF480636279ADF80830D1074FF086
:103F10000003ADF80A30ADF80C3045BF0423ADF80E
:103F20000A3008230C236946920748BFADF80A30CF
:103F30001BF06AFDA279A36DD1071FD412F0080F00
:103F40009A8A16D122F008021204120C9A829A89D7
:103F500092B242F400529A8104B010BD13F00203F1
:103F6000ADF8042025D04FF400511346ADF80610EB
:103F7000C9E792B242F008029A82E8E710498B4200
:103F800015D0A1F548418B420FD001F580618B42DD
:103F900009D00C498B42D1D105200121F5F760FCF5
:103FA000A279A36DCAE70320F7E70220F5E7002016
:103FB000F3E7ADF80630A6E74FF400539FE700BFE4
:103FC0000010014000140140002328220360027009
:103FD0002922C2700122436083608271437270475C
:103FE000F8B50468C4F30D0405460E4604B32F6803
:103FF0001BF042FE092840F08880454C236923F4D9
:1040000040732361236943F400732361236943F000
:10401000010323613E601BF02FFE2369092823F072
:104020000103236171D12B6804332B600020F8BD9C
:10403000384B394A93422BD902F58042934226D914
:1040400002F5804293422AD902F58042934228D950
:1040500002F58032934226D902F50032934224D9E8
:1040600002F50032934222D902F50032934220D960
:1040700002F5003293421ED902F5802293421CD9E8
:10408000B3F1016F1BD30520F7F7B2FFFBE708245C
:104090001BF0F2FD092814D04FF0FF30F8BD1024BA
:1040A000F6E71824F4E72024F2E72824F0E7302488
:1040B000EEE73824ECE74024EAE74824E8E7582410
:1040C000E6E7134F3B6923F440733B613B6943F4DC
:1040D00000733B613B6923F0F8033B613B6943F0AC
:1040E00002031C433C613B6943F480333B611BF09A
:1040F000C3FD3B6923F002033B613B69092823F0C0
:10410000F8033B613FF473AFC6E76FF00100F8BD01
:10411000003C024000400008FF3F0008F8B504469C
:104120000D468E180027B54201D12069F8BDE3681D
:10413000591CE160234415F8012B1A720429F2D1AD
:10414000206918B9A1682046FFF74AFF2061E7609F
:10415000E9E703685B6A03B11847704703681B6AA5
:1041600003B11847704703682DE9F041DF691FB1BB
:104170003B46BDE8F0411847002A164611DD0446CB
:104180000D460E4400E023689B68204698470028AF
:10419000F9D0236815F8011B1B6820469847AE42EA
:1041A000F1D1BDE8F08103689B69184703685B693A
:1041B000184703681B6918470368DB6818470368DA
:1041C0009B68184703685B68184703681B681847B3
:1041D000014B1868F9E700BFA41F002038B50C4652
:1041E000097849B1054601342B6828461B68984771
:1041F00014F8011B0029F7D138BD064B53F82030C5
:104200002BB11A689B8851690B4201D11383704707
:10421000538370470885002003682DE9F04F03F1B0
:104220003F4404F57E04604EA40A0125345D04F089
:104230001F066409032C05FA06F500F0AF80042C74
:1042400000F0A780022C54D08588B5FA85F0C0F123
:104250001F0080B2C40803EB840400F00700266A44
:1042600080000F27874026EA07062662276A01F0AA
:10427000030602FA00F0721E3843012AC1F3810CD2
:10428000C1F300182062C1F3411137D9002422463E
:1042900001274FF0030E03E0102A04F1020426D098
:1042A00007FA02F0A84302F10102F5D1D3F800C0E9
:1042B0000EFA04F0C04300EA0C0CC3F800C0D3F8B7
:1042C000008006FA04FC4CEA080CC3F800C0D3F8DE
:1042D0000CC000EA0C00D860D3F80CC001FA04F05E
:1042E00040EA0C00102AD86004F10204D8D1BDE8DD
:1042F000F08F2E4C666C35436564A5E700200246BE
:104300004FF0010E4FF0030904E00132102A00F1D2
:1043100002003CD00EFA02F737EA0504F5D1D3F8D3
:1043200000A009FA00F4E4430AEA040AC3F800A072
:10433000D3F800B006FA00FA4AEA0B0AC3F800A064
:10434000D3F808A004EA0A0AC3F808A0D3F808B012
:104350000CFA00FA4AEA0B0AC3F808A0D3F804A042
:104360002AEA07075F60D3F804A008FA02F747EAD1
:104370000A075F60DF683C40DC60DF6801FA00F438
:1043800001323C43102ADC6000F10200C2D1BDE8DA
:10439000F08F064C266B3543256355E7034C266C9E
:1043A0003543256450E700BFB84F04080038024089
:1043B000026802F13F4303F57E032DE9F04F9B0AAB
:1043C000544DEB5C03F01F055B090124032B04FA39
:1043D00005F400F09980042B00F09180022B3ED070
:1043E00001F00306731E012BC1F3810CC1F3001809
:1043F0008588C1F3411137D90024234601274FF0A6
:10440000030E03E0102B04F1020426D007FA03F098
:10441000A84303F10103F5D1D2F800C00EFA04F06D
:10442000C04300EA0C0CC2F800C0D2F8008006FAC3
:1044300004FC4CEA080CC2F800C0D2F80CC000EA38
:104440000C00D060D2F80CC001FA04F040EA0C0075
:10445000102BD06004F10204D8D1BDE8F08F2E4BB0
:104460005D6C2C435C64BBE7002003464FF0010EFB
:104470004FF0030904E00133102B00F102003CD09F
:104480000EFA03F737EA0504F5D1D2F800A009FACD
:1044900000F4E4430AEA040AC2F800A0D2F800B02B
:1044A00006FA00FA4AEA0B0AC2F800A0D2F808A0FD
:1044B00004EA0A0AC2F808A0D2F808B00CFA00FA16
:1044C0004AEA0B0AC2F808A0D2F804A02AEA0707B1
:1044D0005760D2F804A008FA03F747EA0A075760C2
:1044E000D7683C40D460D76801FA00F401333C43FC
:1044F000102BD46000F10200C2D1BDE8F08F064B52
:104500001D6B2C431C636BE7034B1D6C2C431C641D
:1045100066E700BFB84F04080038024010B5040930
:10452000013C032C17D80D4B33F8142000F00F007A
:1045300042FA00F313F001030DD0012303FA00F057
:10454000013810402CF098FB054A064B125D1044D0
:1045500003EBC00010BD002010BD00BF2C510408AB
:10456000285104087C8300202DE9F04F4A484B492C
:104570004B4B4C4C4FF0010A4FF002094FF004082E
:104580004FF0080C4FF0100E20274026802530F801
:10459000022B12F0010F03D01960A3F804A0083316
:1045A00012F0020F03D01960A3F80490083312F040
:1045B000040F03D01960A3F80480083312F0080F29
:1045C00003D01960A3F804C0083312F0100F03D011
:1045D0001960A3F804E0083312F0200F02D019602C
:1045E0009F80083312F0400F02D019609E8008337C
:1045F00012F0800F02D019609D80083312F4807F82
:1046000005D04FF4807B1960A3F804B0083312F48E
:10461000007F05D04FF4007B1960A3F804B0083385
:1046200012F4806F05D04FF4806B1960A3F804B0CA
:10463000083312F4006F05D04FF4006B1960A3F833
:1046400004B0083312F4805F05D04FF4805B19602A
:10465000A3F804B0083312F4005F05D04FF4005BF8
:104660001960A3F804B0083312F4804F05D04FF45A
:10467000804B1960A3F804B00833D20B04D04FF478
:10468000004219609A80083301F58061A1427FF4ED
:104690007EAFBDE8F08F00BF2C510408000002403F
:1046A0007C8300200010024000286AD003682DE9B6
:1046B000F04F03F13F4404F57E045F4EA40A012548
:1046C000345D04F01F066409032C05FA06F559D081
:1046D000042C00F0AC80022C59D08588B5FA85F006
:1046E000C0F11F0080B2C40803EB840400F007008F
:1046F000266A80000F27874026EA07062662276A77
:1047000001F003068240701E3A430128C1F3810C78
:10471000C1F300182262C1F341113DD900242246A1
:1047200001274FF0030E03E0102A04F1020426D003
:1047300007FA02F0A84302F10102F5D1D3F800C054
:104740000EFA04F0C04300EA0C0CC3F800C0D3F822
:10475000008006FA04FC4CEA080CC3F800C0D3F849
:104760000CC000EA0C00D860D3F80CC001FA04F0C9
:1047700040EA0C00102AD86004F10204D8D1BDE848
:10478000F08F70472D4C266C35432564A5E72B4CE4
:10479000666C35436564A0E7002002464FF0010EC9
:1047A0004FF0030904E00132102A00F102003CD06E
:1047B0000EFA02F737EA0504F5D1D3F800A009FA9A
:1047C00000F4E4430AEA040AC3F800A0D3F800B0F6
:1047D00006FA00FA4AEA0B0AC3F800A0D3F808A0C8
:1047E00004EA0A0AC3F808A0D3F808B00CFA00FAE1
:1047F0004AEA0B0AC3F808A0D3F804A02AEA07077C
:104800005F60D3F804A008FA02F747EA0A075F607E
:10481000DF683C40DC60DF6801FA00F401323C43B1
:10482000102ADC6000F10200C2D1BDE8F08F034C19
:10483000266B3543256350E7B84F04080038024023
:10484000002855D0026802F13F4303F57E032DE9AD
:10485000F04F9B0A544DEB5C03F01F055B090124EC
:10486000032B04FA05F444D0042B00F09780022BAC
:1048700044D001F00306731E012BC1F3810CC1F378
:1048800000188588C1F341113DD900242346012732
:104890004FF0030E03E0102B04F1020426D007FAB8
:1048A00003F0A84303F10103F5D1D2F800C00EFADA
:1048B00004F0C04300EA0C0CC2F800C0D2F800803B
:1048C00006FA04FC4CEA080CC2F800C0D2F80CC08E
:1048D00000EA0C00D060D2F80CC001FA04F040EA03
:1048E0000C00102BD06004F10204D8D1BDE8F08F89
:1048F00070472E4B1D6C2C431C64BAE72B4B5D6C30
:104900002C435C64B5E7002003464FF0010E4FF0E6
:10491000030904E00133102B00F102003CD00EFA31
:1049200003F737EA0504F5D1D2F800A009FA00F43C
:10493000E4430AEA040AC2F800A0D2F800B006FA7A
:1049400000FA4AEA0B0AC2F800A0D2F808A004EA6A
:104950000A0AC2F808A0D2F808B00CFA00FA4AEA2B
:104960000B0AC2F808A0D2F804A02AEA0707576089
:10497000D2F804A008FA03F747EA0A075760D76895
:104980003C40D460D76801FA00F401333C43102B5B
:10499000D46000F10200C2D1BDE8F08F034B1D6B63
:1049A0002C431C6365E700BFB84F04080038024081
:1049B00010B1036882885A83704710B103688288F7
:1049C0001A83704718B10368828809B95A837047FF
:1049D0001A83704710B40A4B0A4A1C78012383409B
:1049E000234052F8200029B9B3FA83F149095DF850
:1049F000044BE7E7191C18BF01215DF8044BE1E700
:104A0000048500200885002030B1036882881B6976
:104A10001A4214BF0120002070472DE9F0410B4ECF
:104A2000346873691C400FD0DFF824800127B4FA82
:104A300084F3C3F11F0307FA03F558F82300036852
:104A40009847AC437561F2D1BDE8F081003C01406C
:104A5000448500202DE9F0410B4E346873691C40F9
:104A60000FD0DFF828800127B4FA84F3C3F11F03C5
:104A700007FA03F558F8230003689847AC437561BB
:104A8000F2D1BDE8F08100BF003C01404485002028
:104A90002DE9F0410B4E346873691C400FD0DFF8EC
:104AA00028800127B4FA84F3C3F11F0307FA03F542
:104AB00058F8230003689847AC437561F2D1BDE80C
:104AC000F08100BF003C0140448500202DE9F04109
:104AD0000B4E346873691C400FD0DFF82880012723
:104AE000B4FA84F3C3F11F0307FA03F558F823005F
:104AF00003689847AC437561F2D1BDE8F08100BF0F
:104B0000003C0140448500202DE9F0410B4E346803
:104B100073691C400FD0DFF828800127B4FA84F3B2
:104B2000C3F11F0307FA03F558F8230003689847F9
:104B3000AC437561F2D1BDE8F08100BF003C01409B
:104B4000448500202DE9F0410B4E346873691C4008
:104B50000FD0DFF828800127B4FA84F3C3F11F03D4
:104B600007FA03F558F8230003689847AC437561CA
:104B7000F2D1BDE8F08100BF003C01404485002037
:104B80002DE9F0410B4E346873691C400FD0DFF8FB
:104B900028800127B4FA84F3C3F11F0307FA03F551
:104BA00058F8230003689847AC437561F2D1BDE81B
:104BB000F08100BF003C014044850020084A0948BC
:104BC00008B5536C43F480435364002140222DF018
:104BD00094FB054B4FF0FF321A60C3F8032008BD69
:104BE00000380240448500208485002003685B6A09
:104BF00018472DE9F041044618460D4616469846DA
:104C00002BF040FB2768E6722844A07229467D6994
:104C1000434632462046AC46BDE8F0416047036853
:104C200010B504461B689847236820469B68984740
:104C3000A37B0133A37310BD10B5036804469B68C2
:104C40009847FF2301226373227310BD08B5FFF755
:104C500065FC38B12D2282710022C2712021BDE88D
:104C60000840EDE508BD0B4B984206D0A3F5744310
:104C700098420DD04FF0FF3070470022064B03EBF7
:104C800002135A89013292B25A81588980B2704710
:104C90000222F3E700300140606F002070B58368A6
:104CA0000446164613B11A689B885383606840F225
:104CB000E93301E0002B30D00589013B15F0020FEC
:104CC0009BB2F7D089B2818140F2E93300E023B38F
:104CD0000289013B12F0010F9BB2F8D0838940F2A8
:104CE000E93300E0EBB10189013B11F0020F9BB207
:104CF000F8D0B6B2868140F2E93300E08BB1028988
:104D0000013B12F0010F9BB2F8D08389A36813B165
:104D10001A689B881383012070BDFFF7A4FF6068A9
:104D2000DDE7FFF7A0FFF1E72DE9F0410678012E5E
:104D300082B005464CD0022E52D1806841F08001ED
:104D400010B1046880886083686840F2E93402E04A
:104D5000002C00F099800689013C16F0020FA4B2E5
:104D6000F6D089B2818140F2E93102E0002900F0F9
:104D70008B800489013914F0010F89B2F6D0818942
:104D800081894FF0000C4FF47A714FF6FF764FF0A7
:104D9000FF0E634502D129E0B14225D004890139D3
:104DA000A70789B2F8D5A0F80CE04FF47A7102E0B9
:104DB000B9B2B14218D00489E40701F1FF37F7D541
:104DC0008489A4B20AB1147001320CF1010CE0E73D
:104DD00090F904E0BEF1FF3F02D0BEF1030F0FDDFA
:104DE000002002B0BDE8F081FFF73DFFAB68002B6B
:104DF0005CD01A689B881383012002B0BDE8F08163
:104E00004FEACE08DFF8ACC008EB0E070CEB8707C3
:104E100078680028E5D06C793A6264000025E4B235
:104E2000BC75F9757D76BE763B767E753D7583885B
:104E3000FA61990514D40388DA050CD44FF4805430
:104E400001E0013C28D003889B05FAD403889BB27B
:104E500043F48073038083889BB243F44073838060
:104E6000F0440CEB88024FF4805401E0013C13D075
:104E7000537D002BFAD10CEB880898F8144084F08D
:104E8000010002B0BDE8F0818DE80C00FFF7EBFEF9
:104E900068689DE80C0073E7054A13880133704683
:104EA0009BB21380F5F752FA20469AE7012098E763
:104EB0007C420020B43A002030B40578012D08D09F
:104EC000022D03D101F07F0130BCE7E6002030BCA9
:104ED0007047134630BC0A46417990F90400F5F753
:104EE0000FBC427A02B9704710B5044603684068A7
:104EF00004F10A0198470023637210BD437A5A1CDB
:104F00000344D2B242729972037A934200D802B932
:104F1000704710B504460368406804F10A019847D9
:104F20000023637210BD50B30123302803FA01F14E
:104F300022D0312820D032281ED033281CD034284B
:104F40001ED035281CD020281AD0212818D010288F
:104F500012D0112810D012280ED013280CD01428EB
:104F60000ED015280CD0162801D0172806D111F024
:104F7000030018BF012070474A0703D10020704783
:104F80008B07FBD001207047302829D0312829D049
:104F9000322829D0332829D0342829D0352829D0BF
:104FA000202829D0212829D0102829D0112829D01B
:104FB000122829D0132829D0142829D0152829D01F
:104FC000162805D0172808BF0F2302D000207047ED
:104FD0000E23114A03EB4303134493F87A007047FE
:104FE0000023F6E70123F4E70223F2E70323F0E7C7
:104FF0000423EEE70523ECE70623EAE70723E8E7C7
:105000000823E6E70923E4E70A23E2E70B23E0E7C6
:105010000C23DEE70D23DCE7B824040870B54488D0
:1050200006460D46C4F30B042246002128462DF007
:1050300064F93369094A934209D3094A934206D273
:10504000224628461946BDE870402CF059B823B1D5
:1050500021462846BDE87040184770BD400600084C
:1050600040070008064B07498B4202D3002318462D
:1050700070471A88C2F30B029042F8D01433F3E75A
:105080009001000840060008024A136823EA000065
:10509000106070476C630020F8B5174D2B78A52B76
:1050A00028D16B78BE2B25D1022229464FF6FF70FE
:1050B000FEF778FE114FAC1C22884AB1A618BE42FA
:1050C00018D2052A16D92146FEF76CFE3446F3E7BE
:1050D00021460222FEF766FE0222A118FEF762FEBA
:1050E0000634074B641B1C8041F60F53C31A584209
:1050F0005841F8BD0020F8BD0040000800800008BD
:105100007E4200202DE9F04FDFF84C914D4F8BB0DF
:105110000326A7EB09071822002104A82DF0EDF8BB
:10512000494BCDF8109005971A69002A04DA474ACE
:105130005A6002F188325A6001228DF82420F3224D
:10514000DA60434B434C1B88ADF8003002226946BD
:1051500004A8FEF7E3FF022269464FF6FF70FEF750
:1051600021FEDFF8F8A080464FF0000B544539D3FC
:105170000AAC002524F8245D0222214604A8FEF78B
:10518000CDFF022221464046FEF70CFE40BAC04346
:10519000ADF80800022202A904A8FEF7BFFF079895
:1051A00078B106ABC0F10402294618442DF0A5F8E9
:1051B000089818B9069904A8FEF712FF0023089072
:1051C00007939DF82430089A23B11F490B6943F0D7
:1051D00000430B61013E2DD0002A9CD1FFF75CFFFC
:1051E00050B32CE065888DF80DB0C5F30B05AB1DF1
:1051F000ADF808302388C3F30B02ADF80A201B0B6F
:10520000062202A904A88DF80C30FEF787FF0622BB
:1052100002A94046FEF7C6FD616880462A4604A8FA
:10522000FEF77CFF616840462A46FEF7BBFD14345A
:1052300080469BE7002AD1D00520F6F7D9FE0BB0B7
:10524000BDE8F08F00800008003C02402301674564
:10525000602504089001000800400008400600088E
:105260000378202B024600F10100F9D0092BF7D07A
:105270002D2B2CD02B2B03BF5378B7EE000A024600
:10528000B7EE000AA3F13001C8B209289FED467AB3
:1052900010D8F2EE046A07EE901AF8EEE77A12F8E8
:1052A000013FE7EE267AA3F13001C8B20928B0EE3B
:1052B000677AF0D92E2B4CD003F0DF03452B0BD0AF
:1052C000F7EE007A67EE276A20EE260A70475378D9
:1052D000BFEE000A0246D5E710B451782D2959D007
:1052E0002B290ABF9178501C901C0024A1F1300397
:1052F000092B53D8002303EB830301EB430310F87E
:10530000011FA1F13002092AA3F13003F3D9B3F54B
:105310009A7F28BF4FF49A73072B42D9DFED236A97
:105320001A46F7EE007A083A072A67EEA67AFAD804
:1053300003F007032BB1F2EE046A013B67EEA67A95
:10534000FBD124B3C7EE276A5DF8044B20EE260A92
:1053500070475378A3F13001C8B2092802F1010265
:10536000AAD8F2EE046AF0EE665A07EE901AF8EE4A
:10537000E77A12F8013F87EEA66AA3F13001C8B2BE
:10538000092866EEA56A37EE067AEED994E767EE4D
:10539000276AD9E7901C91780124A7E7F7EE007AF5
:1053A000CFE7F7EE007AC5E70000000020BCBE4C56
:1053B000B5EEC00ADFED317AF1EE10FACCBF30EE77
:1053C000270A30EE670ADFED2E7A20EE270A30B585
:1053D000FDEEC07A87B017EE904A054684EAE47085
:1053E000002303A9A0EBE47001930093029329F03A
:1053F000F8FE002CACBF20232D2303A88DF800302D
:105400002AF040FF012803A924D002282DD0032828
:1054100005BF3023684668468DF801302CF075FFD3
:1054200068462AF02FFF0338C4B222466946284650
:105430002CF0A2FF00232B5528462AF023FF2E2212
:10544000431C2A540DEB0401E8182CF07BFF28467E
:1054500007B030BD302368468DF801308DF802303A
:105460008DF803302CF051FFDAE7302368468DF8D1
:1054700001308DF802302CF048FFD1E76F12033A6B
:1054800000007A442DE9F041064615460846B6FB71
:10549000F2F43CB905FB1464124B1B5D00F8013BB0
:1054A000BDE8F081B4FBF2F767B90E4B05FB174777
:1054B00005FB1464DA5D00F8012B1B5D00F8013B6D
:1054C000BDE8F081B7FBF2F8B8F1000F02D040461A
:1054D000FFF7D8FF05FB1878024B13F8082000F8F7
:1054E000012BE3E7F85B0408104B2DE93048D3E9C2
:1054F000004554EA05020BD1034601220020187131
:10550000587198719A70DA7018801881BDE83088E7
:10551000074B1A6814EB020B45F1000C5A46634620
:10552000FEF7BEFA0120BDE8308800BFF824002055
:105530003C850020F0B402888578164FC378047942
:105540004179A2F2B27202F0030606EB4606013D73
:1055500005EB860507EB4505013B2E8B8579008918
:1055600040F2B557920807FB0232931903EB43034D
:1055700004EBC303C3EB031301EB8303C3EB03137C
:1055800005EB830300214FF47A72C2FB0301F0BCE8
:10559000704700BFB8240408FAB170B48E180446EE
:1055A00003E0101A14D1B14214D014F8012BA2F167
:1055B0004103192B11F8013BA3F1410598BF20329B
:1055C000192D03F12000ECD9D01A01D1002BEAD11A
:1055D00070BC7047002070BC7047104670474FF099
:1055E000FF32FFF7D9BFA0F16103192B98BF203814
:1055F0007047A0F14103192B98BF20307047202835
:1056000005D0093804288CBF0020012070470120F4
:105610007047613819288CBF00200120704741383D
:1056200019288CBF002001207047303809288CBF12
:10563000002001207047A0F13003092B07D920F08A
:105640002000413819288CBF00200120704701201C
:10565000704730B402681146531C036011F8024BC6
:105660000160D31C517803609378151D05601B04FD
:1056700043EA0123D078234343EA006030BC7047FB
:105680000368591C1A46016012F8021B0260587820
:1056900041EA0020704703685A1C0260187870477E
:1056A00038B50446006815462BF02AFD22682A44C6
:1056B000226038BD036810B40A0E5C1C04601A70C6
:1056C00003680A0C5C1C04601A7003680A0A5C1CFC
:1056D00004601A7003685A1C026019705DF8044B6C
:1056E0007047036810B40A0A5C1C04601A700368EF
:1056F0005A1C026019705DF8044B704703685A1C0D
:10570000026010B4197003680A0A5C1C04601A7005
:1057100003680A0C5C1C04601A700368090E5A1CAA
:10572000026019705DF8044B704703685A1C0260F0
:1057300019700368090A5A1C0260197070472DE934
:10574000F047002488B080460F461E46A14605ADAE
:10575000531C0393117839B3252933D1931CCDF809
:1057600010900393507830284ED04FF0000AA0F1EB
:105770003003DBB2092B42D96C2819D0642800F021
:10578000938024D825281CD063D9582876D0632844
:105790001BD131784046B847039A531C03931178C4
:1057A000043601340029D7D1204608B0BDE8F0877F
:1057B000039B5A1C03921B78642B7CD02AD8252B80
:1057C00054D1252140460134B847039AC0E77328D5
:1057D00033D044D975284FD106F1040E30682B46DA
:1057E00000220A217646FEF723F9049A00955346D3
:1057F00039464046FEF70FFA039A0444A8E704AA84
:1058000003A929F0CBFCB7E7D31C039390784FF0A2
:10581000010AACE7732B10D05BD9752B3AD0782BEB
:1058200096D1A3F15802B2FA82F2306852092B469F
:1058300010210436FEF7FCF8D7E73368049A00938A
:10584000394600234046FEF7E6F904360444039A3D
:105850007EE70028B9D1204608B0BDE8F0876E2861
:10586000B3D1039A336804361C6071E72AD9582BE8
:10587000D7D0632B8DD06BE77828A6D1A0F1580242
:10588000B2FA82F2306852092B461021FEF7D0F8A6
:105890000436AAE706F1040E30682B4600220A21DE
:1058A0007646FEF7C5F8A0E7331D306829461E4648
:1058B000FEF791F899E7331D306829461E46FEF73A
:1058C0008AF892E7002B7FF443AF204608B0BDE88A
:1058D000F0876E2BC6D03BE70EB400B584B005ABA5
:1058E000019053F8042B0649039301A8FFF727FF03
:1058F000019B00221A7004B05DF804EB03B07047FE
:105900000D3C01082DE9F047484BB3F900708CB00D
:105910000646002F56D13D463C460A8840F2B173F8
:105920009A4203D98B78581E0B282FD900230120C7
:105930001946ADF824308DF828308DF829308DF8CF
:105940002A30ADF82C309C469A4699461A4698461D
:1059500086468DF826008DF827000346002CACBF44
:105960002B242D24049107950697CDF80CC0CDF873
:1059700008A0CDF80490CDF800E0304605942C49FD
:10598000FFF7AAFF40460CB0BDE8F08791F803E0AE
:105990000EF1FF301E28C9D891F80490B9F1170F05
:1059A000C4D891F805A0BAF13B0FBFD891F806C052
:1059B000BCF13B0FBAD80989B1F57A7FB6D24FF066
:1059C0000108CBE71B4C84FB0734E319FC17C4EB3D
:1059D0006314C4EB0415A7EB85052DB2002D084612
:1059E000B8BF6D42FFF7A6FD4FF47A7200238046E0
:1059F00089462BF0F1F83C2307FB03074FF47A723A
:105A00000023404649462BF0E7F824B24FF47A7160
:105A100092B20023C1FB072309A884EAE477FEF7CA
:105A20003FF8A7EBE47709A977E700BFD42400206B
:105A3000205C0408898888880FB430B583B006AB31
:105A40000A490B4853F8042B096800680193FFF7D3
:105A500076FE084C05462068FEF7A8FB0028FAD021
:105A6000284603B0BDE8304004B07047783A0020C3
:105A70007C3A0020A41F0020DFED2B7AB4EEE70A69
:105A8000F1EE10FA4ADDDFED296A9FED297A01E097
:105A9000B0EE670AB4EEC70AF1EE10FA70EE667A5D
:105AA000F6DC9FED247AF4EEC77AF1EE10FA38D5E1
:105AB000DFED1E6A9FED207A01E0F0EE407AF4EE11
:105AC000C77AF1EE10FA37EEA60AF6D4DFED1B7AAC
:105AD000B4EEE70AF1EE10FA14DDDFED137A37EEDB
:105AE000C00A60EE006A9FED166A9FED167ADFED40
:105AF000167AA6EE867A20EE266AE6EE877AA6EE7B
:105B0000270A7047DFED117AB4EEE70AF1EE10FADA
:105B100044BFDFED087A37EEC00AE2E7F0EE407AE4
:105B2000BFE7B0EE670AD1E7DB0F4940DB0FC940A2
:105B3000E4CB1641DB0F49C0E4CB16C1DB0FC93FF4
:105B400092E741B99730083C15A82ABEDB0FC9BFC0
:105B500080EAE073A3EBE0738B4205DB002801DDF4
:105B6000401A704702D170470020704708447047C0
:105B700009B909E0194690FBF1F301FB130308464C
:105B8000002BF7D1084670470146FBE7F0EEC07ADC
:105B9000B0EEE07AB4EEE77AF1EE10FAB4BFB0EE10
:105BA000676AB0EE476AB5EE406AF1EE10FA46D089
:105BB000B4EEE77AF1EE10FA8CBFF0EE675AF0EE31
:105BC000475AC5EE866A9FED1F3A9FED1F6A9FED0B
:105BD0001F4A9FED1F5ADFED1F3ADFED1F4ADFED31
:105BE0001F5AA6EEC36AE6EEA34AA6EE864AB7EEB1
:105BF000006AA6EE845AA6EEA46AE6EE855AC5EEC1
:105C0000866AB4EEE77AF1EE10FA48BFDFED147A57
:105C1000F5EEC00A48BF77EEE66AF1EE10FA48BF2B
:105C2000DFED107AB5EEC00A48BF77EEE66AF1EE16
:105C300010FA48BFF1EE666AB0EE660A7047DFED13
:105C4000076ADEE739094E3DE3B59E3E88FA163E07
:105C500045FE7F3F99FB243F69A2163EA7DFA8348B
:105C6000DB0FC93FDB0F4940DFED317A30EE277A99
:105C7000FDEEC76A16EE903A2033402B02D99FED15
:105C80002D0A7047B4EEE70AF1EE10FA4DDD9FEDF4
:105C90002A6ADFED2A6A01E0B0EE677AB4EEE67AAE
:105CA000F1EE10FA77EE467AF6DC9FED257AF4EE07
:105CB000C77AF1EE10FA35D5DFED1F6A9FED217A34
:105CC00001E0F0EE407AF4EEC77AF1EE10FA37EE2A
:105CD000A60AF6D4DFED167AB4EEE70AF1EE10FA72
:105CE0001BDCDFED197AB4EEE70AF1EE10FA44BFDF
:105CF000DFED137A37EEC00A60EE006A9FED136A9B
:105D00009FED137ADFED137AA6EE867A20EE266AEF
:105D1000E6EE877AA6EE270A7047DFED0F7A37EEB8
:105D2000C00AE9E7B0EE670AD4E7F0EE477ABCE7CD
:105D3000DB0FC93F00000000DB0FC940E4CB164178
:105D4000DB0F49C0E4CB16C1DB0FC9BF92E741B9F5
:105D50009730083C15A82ABEDB0F4940FDEEC07AFB
:105D600017EE903A2033402B51D8DFED2D7AB4EE68
:105D7000E70AF1EE10FA50DDDFED2A6A9FED2A7A8C
:105D800001E0B0EE670AB4EEC70AF1EE10FA70EE69
:105D9000667AF6DC9FED257AF4EEC77AF1EE10FA1A
:105DA00038D5DFED206A9FED227A01E0F0EE407AEF
:105DB000F4EEC77AF1EE10FA37EEA60AF6D4DFED6C
:105DC0001D7AB4EEE70AF1EE10FA1BDCDFED1A7A69
:105DD000B4EEE70AF1EE10FA44BFDFED147A37EEC5
:105DE000C00A60EE006A9FED156A9FED157ADFED3F
:105DF000157AA6EE867A20EE266AE6EE877AA6EE79
:105E0000270A7047DFED067A37EEC00AE9E79FED13
:105E10000E0A7047B0EE670AD1E7F0EE407AB9E7B4
:105E2000DB0F4940DB0FC940E4CB1641DB0F49C013
:105E3000E4CB16C1DB0FC93FDB0FC9BF92E741B905
:105E40009730083C15A82ABE0000000007EE901A03
:105E5000F8EE677A9FED837A27EE800A20EE070A34
:105E6000FDEEC07A17EE903A2033402B00F28C8082
:105E7000DFED7D7AB4EEE70AF1EE10FA40F3E88048
:105E8000B0EE407A9FED796ADFED796A01E0B0EE1D
:105E9000677AB4EEE67AF1EE10FA77EE467AF6DC3F
:105EA0009FED747AF4EEC77AF1EE10FA40F1CD80EE
:105EB0009FED6E6ADFED706A01E0F0EE477AF4EE76
:105EC000E67AF1EE10FA37EE867AF6D4DFED6B7AE9
:105ED000B4EEE77AF1EE10FA51DCDFED697AB4EE58
:105EE000E77AF1EE10FA44BFDFED627A37EEC77A57
:105EF00027EE076ADFED635ADFED637ADFED636A51
:105F00009FED635AE6EE257A67EE065AE6EE276ABB
:105F1000F7EE007AA5EEA67AF0EE675AE7EE055A9C
:105F2000E7EE457A87EEA55ADFED547A30EE277A10
:105F3000FDEEC76A16EE903A2033402B29D99FED2B
:105F4000557AF6EE006AB7EE006AF7EE004AC4EE44
:105F5000A57A0023836143610362C36180ED045A23
:105F600067EEA66A27EE866A27EE877AC0ED006A9A
:105F7000C0ED026A80ED016A80ED037A7047DFEDC3
:105F80003A7A37EEC77AB3E7B7EE005AF0EE455AE1
:105F9000CAE7B4EEE70AF1EE10FA5FDD9FED336A6F
:105FA000DFED336A01E0B0EE677AB4EEE67AF1EE47
:105FB00010FA77EE467AF6DC9FED2E7AF4EEC77A89
:105FC000F1EE10FA47D59FED296ADFED2B6A01E06B
:105FD000F0EE477AF4EEE67AF1EE10FA37EE867AD2
:105FE000F6D4DFED267AB4EEE77AF1EE10FA27DC8C
:105FF000DFED237AB4EEE77AF1EE10FA44BFDFED7D
:106000001D7A37EEC77A27EE076ADFED1E4ADFED0D
:106010001E6ADFED1E7AE6EE246A67EE064AE6EEB9
:10602000267AB7EE006AA4EEA77AF6EE006A36EE9C
:10603000476AF8EE007A27EE277A66EE266A84E74A
:10604000DFED097A37EEC77ADDE7B0EE677A3DE734
:10605000F0EE407A24E7B0EE677AC2E7F0EE477AD6
:10606000AAE700BF27D4D236DB0F4940DB0FC94077
:10607000E4CB1641DB0F49C0E4CB16C1DB0FC93FAF
:10608000DB0FC9BF92E741B99730083C15A82ABE7B
:10609000F304353F0000008070B406688E4217D9C3
:1060A0000139751E002311F8014F0822634013F0D7
:1060B000800F4FEA430318BF83F0D503013ADBB2E8
:1060C000F5D18D42EFD1721C0260337070BC704705
:1060D0000023F8E710B44C09012250F8243001F0F5
:1060E0001F0102FA01F10B4340F824305DF8044B24
:1060F00070474B0901F01F0150F82320012303FAD8
:1061000001F1114214BF18460020704770B5104DC0
:10611000104E2B7831788B4284B016D00E4A039201
:106120001A4402928CBF0C46CA1A04A98CBFC3F150
:1061300080020024012341F8102D02A802220194BC
:10614000F3F7DAFE002333702B7004B070BD00BF8C
:106150001D640020A064002020640020F0B5124BD4
:106160009D6885B00DB905B0F0BDED0A14D00027CB
:1061700004AE7C196410E00210226946F3F7C6FFF2
:106180000F2809DD6B4653F8042B01320AD1B342C4
:10619000F9D12546AF42ECDBFFF7B8FF034BED0228
:1061A0001D60E0E7671CF5E7A01A0020686E00207C
:1061B00070B5194C194D23782978994284B027D0AD
:1061C000174A03921A44029234BF0E46CA1A04A90F
:1061D00034BFC3F180020026002341F8102D02A82D
:1061E00002220196F3F788FE23781844C0B2030612
:1061F0002B7848BF80F080008342207002D00020BE
:1062000004B070BD002301202B70237004B070BD5A
:10621000012004B070BD00BF1D640020A0640020F8
:1062200020640020074A084B10781B78074A8342F5
:1062300096BFC31AC3F180030020126818441044AB
:10624000704700BFA06400201D640020686E00201D
:106250002DE9F04F95B0B0F908500D81EDB2442D05
:1062600000AF0C46904600F03082064643D9812D9F
:1062700000F0718200F29880542D00F0CC8040F242
:10628000BD816E2D00F0EF81802D40F0D080AA4BB3
:1062900093F800A00AF1020A1AF0FF0A00F09780B2
:1062A000A64BDFF8D482A64EDFF8D0B29A4403F1B1
:1062B00001090A2516E0322D00F00883A5F13C0003
:1062C000C0B2132840F2088300232268511C2160C9
:1062D00015702268CA4502F101012160137076D061
:1062E00019F8015B0A2DE6D1BBF80030FF2BA8BFDF
:1062F000FF23DBB2E9E7052D00F0D58120D8022D80
:1063000000F0818040F26781032D00F0A381042D0D
:1063100040F08D808B4920462A46FFF7C1F90021C5
:106320002046FFF702FA22680021531C0125236052
:1063300028462B46543711706381BD46BDE8F08F67
:10634000242D5ED040F2D980282D00F0C681382D52
:106350006DD10A687C4B0125511C216015702268A3
:10636000052150192060117022680A2150192060FF
:10637000117022680021501920601170226819786C
:1063800050192060117022685978501920601170DE
:1063900022689978531923602B4611702846543788
:1063A0006381BD46BDE8F08FA02D18D040F2E88093
:1063B000B82D00F0CE81FE2D39D1644D05F10806CF
:1063C00035F8021B2046FFF7B0F9B542F8D1012598
:1063D0002B46284654376381BD46BDE8F08F5C4BA1
:1063E00008461968FFF78AF95A4B20461968FFF7E3
:1063F00085F9594B196820460125FFF77FF92B468F
:10640000E7E7564BF6E70422554920460125FFF7FA
:1064100047F92B46C2E70B6800215A1C226019700D
:1064200022680125531923602B461170B6E72146D7
:10643000284606F07FFE03460028C8D1742D00F0E0
:10644000FB80772D0DD13268716891421EBF531CBD
:1064500033601178434A08BF1946204625F0DCFC1A
:10646000B5E7F52D01F0E983762D00F0DB81472DAE
:1064700000F0848270683268292DA0EB020100F0E0
:10648000518340F25982392D00F03A83532D40F068
:106490006983531C33601078032800F28985431EFA
:1064A000314D324ADBB203EB430305EB430310707B
:1064B0005D7800288BD04B1EDBB2AB4240F0788574
:1064C0000021C2F80610C2F8021091725BB1591C8B
:1064D0003368114401320133336013F8010C02F8C0
:1064E000010F8A42F7D1224B1B78002B3FF46FAF8C
:1064F000012521F095FE2B4650E7202D97D10B6802
:106500001C4D591C6A7821601A7023682A78591C1E
:1065100021601A702368AA78591C21601A70298991
:106520002046FFF702F923686A79591C21601A7026
:106530002268A979F9E600BF1D99002064250408A6
:10654000FC2700202E9C0020236200204099002080
:10655000107AFF1F147AFF1F187AFF1F6C63002048
:10656000505C0408BDAF0308BC2C0408B8760020BA
:1065700053280020B8510020676666662428002052
:10658000822D7FF454AF0B68BA4ABB4D1178BB4AD9
:10659000581C2060197011892046FFF7C6F8B84BC7
:1065A00022681B88FF2B02F10101A8BFFF23216095
:1065B0001370A96881F3100189B22046FFF7B5F87E
:1065C000296801F30F0189B22046FFF7AEF8AD4B01
:1065D00022681978A9E6012D7FF429AF0B68002203
:1065E000591C21601A7023685A1C22601D70226891
:1065F0002521531C23602B461170CFE6522D7FF4CA
:1066000016AF0A68A04D531C0321236005F10C0E40
:1066100011702B46062001212268561C266011703D
:1066200022689E4502F101012160107000F0DB80BC
:106630009979D8790633EFE73268716891421EBFC5
:10664000531C33601178914A08BF1946204625F043
:10665000E3FBBCE60B685A1C0A601D700B685A1CF1
:106660000A601D705FE6864B0A681B88824DFF2B0F
:10667000A8BFFF23511C21601370A96881F310018A
:1066800089B22046FFF751F8814B20461988FFF761
:106690004CF8296801F30F0189B220460125FFF764
:1066A00044F82B467AE60B227A492046FEF7F8FF9B
:1066B000082279492046FEF7F3FF01250722774992
:1066C0002046FEF7EDFF2B4668E6002A3FF47FAE3A
:1066D000734B136001252B4660E60B68DFF8E491ED
:1066E000704E591C022221601A7023684FF0060870
:1066F0005A1C226083F8008023680A22591C2160FA
:106700001A70236801255A1922601D70B9F800100B
:106710002046FFF70AF8B9F802102046FFF705F8FF
:1067200023685A19226083F800802368502259197F
:1067300021601A7023680022591921601A7031886B
:106740002046FEF7F2FF71882046FEF7EEFF2B464B
:1067500024E6554B4EE6554B1E78033616F0FF06E1
:106760003FF435AE524BDFF860811E4403F1010A5D
:106770004FF00A091FE0B9F1500F78D0B9F1320F8C
:1067800000F0BF80A9F13C00C0B2132840F2BC80E9
:106790000025294623685A1C2260204683F8009071
:1067A000FEF7C3FF29462046FEF7BFFFB2453FF480
:1067B0000EAE1AF8019BB9F10A0FDCD13D4B9D6872
:1067C000196805EB85054FF6FF736D009D42A8BF64
:1067D0001D469942A8BF194625EAE57521EAE171EF
:1067E000ADB289B2D6E7344B21681A78481C2060D4
:1067F0000A70002A3FF4EBAD013AD2B202EB42023A
:1068000005EB42025578002D3FF4E1AD01351D4402
:106810000133226813F8011F501C9D422060117043
:10682000F7D1D4E53268511C31601278002A01F0AA
:10683000EA82102A01F01F831E46194625686B1C48
:10684000236020462A70FEF759FF31462046FEF7A6
:1068500055FF1A4B20461968FEF750FF20460021CD
:10686000FEF763FF00212046FEF75FFF5BE5144B58
:10687000A5E700BF2E9A0020F04F0020B85100205D
:10688000189A00201D470020BC2C040829B00308DA
:10689000B0510020585C0408645C0408705C040873
:1068A00015D10108E42700209C4500201D990020F7
:1068B00074250408B0270020B8760020DC260020CC
:1068C000E82700202C6E0020F42700203388FF2BBF
:1068D000A8BFFF23DBB2F8E426F09CF800283FF4C1
:1068E000F3AC03780A2B25D8B0F9023088FB0312E9
:1068F000DB17C3EBA2039BB2FF2BA8BFFF23DBB2C6
:10690000E3E498E822005CE726F084F800283FF4EE
:106910003FAF03780A2B3FF63BAFB0F90430B0F934
:10692000061003EB830383F3500521EAE171ADB256
:1069300089B22FE70023E2E7212D40F013811346AF
:10694000511C3160834D13F8021B6970336053781A
:106950002B70D31C33609378AB703046FEF790FEFB
:1069600033682881591C1A46316012F8021B69717C
:1069700032605B78AB7101252B460FE57268356894
:106980007B623046551BFEF764FE052D38627B6A3C
:1069900001F216828026B346012594E80600521AB9
:1069A000103A9642C8BF1FFA82FB6B4A396A926856
:1069B0003A61521A9345396A7B622046FA6088BF71
:1069C0001FFA82FBFEF79AFE7B6A002B01F0D7814B
:1069D000002D41F0B3812368C7F800D05D71C0B0CD
:1069E0000533C7F808D0FB61BBF1000F01F05F82EF
:1069F0003B6A3A69934281F05682AA463E6A7D62BA
:106A00007C6080255446FB681C1B534BB4F5807F8B
:106A100028BF4FF480749B68A2199A4288BF9C1BC0
:106A2000FFF774FB2246BC6830462146F3F76EFB45
:106A3000F969B86104EB000C0B787B6164452ED2D8
:106A4000DFF818910CF1FF3C04F1FF3E1EF8013F06
:106A500009EB830219F823405688ECB100234FF468
:106A6000004204F1FF3816424FEA520202D0087881
:106A7000284308706D0806D10AF1010A4D701FFA0B
:106A80008AFA01318025D34503D8F44532D8984598
:106A900030DC01339C42E6D1F445D7D1F9617B6A01
:106AA000BA6913449BB2D3457B6206D97B6A3A6AC2
:106AB0001C46D6183B699E42A5D37C68802D1CBF1E
:106AC0000AF101031FFA83FA0AF1020189B2204692
:106AD000FEF72BFE2368796A01255A1922602046A9
:106AE0001D70FEF722FE2368534423602B46D7F81F
:106AF00000D053E4FB697C681A463B7D1370DDE7E8
:106B0000531C336013780A2B01F06E813046FEF778
:106B1000C2FD3046FEF7BFFD01253046FEF7BBFD46
:106B20002B463BE4531C336013780A2B01F055814C
:106B3000502B40F0A7863046FEF7A2FDDFF82080FC
:106B4000A8F800003046FEF79BFD0125A8F80200DA
:106B50002B4623E4B8510020A01A00208425040805
:106B6000E42700200B3DEF2D00F222820FF2040EED
:106B70005EF825F023790108B16F0108B16F0108B3
:106B8000B16F0108B16F0108B16F0108B16F010861
:106B9000B16F0108B16F0108B16F0108B16F010851
:106BA000B16F0108B16F0108B16F0108B16F010841
:106BB000B16F0108B16F0108B16F0108B16F010831
:106BC000B16F0108B16F0108B16F0108B16F010821
:106BD000B16F0108AF780108B16F0108BB790108F6
:106BE000B16F010891790108B16F0108B16F010817
:106BF000B16F0108DD790108B16F0108E177010883
:106C0000B16F0108F77B0108B16F0108D17B010862
:106C1000B16F0108297C0108B16F01084D7B0108A3
:106C2000B16F0108356F0108B16F0108B16F01083C
:106C3000B16F0108B16F0108CF630108B16F01089E
:106C4000A57B0108B16F0108B16F010895780108B3
:106C5000B16F01083B780108B16F0108B16F0108FD
:106C6000B16F0108B16F0108D37A0108B16F010853
:106C7000B16F0108B16F0108937A0108B16F010883
:106C8000457A0108B16F0108B16F0108057A010862
:106C9000B16F0108B16F0108B16F0108B16F010850
:106CA000B16F0108B16F0108B16F0108DF7A010807
:106CB000B16F01086D770108B16F0108FB7601081B
:106CC000B16F01084D760108B16F0108D375010855
:106CD000B575010899750108B16F0108B16F010818
:106CE000B16F0108B16F0108B16F0108B16F010800
:106CF000B16F0108B16F0108B16F0108B16F0108F0
:106D0000B16F0108B16F0108B16F0108B16F0108DF
:106D1000B16F0108B16F0108B16F0108B16F0108CF
:106D2000B16F0108B16F0108B16F0108B16F0108BF
:106D3000B16F0108B16F0108B16F0108B16F0108AF
:106D4000B16F0108B16F0108B16F0108B16F01089F
:106D5000B16F0108B16F0108B16F0108B16F01088F
:106D6000B16F0108B16F0108B16F0108B16F01087F
:106D7000B16F0108B16F0108B16F0108B16F01086F
:106D8000B16F0108B16F0108B16F0108B16F01085F
:106D9000B16F0108B16F0108B16F0108B16F01084F
:106DA000B16F0108B16F0108B16F0108B16F01083F
:106DB000B16F0108B16F0108B16F0108B16F01082F
:106DC000B16F0108B16F0108B16F0108B16F01081F
:106DD000B16F0108B16F0108B16F0108B16F01080F
:106DE000B16F0108B16F0108B16F0108B16F0108FF
:106DF000B16F0108B16F0108B16F0108B16F0108EF
:106E0000B16F0108B16F0108B16F0108B16F0108DE
:106E1000B16F0108B16F0108B16F0108B16F0108CE
:106E2000B16F01086F750108B16F01085375010852
:106E300027750108B16F0108B16F0108B16F010832
:106E4000B16F0108B16F0108B16F0108B16F01089E
:106E5000B16F0108B16F0108B16F0108B16F01088E
:106E6000B16F0108B16F0108C97401087774010896
:106E70003F740108B16F01089D7301088373010815
:106E800067730108B16F01084D730108E1720108D1
:106E9000737201086172010801720108B16F010883
:106EA000D1710108B16F0108B16F0108A771010824
:106EB00079710108657101083D7101081D710108B2
:106EC000F3700108C7700108AF700108B16F0108C5
:106ED000B16F0108B16F0108B16F0108B16F01080E
:106EE000B16F0108B16F0108B16F0108B16F0108FE
:106EF000B16F0108B16F0108B16F0108B16F0108EE
:106F0000B16F01088F700108B16F0108B16F0108FE
:106F100037700108B16F0108B16F0108B16F010846
:106F2000D36F0108B16F0108B16F0108B16F01089B
:106F3000BB6F01080723B1FBF3F3C3EBC300091ACE
:106F400036D1DBB203F1FF385FFA88F8002B3FF44B
:106F50003EAA08F101080D461FE080F802A0304665
:106F6000FEF78EFB3368A9F800001A46591C316001
:106F700012F8021B89F8031032605A7889F804204D
:106F8000DA1C32609A7889F806201A1D3260DB78A4
:106F900089F8053045453FF41AAA531C336092F92D
:106FA00000A0504624F022FC013581460028D4D1AF
:106FB0004FF0FF352B46FFF7F1B9B84B1B78DB07D5
:106FC000F6D40125F5F70AF8F5F7E2F92B46FFF7B5
:106FD000E5B93046FEF754FB3368B8851A46591CAC
:106FE000316012F8021B326087F82E105A7887F849
:106FF0002F20DA1C32609A7887F830201A1D326010
:10700000DA7887F831205A1D32601B7987F83230E0
:1070100007F12C000023BB86FEF78CFAA04AA14B97
:107020001268801A4FF0010561F10001C3E9060101
:107030002B46FFF7B3B9531C336013780F2BB7D827
:10704000911C3160C3EBC30397495078C854D01CDE
:1070500030600B4491785970111D3160D17899706E
:10706000511D31601179D970911D316051791971BB
:10707000D11D31609179597102F108013160D279E5
:107080009A7101250FF0B0F82B46FFF787B930460B
:10709000FEF7F6FADFF82082A8F80E003046FEF779
:1070A000EFFA0125A8F80C002B46FFF777B9304618
:1070B000FEF7E6FA7D4A00EB8000430001251380CD
:1070C0002B46FFF76BB91146531C3360784B11F810
:1070D000020B1870316051785970D11C3160917871
:1070E0009970111D3160D278DA7001252B46FFF7B7
:1070F00055B93046FEF7C4FADFF8D481A8F810007D
:107100003046FEF7BDFAA8F812003046FEF7B8FA8E
:107110000125A8F814002B46FFF740B91346511C6F
:10712000316013F8020B3360D31C517833609278CE
:1071300017F0B8FC00287FF44AA939E71346511C20
:1071400031605C4913F8020B087033605A49537878
:107150008B70D31C3360554B92789A7001252B4667
:10716000FFF71CB9554B564918684E22012529F0E6
:10717000C7FF2B46FFF712B91146531C3360514B22
:1071800011F8020B1870316051785970D11C3160C0
:1071900092789A703046FEF773FA4B4B0125D880EF
:1071A0002B46FFF7FBB83046FEF76AFADFF8188186
:1071B000A8F800003046FEF763FAA8F8020030464F
:1071C000FEF75EFA0125A8F804002B46FFF7E6B8A3
:1071D000DFF8009199F80030002B3FF4F8A8DFF8B1
:1071E000F88000253046FEF74BFA1BF07BFE99F83D
:1071F0000030A8EC010A01359D42F3DBFFF7E7B848
:107200000D297FF4D5AE531C33601578072D3FF65A
:10721000CFAEDFF8C89030464FF00C08FEF730FADA
:1072200008FB05F809EB0805A8803046FEF728FAA8
:10723000E8803046FEF724FA336828811A46591C44
:10724000316012F8021BA97232605B78EB72304633
:10725000FEF7FFF9012549F808002B46FFF79EB815
:107260003046FEF70DFA194B012518802B46FFF723
:1072700095B8531C33601078060600F19C86074BC6
:107280001B78DD073FF5A3A8032828BF00200125B0
:10729000F4F788FE2B46FFF781B800BF006200209C
:1072A0003C850020E0240020B04400204C6E0020EB
:1072B0004C4700209C8D00203C6E0020285200206E
:1072C000044C0408346E0020846B0020684A0020BF
:1072D000C08F00201D99002084420020F043002030
:1072E000531C3360304692F800A0FEF7B2F9814695
:1072F0003046FEF7AEF905463046FEF7AAF980465D
:107300003046FEF7BDF93046FEF7BAF93046FEF7D3
:10731000C2F9BAF1000F00F03786BAF1100F7FF40E
:1073200056A8B64BC3F804909D60B8F1000F02D088
:10733000B34BC3F80080B349B34B0222081F0125A9
:107340001A701EF06DFF2B46FFF728B8AF4B1B7865
:10735000D8073FF53CA80125F5F7F0F9F5F718F83F
:107360002B46FFF71BB8A94B1B78DA073FF52FA870
:10737000A74A1378012543F0040313702B46FFF747
:107380000DB8A24B1B78D9073FF521A8A14B4FF4AC
:10739000C87201251A802B46FFF700B809297FF72C
:1073A00007AEDFF8A0821346511CD8F800503160B8
:1073B00013F8021B297033605378AB70D31C336011
:1073C0009378642B02F10401A8BF64236B713160D0
:1073D000D378642B02F10501A8BF6423AB7131603F
:1073E0001379EB71931D33605379642B02F107011C
:1073F000A8BF64232B7231609379EB7002F108030C
:107400003360D3792B713046FEF73AF972683368EE
:107410006881D11A00290CDD591CD8F800003160B0
:10742000521A002A1978417203DD9A1C32605B7887
:10743000437001251CF050FB2B46FEF7AFBF764B87
:107440001868D31C014621329D1E356013F8035C79
:107450000D705D1E356013F8025C4D70336013F8DB
:10746000015C8D7003339A4201F10301ECD11BF0F2
:10747000E3FBFEF7ACBF531C336013786449002B69
:1074800000F01A850B7843F00203901C0B70634DDB
:10749000306053782B753046FEF7DBF828603046B5
:1074A000FEF7D7F868603046FEF7EAF828813046E4
:1074B000FEF7E6F85A4AE8811378012543F0020303
:1074C00013702B46FEF76ABFC1F34705122D3FF636
:1074D0006FADC5B107F1500307F12A0903EB450A67
:1074E000C846AAF1260A3046FEF7CAF828F8020F65
:1074F000D045F8D14B4B39F8022F23F8022FC8455D
:10750000F9D1112D09D8484A6B00023B13440021E0
:10751000223223F8021F9A42FBD1444A01231D461E
:107520001370FEF73BBF531C41483360017813785A
:10753000002900F0C68404297EF449AF3D4A9B002F
:107540001380F5F7B1FE2D4B012518622B46FEF78F
